S01800004762544D6F64756C65535733305765622E737265637E
S315080080000000012081E7000885DF00088DDF0008F1
S3150800801095DF00089DDF0008A5DF000800000000C6
S31508008020000000000000000000000000ADDF0008AE
S31508008030B9DF000800000000C5DF0008D1DF00082E
S31508008040D1E70008D1E70008D1E70008D1E7000822
S31508008050D1E70008D1E70008D1E70008D1E7000812
S31508008060D1E70008D1E70008D1E70008D1E7000802
S31508008070D1E70008D1E70008D1E70008D1E70008F2
S31508008080D1E70008D1E70008D1E70008D1E70008E2
S31508008090DDDF0008D1E70008D1E70008D1E70008CE
S315080080A0D1E70008D1E70008D1E70008D1E70008C2
S315080080B0D1E70008D1E70008D1E70008D1E70008B2
S315080080C0D1E70008D1E70008D1E70008D1E70008A2
S315080080D0D1E70008F1DF000805E0000819E000080C
S315080080E0D1E70008D1E70008D1E700080000000042
S315080080F00000000000000000000000000000000072
S315080081000000000000000000D1E70008D1E70008E1
S31508008110D1E700082DE00008D1E70008D1E70008FC
S31508008120D1E70008D1E70008D1E70008D1E7000841
S31508008130D1E70008D1E70008D1E7000841E00008C8
S31508008140D1E7000855E00008D1E70008D1E70008A4
S315080081500000000000000000000000000000000011
S315080081600000000000000000000000000000000001
S3150800817000000000000000000000000000000000F1
S3150800818000000000000000000000000000000000E1
S3150800819000000000000000000000000000000000D1
S315080081A000000000000000000000000000000000C1
S315080081B000000000000000000000000000000000B1
S315080081C000000000000000000000000000000000A1
S315080081D00000000000000000000000000000000091
S30D080081E05FF8E0F166666666C9
S315080081E810B5054C237833B9044B13B10448AFF3DB
S315080081F800800123237010BD5002002000000000F3
S315080082080865010808B5034B1BB103490348AFF3D2
S31508008218008008BD00000000540200200865010817
S31508008228034613F8012B002AFBD1181A01387047A0
S3150800823881F0004102E000BF83F0004330B54FEA01
S3150800824841044FEA430594EA050F08BF90EA020F6E
S315080082581FBF54EA000C55EA020C7FEA645C7FEA01
S31508008268655C00F0E2804FEA5454D4EB5555B8BF24
S315080082786D420CDD2C4480EA020281EA030382EA95
S31508008288000083EA010180EA020281EA0303362D27
S3150800829888BF30BD11F0004F4FEA01314FF4801CFA
S315080082A84CEA113102D0404261EB410113F0004F0C
S315080082B84FEA03334CEA133302D0524263EB4303C3
S315080082C894EA050F00F0A780A4F10104D5F1200E61
S315080082D80DDB02FA0EFC22FA05F2801841F10001BC
S315080082E803FA0EF2801843FA05F359410EE0A5F190
S315080082F820050EF1200E012A03FA0EFC28BF4CF0C1
S31508008308020C43FA05F3C01851EBE37101F0004576
S3150800831807D54FF0000EDCF1000C7EEB00006EEB83
S315080083280101B1F5801F1BD3B1F5001F0CD349080D
S315080083385FEA30004FEA3C0C04F101044FEA445264
S3150800834812F5800F80F09A80BCF1004F08BF5FEAEB
S31508008358500C50F1000041EB045141EA050130BDCB
S315080083685FEA4C0C404141EB0101013C28BFB1F5DD
S31508008378801FE9D291F0000F04BF01460020B1FA28
S3150800838881F308BF2033A3F10B03B3F120020CDAFB
S315080083980C3208DD02F1140CC2F10C0201FA0CF0D9
S315080083A821FA02F10CE002F11402D8BFC2F1200C3E
S315080083B801FA02F120FA0CFCDCBF41EA0C019040F4
S315080083C8E41AA2BF01EB0451294330BD6FEA04043D
S315080083D81F3C1CDA0C340EDC04F11404C4F1200228
S315080083E820FA04F001FA02F340EA030021FA04F33A
S315080083F845EA030130BDC4F10C04C4F1200220FA91
S3150800840802F001FA04F340EA0300294630BD21FACE
S3150800841804F0294630BD94F0000F83F4801306BF94
S3150800842881F480110134013D4EE77FEA645C18BF88
S315080084387FEA655C29D094EA050F08BF90EA020F1F
S3150800844805D054EA000C04BF1946104630BD91EA17
S31508008458030F1EBF0021002030BD5FEA545C05D11A
S315080084684000494128BF41F0004130BD14F5800459
S315080084783CBF01F5801130BD01F0004545F0FE41CD
S3150800848841F470014FF0000030BD7FEA645C1ABF02
S31508008498194610467FEA655C1CBF0B46024650EA39
S315080084A8013406BF52EA033591EA030F41F4002165
S315080084B830BD00BF90F0000F04BF0021704730B5EB
S315080084C84FF4806404F132044FF000054FF00001C0
S315080084D850E700BF90F0000F04BF0021704730B581
S315080084E84FF4806404F1320410F0004548BF404256
S315080084F84FF000013EE700BF42004FEAE2014FEAAB
S3150800850831014FEA02701FBF12F07F4393F07F4F85
S3150800851881F06051704732F07F4208BF704793F088
S315080085287F4F04BF41F40021704730B54FF460749B
S3150800853801F0004521F000411CE700BF50EA01029E
S3150800854808BF704730B54FF000050AE050EA010247
S3150800855808BF704730B511F0004502D5404261EBB7
S3150800856841014FF4806404F132045FEA915C3FF4F8
S31508008578D8AE4FF003025FEADC0C18BF03325FEA95
S31508008588DC0C18BF033202EBDC02C2F1200300FA46
S3150800859803FC20FA02F001FA03FE40EA0E0021FA6B
S315080085A802F11444BDE600BF70B54FF0FF0C4CF459
S315080085B8E06C1CEA11541DBF1CEA135594EA0C0F0B
S315080085C895EA0C0F00F0DEF82C4481EA030621EA46
S315080085D84C5123EA4C5350EA013518BF52EA033581
S315080085E841F4801143F4801338D0A0FB02CE4FF033
S315080085F80005E1FB02E506F00042E0FB03E54FF063
S315080086080006E1FB03569CF0000F18BF4EF0010E5A
S31508008618A4F1FF04B6F5007F64F5407404D25FEA56
S315080086284E0E6D4146EB060642EAC62141EA555109
S315080086384FEAC52040EA5E504FEACE2EB4F1FD0C4B
S3150800864888BFBCF5E06F1ED8BEF1004F08BF5FEAC9
S31508008658500E50F1000041EB045170BD06F000467B
S3150800866846EA010140EA020081EA0301B4EB5C0428
S31508008678C2BFD4EB0C0541EA045170BD41F4801120
S315080086884FF0000E013C00F3AB8014F1360FDEBF45
S31508008698002001F0004170BDC4F10004203C35DA21
S315080086A80C341BDC04F11404C4F1200500FA05F3A4
S315080086B820FA04F001FA05F240EA020001F0004245
S315080086C821F0004110EBD37021FA04F642EB0601BB
S315080086D85EEA430E08BF20EAD37070BDC4F10C04E5
S315080086E8C4F1200500FA04F320FA05F001FA04F2A9
S315080086F840EA020001F0004110EBD37041F1000195
S315080087085EEA430E08BF20EAD37070BDC4F120059F
S3150800871800FA05F24EEA020E20FA04F301FA05F207
S3150800872843EA020321FA04F001F0004121FA04F2AF
S3150800873820EA020000EBD3705EEA430E08BF20EA7F
S31508008748D37070BD94F0000F0FD101F000464000B9
S3150800875841EB010111F4801F08BF013CF7D041EA3B
S31508008768060195F0000F18BF704703F0004652003F
S3150800877843EB030313F4801F08BF013DF7D043EA10
S315080087880603704794EA0C0F0CEA135518BF95EAC6
S315080087980C0F0CD050EA410618BF52EA4306D1D14D
S315080087A881EA030101F000414FF0000070BD50EA6C
S315080087B8410606BF1046194652EA430619D094EAF6
S315080087C80C0F02D150EA013613D195EA0C0F05D1E0
S315080087D852EA03361CBF104619460AD181EA030134
S315080087E801F0004141F0FE4141F470014FF00000EC
S315080087F870BD41F0FE4141F4780170BD70B54FF087
S31508008808FF0C4CF4E06C1CEA11541DBF1CEA135506
S3150800881894EA0C0F95EA0C0F00F0A7F8A4EB0504E8
S3150800882881EA030E52EA03354FEA013100F08880DF
S315080088384FEA03334FF0805545EA131343EA1263A8
S315080088484FEA022245EA111545EA10654FEA00265D
S315080088580EF000419D4208BF964244F1FD0404F516
S31508008868407402D25B084FEA3202B61A65EB030572
S315080088785B084FEA32024FF480104FF4002CB6EB2F
S31508008888020E75EB030E22BFB61A754640EA0C00AF
S315080088985B084FEA3202B6EB020E75EB030E22BFEF
S315080088A8B61A754640EA5C005B084FEA3202B6EB30
S315080088B8020E75EB030E22BFB61A754640EA9C00EF
S315080088C85B084FEA3202B6EB020E75EB030E22BFBF
S315080088D8B61A754640EADC0055EA060E18D04FEA7D
S315080088E8051545EA16754FEA06164FEAC30343EA1D
S315080088F852734FEAC2025FEA1C1CC0D111F4801FEA
S315080089080BD141EA00014FF000004FF0004CB6E7E2
S3150800891811F4801F04BF01430020B4F1FD0C88BF81
S31508008928BCF5E06F3FF6AFAEB5EB030C04BFB6EB8C
S31508008938020C5FEA500C50F1000041EB045170BD7F
S315080089480EF0004E4EEA113114EB5C04C2BFD4EBAC
S315080089580C0541EA045170BD41F480114FF0000E30
S31508008968013C90E645EA060E8DE60CEA135594EAAC
S315080089780C0F08BF95EA0C0F3FF43BAF94EA0C0FAF
S315080089880AD150EA01347FF434AF95EA0C0F7FF424
S3150800899825AF104619462CE795EA0C0F06D152EA78
S315080089A803353FF4FDAE1046194622E750EA41065C
S315080089B818BF52EA43067FF4C5AE50EA41047FF46D
S315080089C80DAF52EA43057FF4EBAE12E74FF0FF3CD2
S315080089D806E000BF4FF0010C02E000BF4FF0010CA3
S315080089E84DF804CD4FEA410C7FEA6C5C4FEA430C1C
S315080089F818BF7FEA6C5C1BD001B050EA410C0CBF6B
S31508008A0852EA430C91EA030F02BF90EA020F0020CC
S31508008A18704710F1000F91EA030F58BF994208BF33
S31508008A2890422CBFD8176FEAE37040F001007047F0
S31508008A384FEA410C7FEA6C5C02D150EA013C07D147
S31508008A484FEA430C7FEA6C5CD6D152EA033CD3D092
S31508008A585DF8040B704700BF8446104662468C468C
S31508008A681946634600E000BF01B5FFF7B7FF0028BF
S31508008A7848BF10F1000F01BD4DF808EDFFF7F4FFE8
S31508008A880CBF012000205DF808FB00BF4DF808ED73
S31508008A98FFF7EAFF34BF012000205DF808FB00BF96
S31508008AA84DF808EDFFF7E0FF94BF012000205DF8B8
S31508008AB808FB00BF4DF808EDFFF7CEFF94BF01206D
S31508008AC800205DF808FB00BF4DF808EDFFF7C4FF66
S31508008AD834BF012000205DF808FB00BF4FEA410CAF
S31508008AE87FEA6C5C02D150EA013C0AD14FEA430C92
S31508008AF87FEA6C5C02D152EA033C02D14FF00000CF
S31508008B0870474FF0010070474FEA410212F500120C
S31508008B1815D211D56FF47873B3EB625212D94FEAAE
S31508008B28C12343F0004343EA505311F0004F23FA98
S31508008B3802F018BF404270474FF00000704750EAED
S31508008B48013005D111F0004008BF6FF000407047AA
S31508008B584FF00000704700BF4FEA4102B2F1E04308
S31508008B6824BFB3F5001CDCF1FE5C0DD901F0004CFE
S31508008B784FEAC0024CEA5070B2F1004F40EB83004E
S31508008B8808BF20F00100704711F0804F21D113F17A
S31508008B983872BCBF01F00040704741F480114FEAB3
S31508008BA85252C2F11802C2F1200C10FA0CF320FA3C
S31508008BB802F018BF40F001004FEAC1234FEAD32359
S31508008BC803FA0CFC40EA0C0023FA02F34FEA4303C3
S31508008BD8CCE77FEA625307D150EA01331EBF4FF04C
S31508008BE8FE4040F44000704701F0004040F0FE4067
S31508008BF840F40000704700BF80F0004002E000BF64
S31508008C0881F0004142001FBF5FEA410392EA030F61
S31508008C187FEA226C7FEA236C6AD04FEA1262D2EBAB
S31508008C281363C1BFD218414048404140B8BF5B42B0
S31508008C38192B88BF704710F0004F40F4000020F049
S31508008C487F4018BF404211F0004F41F4000121F05F
S31508008C587F4118BF494292EA030F3FD0A2F10102A9
S31508008C6841FA03FC10EB0C00C3F1200301FA03F1E7
S31508008C7800F0004302D5494260EB4000B0F5000F0A
S31508008C8813D3B0F1807F06D340084FEA310102F1C9
S31508008C980102FE2A51D2B1F1004F40EBC25008BF7B
S31508008CA820F0010040EA03007047490040EB000045
S31508008CB8013A28BFB0F5000FEDD2B0FA80FCACF146
S31508008CC8080CB2EB0C0200FA0CF0AABF00EBC25073
S31508008CD852421843BCBFD0401843704792F0000F61
S31508008CE881F4000106BF80F400000132013BB5E7B4
S31508008CF84FEA41037FEA226C18BF7FEA236C21D02A
S31508008D0892EA030F04D092F0000F08BF084670478E
S31508008D1890EA010F1CBF0020704712F07F4F04D15C
S31508008D28400028BF40F00040704712F100723CBF6F
S31508008D3800F50000704700F0004343F0FE4040F499
S31508008D48000070477FEA226216BF08467FEA236357
S31508008D580146420206BF5FEA412390EA010F40F442
S31508008D68800070474FF0000304E000BF10F000438E
S31508008D7848BF40425FEA000C08BF704743F0964375
S31508008D8801464FF000001CE050EA010208BF704790
S31508008D984FF000030AE000BF50EA010208BF704717
S31508008DA811F0004302D5404261EB41015FEA010C2C
S31508008DB802BF84460146002043F0B64308BFA3F124
S31508008DC88053A3F50003BCFA8CF2083AA3EBC25306
S31508008DD810DB01FA02FC634400FA02FCC2F1200225
S31508008DE8BCF1004F20FA02F243EB020008BF20F05C
S31508008DF80100704702F1200201FA02FCC2F12002C2
S31508008E0850EA4C0021FA02F243EB020008BF20EAB6
S31508008E18DC7070474FF0FF0C1CEAD0521EBF1CEAE4
S31508008E28D15392EA0C0F93EA0C0F6FD01A4480EAD2
S31508008E38010C400218BF5FEA41211ED04FF00063BB
S31508008E4843EA501043EA5111A0FB01310CF00040E7
S31508008E58B1F5000F3EBF490041EAD3715B0040EA0D
S31508008E68010062F17F02FD2A1DD8B3F1004F40EBDD
S31508008E78C25008BF20F00100704790F0000F0CF0B0
S31508008E88004C08BF49024CEA502040EA51207F3A74
S31508008E98C2BFD2F1FF0340EAC250704740F400004F
S31508008EA84FF00003013A5DDC12F1190FDCBF00F040
S31508008EB800407047C2F10002410021FA02F1C2F1EE
S31508008EC8200200FA02FC5FEA310040F1000053EA8A
S31508008ED84C0308BF20EADC70704792F0000F00F0D8
S31508008EE8004C02BF400010F4000F013AF9D040EADE
S31508008EF80C0093F0000F01F0004C02BF490011F472
S31508008F08000F013BF9D041EA0C018FE70CEAD1536F
S31508008F1892EA0C0F18BF93EA0C0F0AD030F0004CEF
S31508008F2818BF31F0004CD8D180EA010000F00040A3
S31508008F38704790F0000F17BF90F0004F084691F061
S31508008F48000F91F0004F14D092EA0C0F01D142029B
S31508008F580FD193EA0C0F03D14B0218BF084608D164
S31508008F6880EA010000F0004040F0FE4040F40000AE
S31508008F78704740F0FE4040F4400070474FF0FF0C41
S31508008F881CEAD0521EBF1CEAD15392EA0C0F93EA88
S31508008F980C0F69D0A2EB030280EA010C49024FEADA
S31508008FA8402037D04FF0805343EA111143EA101393
S31508008FB80CF000408B4238BF5B0042F17D024FF44B
S31508008FC8000C8B4224BF5B1A40EA0C00B3EB510F26
S31508008FD824BFA3EB510340EA5C00B3EB910F24BF0F
S31508008FE8A3EB910340EA9C00B3EBD10F24BFA3EB94
S31508008FF8D10340EADC001B0118BF5FEA1C1CE0D15C
S31508009008FD2A3FF650AF8B4240EBC25008BF20F00E
S31508009018010070470CF0004C4CEA50207F32C2BF62
S31508009028D2F1FF0340EAC250704740F400004FF0FF
S315080090380003013A37E792F0000F00F0004C02BF30
S31508009048400010F4000F013AF9D040EA0C0093F0FA
S31508009058000F01F0004C02BF490011F4000F013B54
S31508009068F9D041EA0C0195E70CEAD15392EA0C0FBC
S3150800907808D142027FF47DAF93EA0C0F7FF470AFF4
S31508009088084676E793EA0C0F04D14B023FF44CAF37
S3150800909808466EE730F0004C18BF31F0004CCAD1CC
S315080090A830F000427FF45CAF31F000437FF43CAF08
S315080090B85FE700BF4FF0FF3C06E000BF4FF0010C2A
S315080090C802E000BF4FF0010C4DF804CD4FEA40020C
S315080090D84FEA41037FEA226C18BF7FEA236C11D056
S315080090E801B052EA530C18BF90EA010F58BFB2EB09
S315080090F8030088BFC81738BF6FEAE17018BF40F089
S31508009108010070477FEA226C02D15FEA402C05D13C
S315080091187FEA236CE4D15FEA412CE1D05DF8040BC1
S31508009128704700BF844608466146FFE70FB5FFF754
S31508009138C9FF002848BF10F1000F0FBD4DF808ED0C
S31508009148FFF7F4FF0CBF012000205DF808FB00BFFD
S315080091584DF808EDFFF7EAFF34BF012000205DF857
S3150800916808FB00BF4DF808EDFFF7E0FF94BF0120A4
S3150800917800205DF808FB00BF4DF808EDFFF7D2FFA1
S3150800918894BF012000205DF808FB00BF4DF808EDE4
S31508009198FFF7C8FF34BF012000205DF808FB00BFB1
S315080091A84FEA4002B2F1FE4F0FD34FF09E03B3EBDE
S315080091B812620DD94FEA002343F0004310F0004F1E
S315080091C823FA02F018BF404270474FF00000704774
S315080091D812F1610F01D1420205D110F0004008BF13
S315080091E86FF0004070474FF0000070477BB972B9BE
S315080091F80029BEBF00204FF0004106E008BF00283E
S315080092081CBF6FF000414FF0FF3000F0D7B9ADF141
S31508009218080C6DE904CE002909DB002B1ADB00F0DF
S315080092284DF8DDF804E0DDE9022304B07047404252
S3150800923861EB4101002B1BDB00F040F8DDF804E088
S31508009248DDE9022304B0404261EB4101524263EB77
S3150800925843037047524263EB430300F02FF8DDF8E7
S3150800926804E0DDE9022304B0404261EB410170479E
S31508009278524263EB430300F021F8DDF804E0DDE928
S31508009288022304B0524263EB4303704753B94AB901
S31508009298002908BF00281CBF4FF0FF314FF0FF30E8
S315080092A800F08CB9ADF1080C6DE904CE00F006F8AB
S315080092B8DDF804E0DDE9022304B070472DE9F0473C
S315080092C8089D8E4604468846002B4AD18A42174688
S315080092D862D9B2FA82F64EB1C6F1200301FA06F847
S315080092E820FA03F3B74043EA0808B4404FEA174E92
S315080092F8B8FBFEF11FFA87FC0EFB118801FB0CF27E
S31508009308230C43EA08439A4209D9FB1801F1FF30AE
S3150800931880F0EB809A4240F2E88002393B449A1A78
S31508009328B2FBFEF00EFB102200FB0CFCA3B243EACC
S3150800933802439C4509D9FB1800F1FF3280F0D78013
S315080093489C4540F2D4803B44023840EA014000215B
S31508009358A3EB0C031DB10022F340C5E90032BDE8B2
S31508009368F0878B4205D90DB1C5E9000100210846E9
S31508009378F5E7B3FA83F1002946D1734502D3824249
S3150800938800F20881841A6EEB030201209046002D2C
S31508009398E5D0C5E90048E2E7002A00F09180B2FA6C
S315080093A882F6002E40F0A5808A1A0121030C4FEA9E
S315080093B8174E80B2BCB2B2FBFEFC0EFB1C2243EA77
S315080093C8024304FB0CF29A4207D9FB180CF1FF3842
S315080093D802D29A4200F2E380C4469B1AB3FBFEF215
S315080093E80EFB123302FB04F440EA03439C4207D9F6
S315080093F8FB1802F1FF3002D29C4200F2CD800246E9
S315080094081B1B42EA0C40A5E7C1F120068B4022FA4D
S3150800941806F71F432EFA06FA4FEA1749BAFBF9F870
S315080094280EFA01FE20FA06F309FB18AA1FFA87FCAA
S3150800943843EA0E0300FA01FE08FB0CF01C0C44EA8A
S315080094480A44A04202FA01F20AD93C1908F1FF3A7D
S3150800945880F09E80A04240F29B80A8F102083C4416
S31508009468241A98B2B4FBF9F309FB134403FB0CFC62
S3150800947840EA0444A44509D93C1903F1FF3080F0B1
S315080094888580A44540F28280023B3C4443EA084072
S31508009498A4EB0C04A0FB028C64454346E14664D35E
S315080094A861D05DB1BEEB030264EB090404FA06F663
S315080094B822FA01F31E43CC40C5E9006400214EE7B1
S315080094C8B1FBF2FC010C41EA0E4180B240EA0142C6
S315080094D83B46B1FBF7F138463C46B846BE46202619
S315080094E8A2EB080241EA0C4165E7014617E7104670
S315080094F82BE7C6F120012EFA01FCB7400EFA06FE44
S3150800950820FA01F141EA0E014FEA174EBCFBFEF8B4
S31508009518BCB20EFB18CC08FB04F90A0C42EA0C424A
S31508009528B04091454FEA104380B23ED9BA1808F1BF
S31508009538FF3C01D291451FD8A2EB0902B2FBFEF9FE
S3150800954809FB04F80EFB192A8AB242EA0A4242457E
S3150800955829D2BA1809F1FF31C2D24245C0D2A9F1B7
S3150800956802013A44BCE7C6459BD2B8EB02036CEB4A
S31508009578070C0138E14694E7A7EB09094A44B2FB08
S31508009588FEF9A8F1020C09FB04F8DBE703467DE7B8
S31508009598D04665E70846FAE63B44023A30E7ACF1B6
S315080095A8020C3B4419E749469AE7A2EB0902B2FBC3
S315080095B8FEF9C44609FB04F8C4E700BF704700BFB4
S315080095C880B584B000AF3B1D00221A605A609A60C5
S315080095D8184B194A1A60174B00229A60154B002235
S315080095E81A73144B00221A75124B4FF46022DA616B
S315080095F8104B00225A600F4B01221A610D4805F0DC
S315080096086BF90346002B01D002F0C2FE08237B60E3
S315080096180123BB600023FB603B1D1946054805F07E
S315080096281FFC0346002B01D002F0B2FE00BF10371C
S31508009638BD4680BD6C0200200024014080B58AB072
S3150800964800AF786007F1180300221A605A609A601A
S31508009658DA607B681B681F4A934237D11E4B9B69A1
S315080096681D4A43F4007393611B4B9B6903F400730B
S315080096787B617B69184B9B69174A43F0040393611E
S31508009688154B9B6903F004033B613B69124B9B69C5
S31508009698114A43F0080393610F4B9B6903F00803CB
S315080096A8FB60FB680823BB610323FB6107F118030A
S315080096B819460A4806F04EFF0323BB610323FB61DC
S315080096C807F118031946064806F044FF00BF28376D
S315080096D8BD4680BD00240140001002400008014034
S315080096E8000C014080B582B000AF03460A46FB71FC
S315080096F81346BB71FB79062B47D801A252F823F00B
S3150800970825970008359700084597000855970008D3
S31508009718659700087597000885970008BB791A4663
S315080097284FF480711D4807F0B0F82FE0BB791A4648
S315080097384FF40071194807F0A8F827E0BB791A46CC
S315080097484FF48061154807F0A0F81FE0BB791A4660
S315080097584FF40061114807F098F817E0BB791A46E4
S315080097684FF480510D4807F090F80FE0BB791A4678
S315080097784FF400410A4807F088F807E0BB791A460B
S315080097880821084807F081F800E000BFFB79064978
S31508009798BA79CA5400BF0837BD4680BD00180140CB
S315080097A800080140001401409C02002080B483B0E0
S315080097B800AF0346FB71FB79034AD35C18460C379E
S315080097C8BD4680BC704700BF9C02002080B582B0A9
S315080097D800AF0346FB71FB79062B3BD801A252F86A
S315080097E823F000BF09980008159800082198000872
S315080097F82D980008399800084598000851980008D7
S315080098080221174807F02AF8034624E004211448D9
S3150800981807F024F803461EE08021124807F01EF8D0
S31508009828034618E08021104807F018F8034612E0A6
S3150800983810210E4807F012F803460CE008210B48D9
S3150800984807F00CF8034606E00221064807F006F872
S31508009858034600E0002318460837BD4680BD00BF0A
S31508009868000801400018014000140140000C01409E
S3150800987880B500AF104805F087FC00210020FFF7E7
S3150800988831FF00210120FFF72DFF00210220FFF7F5
S3150800989829FF00210320FFF725FF00210420FFF7F1
S315080098A821FF01210520FFF71DFF00210620FFF7EC
S315080098B819FF00BF80BD00BF6C02002090B587B0B5
S315080098C800AF78600C4B7B610C4B3B617969786813
S315080098D8FFF796F903461C4639697869FFF79AFA35
S315080098E8034619462046FFF749FB0346FB60FB6813
S315080098F818461C37BD4690BD00007A443211803B95
S31508009908B0B586B000AFF860B9607A603B60F868B1
S31508009918FEF7E0FD1CA3D3E90023FEF76FFF024616
S315080099280B4614461D46B868FEF7E6FD02460B4682
S3150800993820462946FEF738FE02460B4610461946C3
S31508009948FFF70AF903467B6179687869FFF714FC1B
S315080099580346002B01D00E4B10E079697868FFF7AB
S315080099684FF9034619467869FFF708FB034619466F
S315080099783868FFF74FFA03463B613B6918461837BC
S31508009988BD46B0BDAFF300800000000000FEAF4042
S31508009998000080BF80B588B000AF0346FB71FB792D
S315080099A8002B03D0082000F03BF802E0092000F05D
S315080099B837F8174805F068F84FF0FF31144805F0EE
S315080099C83DF9134805F040FAF861114805F00AF917
S315080099D8FB69B3F57A6F01D9142315E00D4BBB6102
S315080099E80D4B7B610D4B3B61F8693B697A69B9692F
S315080099F8FFF786FF03461846FFF760FFF860F86822
S31508009A08FFF7CEFB03461BB218462037BD4680BD76
S31508009A186C020020333353400000A04000007A440B
S31508009A2880B586B000AF78607B68FB6001233B6130
S31508009A3803237B6107F10C031946064805F010FA5B
S31508009A480346002B01D002F0A3FC00BF1837BD4619
S31508009A5880BD00BF6C02002080B500AF174B184ABE
S31508009A681A60164B08225A60144B00229A60134B48
S31508009A780022DA60114B4FF460221A610F4B4FF43B
S31508009A8880125A610D4B00221A760C4B01225A761F
S31508009A980A4B01229A76094B0122DA76074B0022ED
S31508009AA81A77064B01225A77044805F01BFC034629
S31508009AB8002B01D002F06CFC00BF80BDA402002078
S31508009AC80064004080B500AF174B184A1A60164B59
S31508009AD810225A60144B00229A60134B0022DA604F
S31508009AE8114B4FF460221A610F4B4FF480125A61DA
S31508009AF80D4B00221A760C4B01225A760A4B012284
S31508009B089A76094B0122DA76074B00221A77064B12
S31508009B1801225A77044805F0E5FB0346002B01D0D5
S31508009B2802F036FC00BF80BDCC0200200068004069
S31508009B3880B58EB000AF786007F1200300221A605E
S31508009B485A609A60DA607B681B68614A934253D107
S31508009B58604B1B6801335F4A13605E4B1B68012B19
S31508009B680BD15D4BDB695C4A43F00073D3615A4BF2
S31508009B78DB6903F00073FB61FB69574B9B69564A1F
S31508009B8843F020039361544B9B6903F02003BB61A0
S31508009B98BB6901233B6200237B620023BB6207F192
S31508009BA8200319464D4806F0D5FC02233B620223DA
S31508009BB87B620323FB6207F120031946474806F030
S31508009BC8C9FC474B5B683B633B6B23F4C0433B6369
S31508009BD83B6B43F0E0633B633B6B43F4C0433B6337
S31508009BE83F4A3B6B536000220021142006F01DFBF8
S31508009BF8142006F036FB67E07B681B68394A9342EF
S31508009C0862D1354BDB69344A43F08063D361324B02
S31508009C18DB6903F080637B617B692E4B1B68013324
S31508009C282C4A13602B4B1B68012B0BD12A4BDB697B
S31508009C38294A43F00073D361274BDB6903F00073A5
S31508009C483B613B69244B9B69234A43F008039361AC
S31508009C58214B9B6903F00803FB60FB6820233B62E2
S31508009C6800237B620023BB6207F1200319461E48BE
S31508009C7806F070FC40233B6202237B620323FB62E7
S31508009C8807F120031946184806F064FC144B5B686C
S31508009C987B637B6B43F0E0637B637B6B43F48003F6
S31508009CA87B630F4A7B6B5360002200213F2006F036
S31508009CB8BCFA3F2006F0D5FA00220021412006F01A
S31508009CC8B4FA412006F0CDFA00BF3837BD4680BD44
S31508009CD800640040F402002000100240001401400D
S31508009CE80000014000680040000C014080B400AF45
S31508009CF8084B00221A70074B00225A70054B00229F
S31508009D0862F06902DA7300221A7400BFBD4680BC85
S31508009D18704700BFF802002080B500AF1E4B5A787E
S31508009D281E4B1B789A4206D01B4B5A781B4B1A7047
S31508009D38194B00221A701A4B5B78002B03D0164B66
S31508009D4804225A7716E0174B1B7B002B03D0124BBD
S31508009D5807225A770EE0134B5B7B002B03D00E4B7A
S31508009D680A225A7706E00C4B9B7F002B02D10A4B36
S31508009D7800225A77084B5B7F0021184602F0B6F98D
S31508009D880346002B06D0044B5B7F1A46002106487B
S31508009D980AF0C2F900BF80BDF802002017030020A8
S31508009DA8080000200C0A00202065010880B500AFCD
S31508009DB80B4B10221A7000F077FF0A4B42F210720A
S31508009DC81A80084B40F2DC525A80064B40F6B832E5
S31508009DD89A80044B40F69672DA8000BF80BD00BFB1
S31508009DE8180300203003002080B500AF0C4BD3F8C9
S31508009DF80730184603F048FF094B1A78094B5A7179
S31508009E08074B5A78074B9A71054B9A78054BDA71BE
S31508009E18034BD3F80330034AC2F8013000BF80BDAC
S31508009E286C00002038030020B0B584B002AFAB4BF5
S31508009E3893F80A31022B40F0D180A84BD3F80031A9
S31508009E48B3F51C5F47D0B3F51C5F00F2C380B3F5C2
S31508009E58E05F00F0B680B3F5E05F00F2BB80B3F5CB
S31508009E68B85F00F0B280B3F5B85F00F2B380B3F517
S31508009E78B05F00F0AC80B3F5B05F00F2AB80B3F525
S31508009E88A85F00F0A680B3F5A85F00F2A380B3F533
S31508009E98985F00F08680B3F5985F00F29B80B3F56B
S31508009EA8885F6FD0B3F5885F00F29480B3F5805F5A
S31508009EB846D0B3F5805F00F28D80B3F5106F2CD0CD
S31508009EC8B3F5106F00F28680B3F5007F0BD0B3F5B3
S31508009ED8C06F18D07EE0824B01221A707F4B1A8811
S31508009EE8804B1A8076E0804B01221A707F4A7B4B9A
S31508009EF814461D460FCD0FC40FCD0FC40FCD0FC482
S31508009F082B68237066E07A4B01221A70794A734BDC
S31508009F1814460FCB07C423705CE0774B01221A70EE
S31508009F286E4B1B78AA2B03D1744B01221A7002E0D8
S31508009F38724B00221A70694B1A78714B1A7049E0ED
S31508009F4804F09CFC03466F4A13606F4B634A92E819
S31508009F5803001860043319706B4B1B88FB806A4B27
S31508009F685B88C3F57A63BB80FB88684AA2FB032330
S31508009F78DB089AB2664BA3F80F20654BBA88A3F894
S31508009F881B2027E004F07AFC03465E4A1360614BFF
S31508009F98524A07CA03C31A705E4B9A795C4B9A7081
S31508009FA818E004F06BFC0346564A13605A4B4B4AB2
S31508009FB892E8030018600433198002330A0C1A70F1
S31508009FC808E0564B01221A7004E000BF02E000BF01
S31508009FD800E000BF414B002283F80A2104F04EFC3A
S31508009FE802464F4B1B68D21A4E4B1B689A42C0F062
S31508009FF8C7844D4B1B78103B122B00F2A28401A292
S3150800A00852F823F059A000084BA900084BA90008E4
S3150800A0187FA0000891A0000841A100088BA10008AC
S3150800A028FDA100089FA20008F1A200087DA4000867
S3150800A03881A5000813A6000869A60008DBA600087B
S3150800A048C3A8000805A9000825A9000837A9000813
S3150800A05800210020FFF746FB00210120FFF742FBFD
S3150800A068324B1B78032B40F0708400F01DFE00F07D
S3150800A078A9FE00F06ABC142000F0B4FC4FF4FA708C
S3150800A08800F068FD00F07CBC144B93F80A31002BED
S3150800A09801D101F095FAFA2000F05CFD104B1B7807
S3150800A0A8002B02D0152000F09DFC0D4B1B78002BC9
S3150800A0B840F04D8400F042FD034642F21072934286
S3150800A0C840F245841A4800F0D3FD114B09225A7705
S3150800A0D81849042001F01AFA00F039BC7008002063
S3150800A0E82B030020400300202803002044030020F7
S3150800A0F829030020780300202A0300202D030020C6
S3150800A108BC030020C403002088030020CDCCCCCC97
S3150800A118F802002098030020A40300202C0300203E
S3150800A128200300202403002018030020D103002060
S3150800A138FCC0F0FC68650108AF4B93F80A31002BA0
S3150800A14801D101F03DFAFA2000F004FDAB4B5B7A29
S3150800A158002B02D0162000F045FC00F0EFFC034661
S3150800A16842F21072934240F2F4834FF2F04000F044
S3150800A1782BFDA34B0A225A77A249042001F0C6F9F7
S3150800A188FEE39D4B93F80A31002B01D101F018FA2A
S3150800A198FA2000F0DFFC9C4B1B889C4AA2FB032391
S3150800A1A8DB089AB2964BA3F80F20954B002242F08B
S3150800A1B80A02DA7600221A77914B0122DA758F4B52
S3150800A1C8DB79052B02D1172000F00CFC00F0B6FC51
S3150800A1D8034642F21072934240F2BD834FF2F040B2
S3150800A1E800F0F2FC864B0A225A778949042001F0C6
S3150800A1F88DF9C5E3804B93F80A31002B01D101F09C
S3150800A208DFF9FA2000F0A6FC7D4B5B7F002B03D014
S3150800A2184FF2F04000F0D8FC00F090FC034641F2FB
S3150800A2288832934202D9182000F0DCFB794BB3F840
S3150800A23801309BB21946774BB3F907301BB2DA0FD0
S3150800A24813445B101BB2994206DA6D4B01225A7702
S3150800A2587149052001F05AF96E4BB3F801309BB2E3
S3150800A26819466C4BB3F907301BB26C4A82FB0302DA
S3150800A2789210DB17D31A1BB2994280F26E83604B91
S3150800A28801225A776649052001F040F94FF2F04055
S3150800A29800F09AFC61E35A4B0022DA7300221A741A
S3150800A2A8574B0022DA7600221A77554B0022DA75C0
S3150800A2B800F044FC034641F2883293420BD94FF228
S3150800A2C8F04000F081FC4E4B0A225A775549042083
S3150800A2D801F01CF954E3494B9B7A002B40F03F8365
S3150800A2E8192000F07FFB3AE3434B93F80A31002B19
S3150800A2F802D1002001F078F9FA2000F02BFC4A4B2D
S3150800A3081B78002B60D01A2000F06CFB4749072001
S3150800A31801F0FCF8464B1B781A46454B5B781946FC
S3150800A328434B9B7800930B464249072001F0EEF809
S3150800A3383F4BDB781A464049072001F0E7F83C4BC3
S3150800A3489B881A463D49072001F0E0F8384BDB8818
S3150800A3581A463B49072001F0D9F83A4A3A490720EC
S3150800A36801F0D4F8324BDB681A463849072001F061
S3150800A378CDF82F4B9B7C1A462D4B5B7C19462C4BEC
S3150800A3881B7C03F2C17300930B463149072001F081
S3150800A398BDF8274BDA7C9B8A1B0213431A462D49BC
S3150800A3A8072001F0B3F8224B9B7D1A462A49072055
S3150800A3B801F0ACF8294A2A49072001F0A7F8294AE2
S3150800A3C82949072001F0A2F800F0B8FB034641F234
S3150800A3D88832934240F2C582134B1B78002B40F013
S3150800A3E8C082074B09225A77204800F041FC2049C9
S3150800A3F8042001F08BF8B4E2700800200C0A00204B
S3150800A408F80200207865010840030020CDCCCCCCA2
S3150800A4189865010860000020B865010867666666E1
S3150800A428CC650108FC650108280300201C6601089C
S3150800A43844030020286601083C660108506601089E
S3150800A448686601084C0300208066010898660108BA
S3150800A458AC660108D8660108EC6601085C030020AA
S3150800A468FC6601086D0300200C670108FCC0F0FDB6
S3150800A47820670108B04B93F80A31002B02D1AA20AD
S3150800A48801F0B2F8FA2000F065FBAC4B1B78002BFC
S3150800A4985AD01B2000F0A6FAA949072001F036F879
S3150800A4A8A84B1B88A84AA2FB03235B099BB21A463A
S3150800A4B8A649072001F02AF8A24B5B88A44AA2FB02
S3150800A4C80323DB089BB21A46A249072001F01EF8A7
S3150800A4D89C4B9B889E4AA2FB0323DB089BB21A4621
S3150800A4E89D49072001F012F8964BDB88984AA2FB8B
S3150800A4F80323DB089BB21A469449072001F006F89D
S3150800A508904B1B7A323B1A469449072000F0FEFF07
S3150800A5188C4BB3F809309BB28D4AA2FB0323DB08A0
S3150800A5289BB21A468E49072000F0F0FF854BB3F810
S3150800A5380B309BB2864AA2FB0323DB089BB21A465A
S3150800A5488849072000F0E2FF00F0F8FA034641F2CE
S3150800A5588832934240F20782784B1B78002B40F0EA
S3150800A5680282814B09225A77804800F081FB80498C
S3150800A578042000F0CBFFF6E16F4B93F80A31002B65
S3150800A58801D100F0F9FF022004F082F96A4B93F82A
S3150800A5980A31002B01D101F005F8FA2000F0DAFAA1
S3150800A5A800F0CCFA034641F2883293420DD9714B32
S3150800A5B81B78002B09D16C4B09225A776E4800F094
S3150800A5C857FB6E49042000F0A1FF6D4B1B78002B42
S3150800A5D803D01C2000F006FAC7E100F0AFFA0346DC
S3150800A5E84EF66022934240F2C081624B1B78012BDB
S3150800A5F840F0BB815C4B09225A775F4800F038FB6C
S3150800A6086049042000F082FFAFE14B4B93F80A310A
S3150800A618002B02D1002000F0FDFFFA2000F09AFA7C
S3150800A628594B5B7A002B02D01D2000F0DBF900F0AD
S3150800A63885FA034641F27072934240F29881524B6A
S3150800A6485B7A002B40F093814FF2F04000F0BCFA99
S3150800A658454B0A225A774D49042000F057FF86E1F0
S3150800A668354B93F80A31002B02D1AA2000F0D2FF05
S3150800A678FA2000F06FFA464B1B79002B00F0798117
S3150800A6881E2000F0AFF904F0F9F80346414A1360B2
S3150800A698082000F0BFFC3E4B5B88C3F57A637B80D5
S3150800A6A83B4B1B883B803B88294AA2FB0323DB08D4
S3150800A6B89AB22D4BA3F80F202B4B7A88A3F81B20A8
S3150800A6C8294B0122DA7503F0D5FA0346324A136094
S3150800A6D84FE104F0D3F802462E4B1B68D31AB3F59C
S3150800A6E8FA6F0BD94FF2F04000F06EFA1E4B0922AA
S3150800A6F85A772A49052000F009FF41E11A4B1B78C9
S3150800A708012B02D1264800F07BFA174B1B78032B3E
S3150800A71802D1234800F074FA224B5B78002B45D007
S3150800A7284FF2F04000F050FA0F4B04225A771E49B0
S3150800A738052000F0EBFE23E170080020290300201D
S3150800A74830670108780300201F85EB514067010828
S3150800A758CDCCCCCC4C67010858670108646701085A
S3150800A768706701087C670108F8020020FCC0F1FC44
S3150800A778886701082A030020FCC0F4FC98670108CA
S3150800A7882D030020A86701080C0A0020C0670108E5
S3150800A79888030020C4030020C0030020DC670108E2
S3150800A7A8F0F00004080000200068010800F00EFD1B
S3150800A7B80346032B0BD04FF2F04000F005FA784B0E
S3150800A7C808225A777749052000F0A0FED8E000202D
S3150800A7D8FFF7E0F803465A2B05DC0120FFF7DAF8FD
S3150800A7E803465A2B14DD704800F0EEF96C4B052227
S3150800A7F85A770020FFF7CEF803461C460120FFF7D4
S3150800A808C9F8034622466949052000F07FFEB7E0E5
S3150800A818674BB3F801309BB21946654BB3F9073055
S3150800A8281BB2644A82FB03029210DB17D31A1BB2C7
S3150800A838994206DA5A4B01225A775F49052000F0F1
S3150800A84865FE574B5B7F002B03D04FF2F04000F0B4
S3150800A858BBF95A4B4FF6FD72DA8003F00BFA02463B
S3150800A868574B1B68D31A574AA2FB03235B099AB2AC
S3150800A878524B9A804A4BB3F815309BB2C3F57A63A4
S3150800A8889AB24E4B5A80464BB3F813309BB21A46C7
S3150800A898920013445B009AB2484B1A804A4B93F8C5
S3150800A8A80A31002B05D100F0C9FE312000F052F913
S3150800A8B866E00A2000F04EF962E00A2000F04AF93C
S3150800A8C8374B0022DA75414B1B68184600F0C4FE60
S3150800A8D800F034F9034642F21072934206D93C490D
S3150800A8E8042000F013FE3B4800F0C2F93A4B1B78E7
S3150800A8F8002B40D0202000F075F83CE0FA2000F044
S3150800A90829F900F0C9FE00F019F9034640F6C41201
S3150800A918934232D9222000F065F82EE02F4B1B68A7
S3150800A928184600F0D9FE222000F05CF828E02C4BE7
S3150800A9381B780A2B23D0102000F054F800F0B4F93D
S3150800A9481DE0102000F04EF81AE000BF18E000BF1E
S3150800A95816E000BF14E000BF12E000BF10E000BF19
S3150800A9680EE000BF0CE000BF0AE000BF08E000BF29
S3150800A97806E000BF04E000BF02E000BF00E000BF39
S3150800A98800F024FC0346032B03D1054B01229A77D2
S3150800A99802E0034B00229A7700BF0837BD46B0BDD0
S3150800A9A8F80200201C680108F0F001003C6801085C
S3150800A9B86000002067666666CC650108AC0300205F
S3150800A9C8C00300208988888870080020C8030020EA
S3150800A9D864680108FDC0F0FC2C030020CC030020A5
S3150800A9E8D103002080B582B000AF0346FB71424A06
S3150800A9F8FB79137003F042FF0346404A13603E4B47
S3150800AA081B78102B03D13E49072000F07FFD3A4BEF
S3150800AA181B78132B03D13B49072000F077FD364BEB
S3150800AA281B78142B03D13849072000F06FFD324BE9
S3150800AA381B78152B03D13549072000F067FD2E4BE7
S3150800AA481B78172B03D13249072000F05FFD2A4BE4
S3150800AA581B78192B03D12F49072000F057FD264BE1
S3150800AA681B781A2B03D12C49072000F04FFD224BDF
S3150800AA781B781B2B03D12949072000F047FD1E4BDD
S3150800AA881B781C2B03D12649072000F03FFD1A4BDB
S3150800AA981B781D2B03D12349072000F037FD164BD9
S3150800AAA81B781E2B03D12049072000F02FFD124BD7
S3150800AAB81B781F2B03D11D49072000F027FD0E4BD5
S3150800AAC81B78202B03D11A49072000F01FFD0A4BD3
S3150800AAD81B78212B03D11749072000F017FD064BD1
S3150800AAE81B78222B03D11449072000F00FFD00BF5D
S3150800AAF80837BD4680BD00BF180300201C03002088
S3150800AB08746801088068010894680108A86801083B
S3150800AB18C0680108D0680108EC68010808690108D6
S3150800AB281C6901083469010848690108606901084F
S3150800AB387469010890690108A069010880B500AF21
S3150800AB4803F09CFE0246024B1B68D31A184680BDC2
S3150800AB581C03002080B582B000AF786003F08EFE33
S3150800AB680346044A1360044A7B68136000BF083723
S3150800AB78BD4680BD200300202403002080B582B08E
S3150800AB8800AF78600C4B5B7F002B03D00B4B002281
S3150800AB981A7002E0094B01221A70094A7B68136089
S3150800ABA8084B1B781F2B02D01F20FFF71BFF00BF7F
S3150800ABB80837BD4680BD00BFF8020020D003002034
S3150800ABC8C80300201803002080B582B000AF78605B
S3150800ABD8084B00221A70084A7B681360074B1B78D3
S3150800ABE81F2B02D01F20FFF7FDFE00BF0837BD4602
S3150800ABF880BD00BFD0030020C8030020180300202A
S3150800AC0880B582B000AF7860084B02221A70084AED
S3150800AC187B681360074B1B781F2B02D01F20FFF792
S3150800AC28E1FE00BF0837BD4680BD00BFD00300203F
S3150800AC38C80300201803002080B500AF0A4B01227C
S3150800AC481A700A4B0022DA752220FFF7CBFE00207D
S3150800AC5801F006F900210020FEF744FD0021012035
S3150800AC68FEF740FD00BF80BDD0030020F802002093
S3150800AC7880B582B000AF7860084B01221A707A68EE
S3150800AC880749042000F042FC064A7B681360212025
S3150800AC98FFF7A8FE00BF0837BD4680BDD0030020D1
S3150800ACA8B4690108CC03002080B500AF03F0E6FDBF
S3150800ACB80346314A1360314B00221A70304B002282
S3150800ACC81A70304B00221A702F4B00221A702F4B1D
S3150800ACD800221A702E4B00221A702E4B00229A70E8
S3150800ACE82C4B0022DA752B4B0022DA7600221A77CB
S3150800ACF8284B0022DA7300221A74312200212648CA
S3150800AD0809F01CFA0D220021244809F017FA052231
S3150800AD180021234809F012FA05220021214809F0E2
S3150800AD280DFA02220021204809F008FA0922002112
S3150800AD381E4809F003FA072200211D4809F0FEF902
S3150800AD48082200211B4809F0F9F9082200211A48A7
S3150800AD5809F0F4F9134B4FF47A625A80114B4FF401
S3150800AD68FA721A80154B00221A60154B00221A70BF
S3150800AD7801F080F900BF80BDC40300202803002025
S3150800AD88290300202A0300202B0300202C03002077
S3150800AD982D030020F8020020440300207803002031
S3150800ADA88803002090030020400300209803002011
S3150800ADB8A4030020AC030020B4030020C00300202D
S3150800ADC8BC03002080B500AF01210020FEF78AFCED
S3150800ADD801210120FEF786FC1320FFF703FE00BFBA
S3150800ADE880BD000080B500AF854B1B780C2B00F2A0
S3150800ADF8F38001A252F823F035AE000873AE0008B6
S3150800AE084DAE0008FFAE0008B9AE0008E1AF00086D
S3150800AE18E1AF0008E1AF000853AF0008E1AF00084A
S3150800AE28B5AF0008A7AF000899AF0008002001F0E1
S3150800AE3817F8744B1B78002B00F0D280012000F01D
S3150800AE48E9F8CDE0002001F00BF86F4B5B7F002B8B
S3150800AE5802D1012000F0DEF86B4B1B78032B40F07B
S3150800AE68C180002000F0C8FFBCE0002000F0F8FF11
S3150800AE78654B5B7F002B02D0022000F0CBF8624BB3
S3150800AE881B78032B02D1002000F0B6FF00F09EF9CC
S3150800AE980346032B40F0A8805B4B1B78032B00F076
S3150800AEA8A380042000F0B6F8002000F0D9FF9BE044
S3150800AEB8002000F0D5FF544B1B78032B02D1002045
S3150800AEC800F09AFF00F082F90346032B0FD14E4B88
S3150800AED81B78022B02D1032000F09CF84A4B1B78FA
S3150800AEE8032B40F08380012000F094F87EE00120CF
S3150800AEF800F090F87AE0012000F0B2FF434B1B7887
S3150800AF08222B1AD1424B1B78002B03D10B2000F0B9
S3150800AF1881F812E03E4B1B78012B03D10C2000F078
S3150800AF2879F80AE03A4B1B78022B03D10A2000F07D
S3150800AF3871F802E00B2000F06DF8344B1B781E2BD5
S3150800AF4856D1082000F066F852E0012000F088FF84
S3150800AF582E4B1B78222B4DD12D4B1B78002B03D15A
S3150800AF680B2000F057F845E0294B1B78012B03D135
S3150800AF780C2000F04FF83DE0254B1B78022B03D137
S3150800AF880A2000F047F835E00B2000F043F831E0D6
S3150800AF98002000F065FF0A2000F03CF82DE00020AC
S3150800AFA800F05EFF0A2000F035F826E0002000F0E1
S3150800AFB857FF154B1B78032B02D1002000F01CFF06
S3150800AFC800F004F90346022B16D1002000F048FFCA
S3150800AFD8012000F01FF80FE0002000F01BF80CE035
S3150800AFE800BF0AE000BF08E000BF06E000BF04E0B3
S3150800AFF800BF02E000BF00E000BF00BF80BD00BF81
S3150800B008D1030020160F0020F8020020180300209C
S3150800B018D003002080B582B000AF0346FB713D4AD5
S3150800B028FB7913703B4B1B78002B03D13A49072051
S3150800B03800F06CFA374B1B78012B03D137490720E8
S3150800B04800F064FA334B1B78022B03D134490720E6
S3150800B05800F05CFA2F4B1B78032B03D131490720E4
S3150800B06800F054FA2B4B1B78042B03D12E490720E2
S3150800B07800F04CFA274B1B78052B03D12B490720E0
S3150800B08800F044FA234B1B78062B03D128490720DE
S3150800B09800F03CFA1F4B1B78072B03D125490720DC
S3150800B0A800F034FA1B4B1B78082B03D122490720DA
S3150800B0B800F02CFA174B1B78092B03D11F490720D8
S3150800B0C800F024FA134B1B780A2B03D11C490720D6
S3150800B0D800F01CFA0F4B1B780B2B03D119490720D4
S3150800B0E800F014FA0B4B1B780C2B03D116490720D2
S3150800B0F800F00CFA074B1B780D2B03D113490720D0
S3150800B10800F004FA124AFB79537000BF0837BD46A7
S3150800B11880BD00BFD1030020CC690108E069010899
S3150800B128F8690108106A0108286A0108446A0108CA
S3150800B138646A0108846A0108A46A0108BC6A0108E5
S3150800B148D46A0108EC6A0108086B0108206B010833
S3150800B158F802002080B582B000AF03F08FFB0246E4
S3150800B168164B1B68D31A632B24D903F087FB0346AF
S3150800B178124A136000F034F80346FB71104B1B782B
S3150800B188FA799A4208D003F079FB03460D4A136008
S3150800B1980B4AFB7913700EE003F070FB0246094B65
S3150800B1A81B68D31AB3F5967F05D3054B1A78064B51
S3150800B1B81A7000E000BF0837BD4680BDD4030020DA
S3150800B1C8D8030020DC030020D203002080B400AF97
S3150800B1D8024B1B781846BD4680BC7047D203002030
S3150800B1E880B582B000AF00F051F8786022497868D7
S3150800B1F8FDF7AEFF0346002B08D020497868FDF70F
S3150800B208C5FF0346002B01D0012331E01C497868A5
S3150800B218FDF79EFF0346002B08D01A497868FDF704
S3150800B228B5FF0346002B01D0022321E015497868AB
S3150800B238FDF78EFF0346002B08D013497868FDF7FB
S3150800B248A5FF0346002B01D0032311E00E497868B1
S3150800B258FDF77EFF0346002B09D04FF07E5178682C
S3150800B268FDF794FF0346002B01D0042300E00023D2
S3150800B27818460837BD4680BD0000504100003041D9
S3150800B2886666E6409A9999400000404080B582B0C3
S3150800B29800AF0320FEF7C4FB0E4803F0F5FB642154
S3150800B2A80C4803F0CBFC0B4803F0CEFD7860094840
S3150800B2B803F098FC7868FDF755FD034606491846D5
S3150800B2C8FDF75CFE03463B603B6818460837BD46F3
S3150800B2D880BD00BF6C020020CDCCE24280B500AF2D
S3150800B2E8064B074A1A60054804F0D5FF0346002BA3
S3150800B2F801D001F04DF800BF80BD00BFE003002073
S3150800B3080030024080B485B000AF78607B681B685F
S3150800B318094A93420BD1094B5B69084A43F0400333
S3150800B3285361064B5B6903F04003FB60FB6800BF8B
S3150800B3381437BD4680BC70470030024000100240F2
S3150800B34880B584B000AFF860B9607A607B689BB254
S3150800B3581946B86800F006F87B6818461037BD46DF
S3150800B36880BD000080B485B000AF78600B467B804E
S3150800B37872B600BF0023FB8145E0284BB3F80434B6
S3150800B3889BB2B3F5806F18D3244BB3F802349BB23B
S3150800B39801335A42C3F30903C2F3090258BF534299
S3150800B3A89AB21E4BA3F802241C4BB3F804349BB27A
S3150800B3B8013B9AB2194BA3F80424FB897A6813440B
S3150800B3C8164AB2F8002492B21978144B9954134BBA
S3150800B3D8B3F800349BB201335A42C3F30903C2F3E4
S3150800B3E8090258BF53429AB20C4BA3F800240B4BD8
S3150800B3F8B3F804349BB201339AB2084BA3F8042471
S3150800B408FB890133FB81FA897B889A42B5D362B6F0
S3150800B41800BF00BF1437BD4680BC7047E80300204C
S3150800B42880B483B000AF72B600BF064BB3F80434D5
S3150800B438FB8062B600BFFB8818460C37BD4680BC41
S3150800B448704700BFE803002080B582B000AF72B627
S3150800B45800BF2D4BB3F804349BB2002B02D162B659
S3150800B46800BF4EE0284BB3F80434FB80FB88802BDA
S3150800B47801D98023FB80244BB3F802349BB2C3F569
S3150800B4888063BB80FA88BB889A4201D9BB88FB804F
S3150800B4981D4BB3F804349BB2FA889A420CD11A4B5E
S3150800B4A8B3F802349BB21A46174B1344F98850224C
S3150800B4B8184602F0D3F80BE0134BB3F802349BB2E4
S3150800B4C81A46114B1344F9885122184602F0C6F851
S3150800B4D80D4BB3F802349AB2FB8813449BB2C3F3F4
S3150800B4E809039AB2084BA3F80224074BB3F80434A5
S3150800B4F89AB2FB88D31A9AB2034BA3F8042462B605
S3150800B50800BF0837BD4680BDE80300200EB480B5E5
S3150800B51885B000AF0346FB71154AFB79137007F12E
S3150800B5282003BB60BB68FA697E21124808F0C8FD8B
S3150800B538F860FB68002B01DAFB6812E0FB687D2BD4
S3150800B54801DD7E23FB60FB680133094A0021D154DB
S3150800B558FB689BB202339BB219460548FFF702FF00
S3150800B568FB6818461437BD46BDE8804003B07047E7
S3150800B578F0070020F107002080B582B000AF02F07E
S3150800B58879FB02463B461946104602F0B1FB3B4694
S3150800B598072206214FF4E06000F060FB00BF083779
S3150800B5A8BD4680BD80B500AF044B082206214FF47E
S3150800B5B8006000F053FB00BF80BD00BF30030020C9
S3150800B5C880B582B000AF01233B7101237B7100234C
S3150800B5D8BB713B1D032206214FF4185000F03EFBB1
S3150800B5E800BF0837BD4680BD80B582B000AF0346A8
S3150800B5F8FB71074AFB791370054B082206214FF49D
S3150800B608807000F02BFB00BF0837BD4680BD00BF21
S3150800B6183803002080B584B000AF0346FB71FB7978
S3150800B6283B7307F10C03012204214FF4206000F054
S3150800B63815FB00BF1037BD4680BD000080B500AFBA
S3150800B648044B082206214FF4905000F007FB00BF70
S3150800B65880BD00BFAC03002080B584B000AF786019
S3150800B6687B681B0EDBB23B727B681B0CDBB27B72FA
S3150800B6787B681B0ADBB2BB727B68DBB2FB7207F11D
S3150800B6880803042204214FF4D05000F0E7FA00BF5B
S3150800B6981037BD4680BD000080B500AF0B4BD3F808
S3150800B6A801300B4A53600A4B00229A700022DA705E
S3150800B6B8084B9B889AB2064B1A80054B0722062127
S3150800B6C84FF4E85000F0CAFA00BF80BD38030020DE
S3150800B6D8B4030020AC03002080B584B000AF7860BE
S3150800B6E87B681B0EDBB23B727B681B0CDBB27B727A
S3150800B6F87B681B0ADBB2BB727B68DBB2FB7207F19D
S3150800B7080803042204214FF4F85000F0A7FA00BFF2
S3150800B7181037BD4680BD000080B58AB000AF07F176
S3150800B728140300221A605A609A60DA607D4B9B6996
S3150800B7387C4A43F0100393617A4B9B6903F0100324
S3150800B7483B613B69774B9B69764A43F004039361EF
S3150800B758744B9B6903F00403FB60FB68714B9B6998
S3150800B768704A43F0080393616E4B9B6903F008031C
S3150800B778BB60BB686B4B9B696A4A43F0400393619D
S3150800B788684B9B6903F040037B607B68654B9B6944
S3150800B798644A43F020039361624B9B6903F02003D4
S3150800B7A83B603B68002230215F4805F06EF80022AE
S3150800B7B84FF4F8515D4805F068F800224FF4004147
S3150800B7C85B4805F062F8002218215A4805F05DF82A
S3150800B7D800228021584805F058F802237B61002387
S3150800B7E8BB610023FB6107F114031946504804F0AE
S3150800B7F8B1FE04237B610023BB610223FB6107F1C9
S3150800B808140319464A4804F0A5FE30237B61012330
S3150800B818BB610023FB6102233B6207F11403194647
S3150800B828414804F097FE44F282037B610023BB611A
S3150800B8380023FB6107F1140319463C4804F08AFE05
S3150800B8484FF4F8537B610123BB610023FB61022394
S3150800B8583B6207F114031946344804F07BFE4FF49B
S3150800B86800437B610123BB610023FB6102233B6222
S3150800B87807F1140319462E4804F06CFE18237B6159
S3150800B8880123BB610023FB6102233B6207F1140312
S3150800B8981946284804F05EFE80237B610023BB61B5
S3150800B8A80023FB6107F114031946224804F052FEE7
S3150800B8B818237B610023BB610023FB6107F114038E
S3150800B8C819461D4804F046FE80237B610123BB61A7
S3150800B8D80023FB6102233B6207F114031946164845
S3150800B8E804F038FE4FF440737B611223BB610323CF
S3150800B8F83B6207F1140319460F4804F02BFE0F4B59
S3150800B9085B687B627B6A43F0E0637B627B6A43F031
S3150800B91802037B62094A7B6A536000BF2837BD4623
S3150800B92880BD00BF00100240001001400018014009
S3150800B9380008014000140140000C014000000140C5
S3150800B94890B5CDB040AF786007F10C0300221A60B5
S3150800B9585A6007F10C0307F114020021786804F00D
S3150800B9682DF80346002B40F05381BB699BB245F27C
S3150800B978F462934240F04C81BB691B0A03F47F4387
S3150800B988B3F56C4F13D0B3F56C4F00F20C81B3F5D1
S3150800B9986B4F57D0B3F56B4F00F20581B3F5C85F07
S3150800B9A800F0DD80B3F5F05F00F0B680FBE03B7B86
S3150800B9B8102B3ED17B7B1AB2BB7B1BB21B021BB278
S3150800B9C813431BB29AB2944BA3F80421924B012253
S3150800B9D883F80721FA7B904B83F806218E4B0222BF
S3150800B9E883F808218C4B93F808218B4B83F8092197
S3150800B9F8FB7C1A04BB7C1B0213437A7C13431A4646
S3150800BA08854BC3F80021844BB3F80431FF2B10D8B3
S3150800BA18814C684604F110034FF48072194608F001
S3150800BA289BFC94E80F0000F041F97B4B012283F850
S3150800BA380A213B7BFF2B40F0E680774B002283F8F0
S3150800BA480A21E0E0744B93F80A31012B40F0DD80B7
S3150800BA583B7B002B00F0DB803B7B222B00F2D78058
S3150800BA686D4B93F807213B7B9A4240F0D0803B7B8D
S3150800BA785A1E1346DB009B1A674A981807F10C03E7
S3150800BA8801330722194608F067FC634B93F8073118
S3150800BA980133DAB2604B83F807215F4B93F8072125
S3150800BAA85D4B93F806319A4211D95B4C684604F106
S3150800BAB810034FF48072194608F04EFC94E80F00FC
S3150800BAC800F03AF9544B022283F80A219FE0524BB8
S3150800BAD893F80931002B07D04F4B93F80931013BEE
S3150800BAE8DAB24D4B83F809214B4B93F80931002BF1
S3150800BAF840F08D80484C684604F110034FF4807274
S3150800BB08194608F029FC94E80F0000F0CFF8424BD4
S3150800BB18022283F809217AE040490420FFF7F6FC57
S3150800BB283B7B19467B7B1846BB7BFA7B01920093C5
S3150800BB3803460A463A490420FFF7E8FC3B7C1946BF
S3150800BB487B7C1846BB7CFA7C0192009303460A461E
S3150800BB5834490420FFF7DAFCFFF76EF858E0324953
S3150800BB680720FFF7D3FC3B7B19467B7B1846BB7B34
S3150800BB78FA7B0192009303460A462C490720FFF7E9
S3150800BB88C5FC3B7C19467B7C1846BB7CFA7C019233
S3150800BB98009303460A4623490720FFF7B7FC2448BB
S3150800BBA8FEF7ECFF34E01C4B93F80A31002B2FD133
S3150800BBB87B6A9AB2184BA3F80421174B012283F81B
S3150800BBC80721154B012283F80621134B012283F816
S3150800BBD80821114B002283F80921BB691B0A03F4C3
S3150800BBE87F430D4AC2F800310B4B022283F80A211B
S3150800BBF8094BB3F804311A4607F10C0319460648E7
S3150800BC0808F0AAFB04E000BF02E000BF00E000BF9E
S3150800BC1800BF3437BD4690BD70080020386B010850
S3150800BC285C6B0108786B0108906B0108AC6B01081E
S3150800BC38F0F0004080B500AF074803F073FDFDF744
S3150800BC480BFF00F0B3F8044803F028FD0221024868
S3150800BC5803F0D5FF00BF80BDA402002080B58CB0D4
S3150800BC6800AFF8607B600B46FB721346BB72FB7A23
S3150800BC789A06FB681B02134343F4744343F05603BE
S3150800BC88FB6100237B6204233B62BB7ABB6207F134
S3150800BC98140307F118017A68034803F08CFD00BFFE
S3150800BCA83037BD4680BD00BFA402002084B080B5E9
S3150800BCB882B000AF07F1100C8CE80F0011233B7017
S3150800BCC897F818317B7097F818311A4697F816318D
S3150800BCD8194697F81731CB1A01339A4208DD97F8AF
S3150800BCE8162197F81731D31ADBB20133DBB27B700A
S3150800BCF897F81731BB70FF23FB70FF233B71D7F802
S3150800BD081031DBB27B71D7F810311B0ADBB2BB7175
S3150800BD18D7F810311B0CDBB2FB713B46082207210A
S3150800BD284FF46C40FFF79AFF00BF0837BD46BDE8D9
S3150800BD38804004B07047000084B080B582B000AF78
S3150800BD4807F1100C8CE80F0013233B70164BB3F859
S3150800BD580431DBB27B70144BB3F804311B0A9BB26F
S3150800BD68DBB2BB70104B93F80631FB70FF233B71AF
S3150800BD78D7F81031DBB27B71D7F810311B0ADBB262
S3150800BD88BB71D7F810311B0CDBB2FB713B46082296
S3150800BD9807214FF46C40FFF761FF00BF0837BD461F
S3150800BDA8BDE8804004B070477008002080B58AB0A6
S3150800BDB800AF00237B610023BB610123FB610023DD
S3150800BDC83B6000237B600023BB600023FB600023E5
S3150800BDD83B6101233B623B461946064803F07EFB56
S3150800BDE80346002B01D000F0D3FA00BF2837BD461A
S3150800BDF880BD00BFA402002080B483B000AF03460C
S3150800BE08FB71FB79002B14BF01230023DBB21A460A
S3150800BE18044B9A70034B00221A7200BF0C37BD46B2
S3150800BE2880BC70470800002080B500AF0A4B1B7815
S3150800BE38002B05D08021094804F010FD034609E0C7
S3150800BE488021064804F00AFD0346002B0CBF01238F
S3150800BE580023DBB2184680BD040000200018014004
S3150800BE6880B483B000AF0346FB71044AFB791370AC
S3150800BE7800BF0C37BD4680BC704700BF08000020CD
S3150800BE8880B582B000AF02F0F9FC786000F004F9DA
S3150800BE98724B5B78002B40F0DD80FFF7C5FF034641
S3150800BEA8002B0CBF01230023FB706C4B1B78002B5F
S3150800BEB80CBF01230023BB70684B9B78FF2B04D16A
S3150800BEC8FA78BB789A4200F0AD80644B9B78FF2BD2
S3150800BED809D1BB7883F00103DBB21A465F4B9A7027
S3150800BEE85E4B00221A725D4BDB78022B4AD0022B76
S3150800BEF800F3B180002B02D0012B2AD0ABE0584BB7
S3150800BF081B78002B0FD0554B9B78012B05D10122A6
S3150800BF182021544804F0B9FC14E0012210215148A4
S3150800BF2804F0B3FC0EE04D4B9B78012B05D101229A
S3150800BF3810214C4804F0A9FC04E0012220214948B4
S3150800BF4804F0A3FC454B0122DA70444A7B68536027
S3150800BF5867E0424B5B687A68D31A434A1288934269
S3150800BF685CD3002210213F4804F08FFC00222021D0
S3150800BF783C4804F08AFC394B0222DA70374A7B6857
S3150800BF8853604BE0354B5B687A68D31A312B47D92F
S3150800BF98FFF74AFF0346002B0CBF01230023FB705B
S3150800BFA8FB782E4A9278002A0CBF01220022D2B2C8
S3150800BFB893420CBF012300237B707B78002B09D0A2
S3150800BFC8264BFF229A70254B0022DA70234B002253
S3150800BFD81A7225E0214B1B7A0133DAB21F4B1A7203
S3150800BFE81E4B1A7A214B1B789A4213D31B4B0122F4
S3150800BFF85A701A4A7B68D360184B00229A70174BF6
S3150800C0080022DA70154B00221A7219490420FFF724
S3150800C0187DFA05E0114B0022DA7001E000BF1AE04C
S3150800C02800BF18E00D4BDB78002B0CD0002210213E
S3150800C0380C4804F02AFC002220210A4804F025FCB2
S3150800C048064B0022DA70054BFF229A70034B002232
S3150800C0581A7200E000BF0837BD4680BD08000020F8
S3150800C068050000200010014006000020BB6C0108EE
S3150800C078C86B010880B500AF054B00225A70044BFF
S3150800C0880022DA6003490720FFF740FA00BF80BD9F
S3150800C09808000020D46B010880B500AF0A4B5B780E
S3150800C0A8002B0FD0084BDB68002B0BD002F0E6FB01
S3150800C0B80246054BDB68D21A044B1B689A4201D321
S3150800C0C8FFF7D8FF00BF80BD08000020BC6C010838
S3150800C0D880B400AF034B044A9A6000BFBD4680BCD3
S3150800C0E8704700BF00ED00E00080000880B485B006
S3150800C0F800AF03460A46FB711346BB71BB791F2B73
S3150800C10801D900230EE00023FB73BB79084AD35CE8
S3150800C118FA799A4201D00123FB73BB790449FA7963
S3150800C128CA54FB7B18461437BD4680BC704700BF07
S3150800C1388009002080B584B000AF786002F09EFBC5
S3150800C148B8607B68FB60FB68B3F1FF3F12D0104B01
S3150800C1581B781A46FB681344FB600BE0FEF7FAFFE8
S3150800C168FFF78EFEFEF73EFEFDF75EFE00F0F4FFD3
S3150800C17801F008F902F082FB0246BB68D31AFA688E
S3150800C1889A42EBD800BF00BF1037BD4680BD00BF36
S3150800C1988000002080B500AF0320FDF717FB034693
S3150800C1A8002B02D1024B01221A7000BF80BD00BFC6
S3150800C1B8F802002080B582B002AFFFF789FF02F0C7
S3150800C1C805FB04F087FB00F073F8FFF7A5FAFDF7FF
S3150800C1D8F7F9FDF741FCFDF775FC01F05BF801F08E
S3150800C1E8EBFF02F02BF9FFF779F802F0D3F802F023
S3150800C1F8FBF802F04DF9FDF73BFB00F08DFF4FF415
S3150800C208967002F045FBFDF7D1FD01F0A7F800236B
S3150800C218012222490720FFF779F901F07BF8204B1C
S3150800C2281B889BB21A461F490720FFF76FF91C4B54
S3150800C2389B781A461C490720FFF768F9184B9B880C
S3150800C2489BB21A46164BDB889BB21946144B1B89B8
S3150800C2589BB200930B4615490720FFF757F9FDF7D8
S3150800C268C3FDFFF7E7FC00F07DFAFDF73FFD00F098
S3150800C27887FB00F023FC0A20FFF75CFF00F08EF826
S3150800C288FDF74AFD00F00EFE0A20FFF753FFFFF7F9
S3150800C29881FF3220FFF74EFF00BFE8E7E86B010889
S3150800C2A80C0F0020FC6B0108106C0108246C0108AF
S3150800C2B880B59CB000AF07F138033822002118462C
S3150800C2C807F03CFF07F1240300221A605A609A60B7
S3150800C2D8DA601A613B1D20220021184607F02EFF56
S3150800C2E80523BB634FF480333B6404237B64012333
S3150800C2F8BB640123FB644FF48033FB630223BB65ED
S3150800C3084FF48033FB654FF4E0133B6602237B66E4
S3150800C3184FF4C063BB664023FB6607F1380318462B
S3150800C32804F0A8FB0346002B01D000F031F80F23D0
S3150800C3387B620223BB620023FB624FF480633B6384
S3150800C34800237B6307F124030221184604F0A8FE9C
S3150800C3580346002B01D000F01BF803237B604FF43B
S3150800C3688073BB604FF40043FB603B1D184605F01D
S3150800C3788DF80346002B01D000F00AF8034B01227A
S3150800C3881A6000BF7037BD4680BD00BF70004242C4
S3150800C39880B400AF72B600BF00BFFDE72DE9B04311
S3150800C3A884B000AF2E4B00221A712E4B5B78082BEF
S3150800C3B804D12B4B012283F8242003E0284B0022C2
S3150800C3C883F8242002F05AFAF860254B9B68FA6825
S3150800C3D8D31ABB60224AFB689360224BD3F8033012
S3150800C3E8BA6802FB03F3204AA2FB03239B097B6076
S3150800C3F81B4BD3E90423796800200C46054612EB43
S3150800C408040843EB0509164BC3E90489144BD3E919
S3150800C4180423164BA3FB0223DB0A114A9361104B2C
S3150800C42893F82430002B08D00D4B9A690C4BDB691E
S3150800C438D31A0C4AC2F807300CE00A4B0022DA7104
S3150800C44800221A7200225A7200229A72044B9B69B9
S3150800C458034AD36100BF1037BD46BDE8B08300BFA5
S3150800C468A0090020F8020020D34D6210C5B3A29196
S3150800C47880B582B000AF0346FB71064AFB79D371D3
S3150800C48802F0FCF90346034A136100BF0837BD46A4
S3150800C49880BD00BF0C0A002080B500AF02F0EEF997
S3150800C4A80246024B1B69D31A184680BD0C0A00209F
S3150800C4B880B584B000AF7860884B894A01217868CE
S3150800C4C803F07CFA0346002B40F00481844B5B6832
S3150800C4D8BB603B7A002B40F0FC8002F0CFF903469C
S3150800C4E8804A1360BB7A03F03F03DBB2022B05D1FF
S3150800C4F87D4B7A4A92E8030083E80300BB7A03F087
S3150800C5083F03DBB2042B19D1784B744A92E803002F
S3150800C51883E80300754B1B791A46754BDA61734B2A
S3150800C5281A7A734B83F82020704BDA79704B83F8A4
S3150800C53821206E4B9A796E4B83F82220BB7A03F03A
S3150800C5483F03DBB2062B23D16A4B644A92E8030001
S3150800C55883E80300674B5B781A46664B1B781B0211
S3150800C56813441A46634B9A60624BDB781A46614B4A
S3150800C5789B781B0213441A465E4BDA605D4B5B795F
S3150800C5881A465C4B1B791B0213441A46594B1A6107
S3150800C598BB7A03F03F03DBB2082B05D1564B4F4A4B
S3150800C5A892E8030083E80300BB7A03F03F03DBB293
S3150800C5B8092B40F08F80514B484A92E8030083E8DC
S3150800C5C803004E4BDB791A464C4BDA604B4BDA685C
S3150800C5D84A4B9B791B021343484AD360474BDA6890
S3150800C5E8464B5B791B041343444AD360434BDA68CA
S3150800C5F8424B1B791B061343404AD3603F4BDB78F3
S3150800C6081A463E4B9A603D4B9A683C4B9B781B02F0
S3150800C61813433A4A9360394B9A68384B5B781B043C
S3150800C6281343364A9360354B9A68344B1B781B0676
S3150800C6381343324A9360314B9B68314AA2FB032362
S3150800C6489B09FB812D4BDB682E4AA2FB03235B095A
S3150800C658BB81274AFB895380254ABB899380FB8976
S3150800C668132B8CBF01230023DBB21A46204B9A7280
S3150800C6781F4B01221A721D4B1A791D4B9A711C4BB6
S3150800C688DB79012B26D91A4B5A881F4BA3F8132096
S3150800C698174BB3F904309AB21B4BA3F815201A4B5B
S3150800C6A8B3F815309BB21A46174BB3F813309BB23A
S3150800C6B802FB03F3154A82FB03129210DB17D31AFF
S3150800C6C81A46114BC3F80320094B9A7A0E4B1A7669
S3150800C6D800E000BF1037BD4680BD00BF500A0020E5
S3150800C6E8340A0020300A0020C8090020D40900208E
S3150800C6F80C0A0020E0090020F4090020FC090020A3
S3150800C708D34D62101F85EB51F802002067666666EE
S3150800C71880B58AB000AF0E237B610023BB61012375
S3150800C728FB6100233B6000237B600023BB6000237A
S3150800C738FB6000233B6101233B6201233B610E2317
S3150800C7487B623B461946064802F0C8FE0346002B9C
S3150800C75801D0FFF71DFE00BF2837BD4680BD00BFC4
S3150800C768CC02002080B500AF134802F0DBFFFDF7C6
S3150800C778A9F9FFF7CDFF104802F090FF10210E48DF
S3150800C78803F03DFA242200210C4807F0D7FC0B4B8E
S3150800C7980022DA7102F072F80346084A1361074B59
S3150800C7A847F230525A61054B00221A7600210020BA
S3150800C7B800F006F800BF80BDCC0200200C0A002055
S3150800C7C880B584B000AF03460A46FB711346BB71B1
S3150800C7D807F1080308220021184607F0AFFCFB7981
S3150800C7E8002B15D10D4B1B7A002B13D0BB79002BC8
S3150800C7F80CBF01230023DBB23B72F97907F1080362
S3150800C8081A22F02000F066F81420FFF793FC02E0DD
S3150800C81800BF00E000BF1037BD4680BD0C0A0020E7
S3150800C82880B586B000AF0346FB710B46BB8013463E
S3150800C8387B8007F1080308220021184607F07EFCCA
S3150800C848FB79002B40D1BB88952B01D89623BB8052
S3150800C8581F4B1B7E002B06D1BB88B3F5FA7F02D384
S3150800C86840F2F313BB807B88642202FB03F37B61E7
S3150800C878BB884FF47A7202FB03F33B617B691B0E94
S3150800C888DBB23B737B691B0CDBB27B737B691B0AC8
S3150800C898DBB2BB737B69DBB2FB733B691B0EDBB28E
S3150800C8A83B723B691B0CDBB27B723B691B0ADBB22A
S3150800C8B8BB723B69DBB2FB72F97907F108031C22E4
S3150800C8C8F02000F007F800E000BF1837BD4680BD25
S3150800C8D80C0A002080B58CB000AF3B600346FB719C
S3150800C8E80B46BB7113467B71FB7987F82830BB79F1
S3150800C8F887F829307B7903F03F03DAB297F82A30AC
S3150800C90862F3050387F82A307B8D0A2262F38913B6
S3150800C9187B850A2387F82F30BB6A7B610023FB6176
S3150800C9280423BB6108233B621EE0144803F012F88F
S3150800C9380346002B0ED007F10C0307F110013A68DD
S3150800C9480E4802F038FF034687F82E3097F82E303F
S3150800C958002B0ED00120FFF7EDFB97F92F30DBB23D
S3150800C968013BDBB287F82F3097F92F30002BDCDC38
S3150800C97800E000BF3037BD4680BD00BFCC020020AE
S3150800C98880B582B000AF3B4600221A605A603B4623
S3150800C99804220021F020FFF79DFF1420FFF7CAFBA9
S3150800C9A83B4606220021F020FFF794FF1420FFF7E4
S3150800C9B8C1FB3B4609220021F020FFF78BFF142014
S3150800C9C8FFF7B8FB394BB3F81B309BB2384AA2FBC2
S3150800C9D80323DB089BB21A46344BB3F813309BB2D1
S3150800C9E802FB03F31A46334B5B699A4211D9314B5A
S3150800C9F85A6913469B0013445B001A462B4BB3F837
S3150800CA0813309BB2B2FBF3F39AB2284BA3F8112062
S3150800CA1806E0264BB3F81B309AB2244BA3F811202C
S3150800CA28224BB3F811309BB2B3F57A7F08D91F4B5E
S3150800CA38002262F017025A74002242F003029A741E
S3150800CA481A4BB3F811309BB21A46184BB3F80F3085
S3150800CA589BB202FB03F3184A82FB03129210DB17F8
S3150800CA68D31A1A46114BC3F80B20124B5B7A002BC4
S3150800CA7818D00E4BB3F80F309BB20C4AB2F81120F7
S3150800CA8892B219460020FFF7CBFE1420FFF752FB97
S3150800CA98064BB3F813309BB2B3F5F57F02D9054BAD
S3150800CAA801221A7600BF0837BD4680BDF802002065
S3150800CAB8CDCCCCCC0C0A00206766666698B500AF64
S3150800CAC801F0DCFE0246B44B1B68D31AB3F5FA7FAD
S3150800CAD820D9B24B00221A72B04B00229A72B04B78
S3150800CAE800221A71AE4B00221A72AD4B0022DA7177
S3150800CAF8AB4B00229A71AB4B00229A60A94B0022D5
S3150800CB08DA60A84B00221A61A74B0022DA60A64B06
S3150800CB1800229A60A14B1B7A002B03D09F4B1B78E7
S3150800CB28002B0CD1A14B0022DA7400221A759F4BF0
S3150800CB3800225A7500229A759C4B00221A769B4B3E
S3150800CB489B7F002B0CD001210420FCF7CBFD01F0BC
S3150800CB5895FE0346964A1360904B01221A7010E018
S3150800CB6801F08CFE0246924B1B68D31A4EF66022D9
S3150800CB78934206D900210420FCF7B4FD874B00220E
S3150800CB881A700520FCF722FE03461A46834BDA720A
S3150800CB98824B1B7A002B07D0804B1B7B002B03D1BB
S3150800CBA87E4B1B78002B02D17C4B00225A727B4B9A
S3150800CBB8DB79092B00F2558101A252F823F000BF50
S3150800CBC8F1CB000825CC000841CC000879CC000830
S3150800CBD8C7CC000809CD000873CD00081DCE00088B
S3150800CBE8CDCD000857CE00086C4B00225A7000219C
S3150800CBF80320FCF777FD694B1B7A002B00F035817B
S3150800CC08664B1B78002B00F03081644B1B7B002B8E
S3150800CC1840F02B810120FFF72BFC26E1FFF73CFCAF
S3150800CC280346B3F57A6F40F222815C4B01225A72A9
S3150800CC380220FFF71DFC1AE1584B00221A7600213C
S3150800CC480320FCF74FFD554B5B7A002B03D10020D8
S3150800CC58FFF70EFC1CE1554BDB7D002B00F0098124
S3150800CC6801210020FFF7ACFD0320FFF701FC00E1D6
S3150800CC784A4B9B7A002B0CD0484B5B7A002B08D082
S3150800CC8801F0FCFD03464B4A13600420FFF7F0FB4E
S3150800CC98F1E0FFF701FC034642F21072934240F2B4
S3150800CCA8EA803E4B01225A73404B0A225A770020E3
S3150800CCB8FFF7DEFB40490420FEF728FCDBE00121EC
S3150800CCC80320FCF70FFD354BDB7A002B03D0052034
S3150800CCD8FFF7CEFBD1E0FFF7DFFB0346B3F57A7F14
S3150800CCE840F2CB802D4B01221A73304B07225A7714
S3150800CCF80620FFF7BDFB31490420FEF707FCBCE018
S3150800CD082A4BDB7D002B03D0244B5B7A002B03D1FF
S3150800CD180620FFF7ADFBBBE00520FCF757FD0346E9
S3150800CD281C460320FCF742FD03469C4217D001F037
S3150800CD38A5FD0246224B1B68D31AB3F57A7F40F243
S3150800CD489E801A4B07225A77144B01221A7306201B
S3150800CD58FFF78EFB19490420FEF7D8FB8FE001F090
S3150800CD688DFD0346164A136089E0104B00225A7453
S3150800CD7800229A740D4BB3F815309BB21D2B06D9B1
S3150800CD88FFF78AFB034641F28832934279D908208D
S3150800CD98FFF76EFB75E000BF300A00200C0A00207A
S3150800CDA8D4090020E0090020FC090020F802002028
S3150800CDB8580A00205C0A00203C6C01084C6C0108E3
S3150800CDC8600A002000210320FCF78CFC314BDB7A33
S3150800CDD8002B07D100210020FFF7F2FC0720FFF7F8
S3150800CDE847FB50E0FFF758FB0346B3F57A7F4AD965
S3150800CDF8284B01221A73284B07225A77002100204C
S3150800CE08FFF7DEFC0720FFF733FB24490420FEF76B
S3150800CE187DFB38E01F4B9B7A002B03D10920FFF7CF
S3150800CE2827FB32E0FFF738FB034642F210729342BB
S3150800CE382BD9184B01225A73174B0A225A77002006
S3150800CE48FFF716FB16490420FEF760FB1DE0FFF7FF
S3150800CE5823FB0346B3F57A6F19D90220FFF708FBB7
S3150800CE6815E00020FFF704FB12E000BF10E000BF42
S3150800CE780EE000BF0CE000BF0AE000BF08E000BFF4
S3150800CE8806E000BF04E000BF02E000BF00E000BF04
S3150800CE9800BF98BD0C0A0020F80200204C6C010857
S3150800CEA86C6C010880B500AF344B5B7F002B03D050
S3150800CEB8334800F01FF95FE0304B5B780D2B57D8E5
S3150800CEC801A252F823F000BF09CF000811CF0008C5
S3150800CED819CF000821CF000829CF000831CF00084C
S3150800CEE839CF000841CF000849CF000851CF0008BC
S3150800CEF859CF000861CF000869CF000871CF00082C
S3150800CF08204800F0F7F837E01F4800F0F3F833E058
S3150800CF181B4800F0EFF82FE01C4800F0EBF82BE070
S3150800CF281A4800F0E7F827E0194800F0E3F823E084
S3150800CF38174800F0DFF81FE0154800F0DBF81BE09B
S3150800CF48134800F0D7F817E0124800F0D3F813E0B2
S3150800CF58104800F0CFF80FE00E4800F0CBF80BE0C9
S3150800CF680C4800F0C7F807E0084800F0C3F803E0E3
S3150800CF78044800F0BFF800BF80BD00BFF8020020D3
S3150800CF88540000201800002024000020300000204B
S3150800CF983C0000204800002080B487B000AFF86045
S3150800CFA8B96011461A460B46FB801346BB80FA88B9
S3150800CFB8BB889A4201D9BB88FB80BB88002B01D164
S3150800CFC80123BB80FA8813461B029A1ABB8892FB70
S3150800CFD8F3F3FB82FB681B781A46FB8AC3F1FF0347
S3150800CFE803FB02F2BB681B781946FB8A01FB03F3AD
S3150800CFF81344204A82FB03121A44D211DB17D31AA8
S3150800D008DAB23B6A1A70FB685B781A46FB8AC3F180
S3150800D018FF0303FB02F2BB685B781946FB8A01FB30
S3150800D02803F31344134A82FB03121A44D211DB177B
S3150800D038D31ADAB23B6A5A70FB689B781A46FB8A97
S3150800D048C3F1FF0303FB02F2BB689B781946FB8A08
S3150800D05801FB03F31344074A82FB03121A44D2114D
S3150800D068DB17D31ADAB23B6A9A7000BF1C37BD467B
S3150800D07880BC70478180808080B483B000AF7860B8
S3150800D0887B681B781A46642302FB03F3174A82FB5C
S3150800D09803121A44D211DB17D21A154B1B689A6366
S3150800D0A87B685B781A46642302FB03F30F4A82FB04
S3150800D0B803121A44D211DB17D21A0D4B1B68DA630E
S3150800D0C87B689B781A46642302FB03F3074A82FBAC
S3150800D0D803121A44D211DB17D21A054B1B681A64B5
S3150800D0E800BF0C37BD4680BC704700BF8180808072
S3150800D0F81C0F002080B483B000AF7860054B7A68AF
S3150800D1081068516803C312891A8000BF0C37BD46D8
S3150800D11880BC70476C0A002080B582B000AF002337
S3150800D1283B7100237B710023BB710421094804F075
S3150800D138E1FD0821074804F0DDFD0C21054804F047
S3150800D148D9FD3B1D1846FFF797FF00BF0837BD46B0
S3150800D15880BD00BF1C0F002080B582B002AF01F069
S3150800D1688DFB0246464B1B68D31A142B40F2858062
S3150800D17801F084FB0346424A1360424B5B8801333D
S3150800D1889AB2404B5A803F4B1B78032B67D801A2AB
S3150800D19852F823F0ADD10008DFD100080BD20008F9
S3150800D1A83DD20008374B5A88374BDB781946374B38
S3150800D1B800930B4634493648FFF7EEFE314B5B8839
S3150800D1C8314AD27893424ED92E4B01221A702D4BEA
S3150800D1D800225A8047E02B4B2B4A04331268114623
S3150800D1E819800233120C1A70264B5B88264A127964
S3150800D1F893423AD9234B02221A70224B00225A80AC
S3150800D20833E0204B5A88204B5B7919461F4B00930D
S3150800D2180B461F491C48FFF7BFFE1A4B5B881A4A7C
S3150800D2285279934223D9174B03221A70154B0022B9
S3150800D2385A801CE0134B144A043307321188927833
S3150800D24819809A700F4B5B880F4A9279934210D9C6
S3150800D2580C4B00221A700B4B00225A8009E0094B26
S3150800D26800221A7006E000BF04E000BF02E000BF13
S3150800D27800E000BF0548FFF7FFFE00BFBD4680BDBA
S3150800D288780A0020640A00206C0A0020680A002030
S3150800D298730A002080B500AF0A4B0B4A1A60094B7F
S3150800D2A84FF0FF325A60074B4FF480729A60054870
S3150800D2B804F070FB0346002B01D0FFF769F800BF9E
S3150800D2C880BD00BF7C0A00200028004080B584B0D5
S3150800D2D800AF78607B681B680B4A934210D103F04D
S3150800D2E8EDFA0A4BDB69094A43F00063D361074B39
S3150800D2F8DB6903F00063FB60FB68054B01221A60D3
S3150800D30800BF1037BD4680BD002800400010024007
S3150800D3183C04424280B400AF0E4B1B681B689AB2A5
S3150800D3280D4B1A800B4B1B685A790B4B9A70094B95
S3150800D3381B681A79084BDA70074B01229A80064B44
S3150800D3480022DA80044B01221A8100BFBD4680BC40
S3150800D358704700BF000000200C0F002080B500AF02
S3150800D3684FF404720021054806F0E8FE4FF40472EB
S3150800D3780021034806F0E2FE00BF80BD900A00209F
S3150800D388A00C002080B500AF2A4B93F84230DBB2D8
S3150800D398202B0AD1284B93F80832DBB2002B04D18C
S3150800D3A8FF222649234805F07EFA254B93F8423092
S3150800D3B8DBB2202B04D1FF222249214805F073FA53
S3150800D3C81C4B93F84130DBB2212B19D11A4BD3F8F1
S3150800D3D80C32002B14D001F051FA0246164BD3F83A
S3150800D3E80C32D31A642B0BD9124805F0B9FA002265
S3150800D3F81021154803F049FA0F4B0022C3F80C22EE
S3150800D4080D4B93F80832DBB2002B11D0094B93F871
S3150800D4184130DBB2212B0BD00C4800F0DFF9FF2294
S3150800D4280649044805F03FFA034B002283F8082208
S3150800D43800BF80BDF40F0020900A0020900B002042
S3150800D448640F0020A00D002000140140900C002055
S3150800D45880B582B000AF78600B467B807B681A6817
S3150800D4681C4B1B689A4216D17B881A461A491B48D0
S3150800D47800F080F90346002B04D11422002100206D
S3150800D48800F0ECF8164B00221A70FF2212491148D0
S3150800D49805F009FA19E07B681A68124B1B689A4264
S3150800D4A813D17B881A461049104800F063F90346D9
S3150800D4B8002B05D00A4B01221A700D4800F08EF988
S3150800D4C8FF220949074805F0EEF900BF0837BD46A7
S3150800D4D880BD00BFF40F0020900B0020900A0020A2
S3150800D4E8B00E0020640F0020A00D0020A00C00201C
S3150800D4F8A00E002080B582B000AF78607B681A68F5
S3150800D508084B1B689A4208D100221021064803F0E6
S3150800D518BCF9064B0022C3F80C2200BF0837BD46E3
S3150800D52880BD00BFF40F002000140140900A0020B7
S3150800D53880B485B000AF78600B467B804FF0FF3328
S3150800D548FB6000237B8121E07B897A6813441B787A
S3150800D5581A46FB685340FB6000237B7210E0FB68A1
S3150800D56803F00103002B05D0FB685A080D4B5340FE
S3150800D578FB6002E0FB685B08FB607B7A01337B7221
S3150800D5887B7A072BEBD97B8901337B817A897B8860
S3150800D5989A42D9D3FB68DB4318461437BD4680BC84
S3150800D5A8704700BF2083B8ED80B588B000AFF86033
S3150800D5B87A601A460B467B8113467B720023FB83E7
S3150800D5C8FB8B5A1CFA831A467B6813447A7A1A70B4
S3150800D5D8FB68002B19D00023BB8312E0BB8BFA68C3
S3150800D5E81A44FB8B591CF98319467B680B44127835
S3150800D5F81A70FB8BFA2B01D900232AE0BB8B01335F
S3150800D608BB83BA8B7B899A42E8D3FB8B1946786821
S3150800D618FFF78EFF03463B6107F110037B61002382
S3150800D628BB6112E0BB697A691A44FB8B591CF983FA
S3150800D63819467B680B4412781A70FB8BFE2B01D9A6
S3150800D648002306E0BB690133BB61BB69032BE9DD2F
S3150800D658FB8B18462037BD4680BD000080B584B0D0
S3150800D66800AF78600B467B8013467B707B78798899
S3150800D678154A7868FFF798FF0346FB81FB89002B54
S3150800D6881ED0124B93F84130DBB2212B07D10F4835
S3150800D69805F066F9002210210D4803F0F6F8012274
S3150800D6A810210B4803F0F1F8FB891A460649074882
S3150800D6B805F0C4F801F0E2F80346034AC2F80C324A
S3150800D6C800BF1037BD4680BD900A0020F40F002021
S3150800D6D80014014080B588B000AFF8600B467A6040
S3150800D6E87B817B89042B01D800233FE07B89B3F52E
S3150800D6F8807F01D9002339E07B89043BFB83FB8BB8
S3150800D708FA6813441B781946FB8B0133FA681344E5
S3150800D7181B781B0241EA0302FB8B0233F9680B44A8
S3150800D7281B781B041A43FB8B0333F9680B441B78D5
S3150800D7381B061343BB61FB8B1946F868FFF7F8FE0F
S3150800D7487861BA697B699A4201D000230EE0FB68C2
S3150800D7585A1C7B685A60FB681A787B681A70FB8BB8
S3150800D768DBB2013BDAB27B685A70012318462037C8
S3150800D778BD4680BD80B584B000AFF860B960134671
S3150800D788FB80FB6803F50072FB881946B868FFF743
S3150800D798A1FF0346002B01D1002304E0FB68012200
S3150800D7A883F80822012318461037BD4680BD0000B5
S3150800D7B880B400AFBFF34F8F00BF064BDB6803F496
S3150800D7C8E0620449044B1343CB60BFF34F8F00BF95
S3150800D7D800BFFDE700ED00E00400FA0580B584B057
S3150800D7E800AF78601323FB737B681B78C22B00F3A2
S3150800D7F8CD80B02B0FDA602B42D0602B00F3C680A1
S3150800D808502B43D0502B00F3C180012B00F0A78082
S3150800D818402B2DD0BAE0B03B122B00F2B78001A2FC
S3150800D82852F823F09BD8000895D9000895D900081E
S3150800D83895D9000895D900084BD9000895D9000844
S3150800D84895D9000895D9000895D9000895D90008EA
S3150800D85895D9000895D9000895D9000895D90008DA
S3150800D86895D90008E1D8000845D9000819D900084B
S3150800D87800F0B2F8402258214B48FFF7EFFE90E037
S3150800D88860220A214948FFF7E9FE8AE0FDF7DCFD30
S3150800D89887E07B685B780B2B1BD17B685A68444BFF
S3150800D8A81068516803C31189927A19809A70FCF72F
S3150800D8B89BFA404B01221A70FCF796FA3C4BD3F8B0
S3150800D8C803303B4A3C490720FDF720FE1223FB7329
S3150800D8D85FE01323FB735CE07B685B78012B14D14C
S3150800D8E87B685B681B781A464FF47A7302FB03F366
S3150800D8F81A46324B5A61314B5B691A46304907203A
S3150800D908FDF704FE1223FB7343E01323FB7340E081
S3150800D9187B685B78012B0ED17B685B681A78294B84
S3150800D9281A70284B1B781A4627490720FDF7EEFD7B
S3150800D9381223FB732DE01323FB732AE01323FB73CF
S3150800D94827E0122200210020FFF788FE00BF1F4BA0
S3150800D95893F84130DBB2212BF9D0FFF729FF7B6812
S3150800D9685B78092B0FD17B685A68194B1068516880
S3150800D97803C3127A1A70174B1B78DBB2012B0FD028
S3150800D9881223FB7305E01323FB7302E01323FB73CF
S3150800D99800BFFB7B1A4600210020FFF75FFE00E068
S3150800D9A800BF1037BD4680BDB40E00200C0F0020FE
S3150800D9B86C000020160F0020806C01080C0A002055
S3150800D9C8946C0108F8020020A86C0108F40F0020DE
S3150800D9D860000020B00E0020B0B500AF9D4B9A78C5
S3150800D9E89D4B9A709B4BD3F807309B4AC2F8033075
S3150800D9F8984BB3F80F309AB2974BA3F80720954B74
S3150800DA08B3F81B309AB2944BA3F80920914BB3F894
S3150800DA1813309AB2904BA3F80B208E4BB3F81530F7
S3150800DA289AB28D4BA3F80D208A4B1A7E8A4BDA7365
S3150800DA38884B5A7F884B5A70864B5A78864B1A7089
S3150800DA48854B00221A7400225A74834B00229A7452
S3150800DA58814B0022DA7400221A750420FBF7A6FE09
S3150800DA68034603F00103D9B27B4A537D61F30003E9
S3150800DA7853750320FBF79AFE034603F00103D9B250
S3150800DA88754A537D61F3410353750020FBF78EFEF3
S3150800DA98034603F00103D9B26F4A537D61F3820343
S3150800DAA85375FEF7C1F9034603F00103D9B26A4A6A
S3150800DAB8537D61F3C30353750320FBF787FE0346BB
S3150800DAC8002B0CBF01230023D9B2634A537D61F3A7
S3150800DAD804135375FDF7A4FC0346002B14BF012352
S3150800DAE80023D9B25C4A537D61F3451353755B4BE2
S3150800DAF81B7803F00103D9B2574A537D61F386139D
S3150800DB085375574B1B7A03F00103D9B2524A537D12
S3150800DB1861F3C71353750020FBF73CFF03465AB257
S3150800DB284D4B5A760120FBF735FF03465AB24A4B46
S3150800DB389A764B4BDB695AB2474BDA76494B5B7890
S3150800DB485AB2454B1A77474BDB785AB2424B5A7743
S3150800DB58454B9B889AB2404BDA83424B9A793E4B9F
S3150800DB6883F82020414B9B689AB23B4BA3F82120A7
S3150800DB783E4BDB689AB2384BA3F823203B4B1B690C
S3150800DB889AB2354BA3F82520334B394A273318322E
S3150800DB98156854689068D1681D605C609860D9609B
S3150800DBA8127C1A74324BDA782B4B83F83820304BB0
S3150800DBB89B889AB2284BA3F839202D4BDB889AB252
S3150800DBC8254BA3F83B202A4B9B681A46224BC3F8D9
S3150800DBD83D20274BDB68204AC2F84130244B9A7C03
S3150800DBE81D4B83F84720224B5A7C1B4B83F846204B
S3150800DBF81F4B1A7C184B83F845201D4BDA7C197D78
S3150800DC0809020A435B7D1B0413439AB2124BA3F815
S3150800DC184820174B9A7D104B83F84A200E4B144A16
S3150800DC284B3329321168526819605A600A4B002228
S3150800DC3883F85320084B002283F85420002283F8DF
S3150800DC485520054B002283F85620002283F85720D2
S3150800DC5800BFB0BDF8020020B40E0020290300203A
S3150800DC680C0A0020A403002098030020E0090020DD
S3150800DC784403002080B500AF024800F0A5F8034623
S3150800DC88184680BD7C0A002080B582B000AF78604F
S3150800DC987968034800F0C8F800BF0837BD4680BD54
S3150800DCA87C0A002080B483B000AF78607B680F4A8E
S3150800DCB882FB03129210DB17D31A5BB21B0158B208
S3150800DCC87A680A4B83FB02139910D317C91A0B46AD
S3150800DCD89B000B445B00D11A4BB203435BB2DBB221
S3150800DCE818460C37BD4680BC704700BF676666662F
S3150800DCF890B587B000AF78603960796800200A4621
S3150800DD080346C7E9022307F10803184606F01EFA70
S3150800DD1878617B691B681846FFF7C4FF03461A46ED
S3150800DD283B681A707B695A683B685C1C1046FFF7A3
S3150800DD38B9FF034623707B699A683B689C1C1046A2
S3150800DD48FFF7B0FF034623707B69DA683B68DC1C7B
S3150800DD581046FFF7A7FF034623707B691B695A1C01
S3150800DD683B681C1D1046FFF79DFF034623707B6919
S3150800DD785B6903F26C73134A82FB03125111DA17B3
S3150800DD888A1A642101FB02F29A1A3B685C1D10463E
S3150800DD98FFF788FF034623707B695B6903F26C7398
S3150800DDA8084A82FB03125211DB17D21A3B689C1DDC
S3150800DDB81046FFF777FF0346237000BF1C37BD469A
S3150800DDC890BD00BF1F85EB5180B487B000AF78605F
S3150800DDD800237B8200233B820023FB8100237B618F
S3150800DDE87B681B689B697B827B681B68DB69FB8190
S3150800DDF87B681B689B693B827A8A3B8A9A4208D069
S3150800DE083B8A1A047B681B68DB699BB213437B61F0
S3150800DE1804E07B8A1A04FB8913437B617B691846ED
S3150800DE281C37BD4680BC704780B584B000AF7860A3
S3150800DE3839600023FB73786800F01DF80346002B49
S3150800DE4802D00123FB7311E07B681B683A68120C41
S3150800DE589A617B681B683A6892B2DA61786800F05A
S3150800DE6832F80346002B01D00123FB73FB7B1846C7
S3150800DE781037BD4680BD80B584B000AF78600023F2
S3150800DE88FB6000F0FBFCF86009E000F0F7FC0246CE
S3150800DE98FB68D31AB3F57A7F01D903230FE07B68A9
S3150800DEA81B685B6803F02003002BEED07B681B68B1
S3150800DEB85A687B681B6842F010025A6000231846A5
S3150800DEC81037BD4680BD80B584B000AF78600023A2
S3150800DED8FB607B681B685A687B681B6822F010021F
S3150800DEE85A6000F0CBFCF86009E000F0C7FC02466F
S3150800DEF8FB68D31AB3F57A7F01D9032307E07B6851
S3150800DF081B685B6803F02003002BEED00023184635
S3150800DF181037BD4680BD000080B485B000AF154BEC
S3150800DF289B69144A43F001039361124B9B6903F0FA
S3150800DF380103BB60BB680F4BDB690E4A43F080538D
S3150800DF48D3610C4BDB6903F080537B607B680A4B13
S3150800DF585B68FB60FB6823F0E063FB60FB6843F0E3
S3150800DF680073FB60044AFB68536000BF1437BD465C
S3150800DF7880BC7047001002400000014080B400AF22
S3150800DF8800BFFDE780B400AF00BFFDE780B400AF6F
S3150800DF9800BFFDE780B400AF00BFFDE780B400AF5F
S3150800DFA800BFFDE780B400AF00BFBD4680BC704720
S3150800DFB880B400AF00BFBD4680BC704780B400AFD0
S3150800DFC800BFBD4680BC704780B500AF00F044FC72
S3150800DFD800BF80BD80B500AF024801F035FE00BF1E
S3150800DFE880BD00BFA402002080B500AF024804F037
S3150800DFF8CBFD00BF80BD00BFAC0F002080B500AFC9
S3150800E008024804F0C1FD00BF80BD00BFF40F002020
S3150800E01880B500AF024804F0B7FD00BF80BD00BF59
S3150800E0283C10002080B500AF024804F0ADFD00BFE3
S3150800E03880BD00BF640F002080B500AF024801F01C
S3150800E04803FE00BF80BD00BFCC02002080B500AF2C
S3150800E058024801F0F9FD00BF80BD00BFCC020020D0
S3150800E06880B400AF01231846BD4680BC704780B50A
S3150800E07882B000AF7860396006F02EF9034616229A
S3150800E0881A604FF0FF3318460837BD4680BD80B57D
S3150800E09882B000AF78604FF0FF317868FFF7E7FF86
S3150800E0A800BFFDE780B586B000AFF860B9607A6052
S3150800E0B800237B610AE0AFF300800146BB685A1C5F
S3150800E0C8BA60CAB21A707B6901337B617A697B6860
S3150800E0D89A42F0DB7B6818461837BD4680BD80B47F
S3150800E0E883B000AF78604FF0FF3318460C37BD464B
S3150800E0F880BC704780B483B000AF786039603B68ED
S3150800E1084FF400525A60002318460C37BD4680BCA7
S3150800E118704780B483B000AF7860012318460C377F
S3150800E128BD4680BC704780B485B000AFF860B9605A
S3150800E1387A60002318461437BD4680BC704700002D
S3150800E14880B586B000AF7860144A154BD31A7B6140
S3150800E1587B693B61134B1B68002B02D1114B124A92
S3150800E1681A60104B1A687B6813443A699A4207D2B0
S3150800E17806F0B2F803460C221A604FF0FF3309E09E
S3150800E188084B1B68FB60074B1A687B681344054AEB
S3150800E1981360FB6818461837BD4680BD0000012085
S3150800E1A800040000180F0020D811002080B400AF22
S3150800E1B800BFBD4680BC704780B58EB000AF07F17A
S3150800E1C8280300221A605A609A60DA6007F1200369
S3150800E1D800221A605A603B1D00221A605A609A602B
S3150800E1E8DA601A615A619A61374B384A1A60364BAF
S3150800E1F84FF434725A60344B00229A60324B6422C8
S3150800E208DA60314B00221A612F4B00229A612E4898
S3150800E21803F0C9FC0346002B01D0FEF7B9F84FF402
S3150800E2288053BB6207F128031946274803F0CEFE38
S3150800E2380346002B01D0FEF7ABF8234803F002FD8E
S3150800E2480346002B01D0FEF7A3F800233B62002300
S3150800E2587B6207F1200319461B4804F039FA03467E
S3150800E268002B01D0FEF794F860237B600023BB607F
S3150800E2780023FB6000237B613B1D042219461248D4
S3150800E28803F0E2FD0346002B01D0FEF781F83B1D9B
S3150800E298082219460C4803F0D7FD0346002B01D07F
S3150800E2A8FEF776F83B1D0C221946074803F0CCFD05
S3150800E2B80346002B01D0FEF76BF8034800F026F852
S3150800E2C800BF3837BD4680BD1C0F00200008004037
S3150800E2D880B485B000AF78607B681B68094A9342AA
S3150800E2E80BD1094BDB69084A43F00403D361064B93
S3150800E2F8DB6903F00403FB60FB6800BF1437BD46FF
S3150800E30880BC7047000800400010024080B588B0FD
S3150800E31800AF786007F10C0300221A605A609A6009
S3150800E328DA607B681B68174A934226D1164B9B69A5
S3150800E338154A43F020039361134B9B6903F02003A6
S3150800E348BB60BB684FF46043FB6002233B61022352
S3150800E358BB6107F10C0319460C4802F0FBF80C4B95
S3150800E3685B68FB61FB6943F0E063FB61FB6943F4A7
S3150800E3788053FB61064AFB69536000BF2037BD46D8
S3150800E38880BD00BF0008004000100240001401408C
S3150800E3980000014080B500AF114B124A1A60104BB5
S3150800E3A84FF416525A600E4B00229A600C4B002204
S3150800E3B8DA600B4B00221A61094B0C225A61084B8A
S3150800E3C800229A61064B0022DA61054804F0E6F94C
S3150800E3D80346002B01D0FDF7DBFF00BF80BD00BF59
S3150800E3E8640F00200050004080B500AF114B124A58
S3150800E3F81A60104B4FF4E1325A600E4B00229A60AD
S3150800E4080C4B0022DA600B4B00221A61094B0C22CE
S3150800E4185A61084B00229A61064B0022DA610548C0
S3150800E42804F0BCF90346002B01D0FDF7B1FF00BF85
S3150800E43880BD00BFAC0F00200038014080B500AF92
S3150800E448114B124A1A60104B4FF4E1325A600E4BC0
S3150800E45800229A600C4B0022DA600B4B00221A61E4
S3150800E468094B0C225A61084B00229A61064B002276
S3150800E478DA61054804F092F90346002B01D0FDF746
S3150800E48887FF00BF80BD00BFF40F0020004400408E
S3150800E49880B500AF114B124A1A60104B4FF4E1329F
S3150800E4A85A600E4B00229A600C4B0022DA600B4B1E
S3150800E4B800221A61094B0C225A61084B00229A61FC
S3150800E4C8064B0022DA61054804F068F90346002B72
S3150800E4D801D0FDF75DFF00BF80BD00BF3C100020DE
S3150800E4E80048004080B592B000AF786007F1300365
S3150800E4F800221A605A609A60DA607B681B68954A37
S3150800E508934245D1944BDB69934A43F48013D3610C
S3150800E518914BDB6903F48013FB62FB6A8E4B9B699C
S3150800E5288D4A43F0100393618B4B9B6903F01003E4
S3150800E538BB62BB6A884B9B69874A43F02003936191
S3150800E548854B9B6903F020037B627B6A4FF48053F3
S3150800E5583B6302237B630323FB6307F130031946F6
S3150800E5687E4801F0F7FF04233B6300237B630023FF
S3150800E578BB6307F130031946794801F0EBFF00221F
S3150800E5880021352001F051FE352001F06AFEDCE055
S3150800E5987B681B68734A93423AD16F4B9B696E4AEC
S3150800E5A843F4804393616C4B9B6903F480433B6255
S3150800E5B83B6A694B9B69684A43F004039361664B57
S3150800E5C89B6903F00403FB61FB694FF400733B6323
S3150800E5D802237B630323FB6307F13003194662486A
S3150800E5E801F0B8FF4FF480633B6300237B63002385
S3150800E5F8BB6307F1300319465B4801F0ABFF0022FD
S3150800E6080021252001F011FE252001F02AFE9CE0B4
S3150800E6187B681B68554A934246D14F4BDB694E4A7D
S3150800E62843F40033D3614C4BDB6903F40033BB6115
S3150800E638BB69494B9B69484A43F020039361464B9B
S3150800E6489B6903F020037B617B6920233B630223D4
S3150800E6587B630323FB6307F130031946404801F03F
S3150800E66879FF40233B6300237B630023BB6307F1E1
S3150800E678300319463A4801F06DFF3D4B5B683B6429
S3150800E6883B6C43F0E0633B643B6C43F008033B6434
S3150800E698374A3B6C536000220021262001F0C5FD4D
S3150800E6A8262001F0DEFD50E07B681B68314A93425C
S3150800E6B84BD1294BDB69284A43F48023D361264B7F
S3150800E6C8DB6903F480233B613B69234B9B69224A38
S3150800E6D843F010039361204B9B6903F01003FB601A
S3150800E6E8FB684FF480633B6302237B630323FB6366
S3150800E6F807F130031946194801F02CFF4FF4006357
S3150800E7083B6300237B630023BB6307F13003194689
S3150800E718124801F01FFF164B5B687B647B6C23F07D
S3150800E72830037B647B6C43F0E0637B647B6C43F06B
S3150800E73810037B640E4A7B6C536000220021272055
S3150800E74801F073FD272001F08CFD00BF4837BD4650
S3150800E75880BD00BF00500040001002400010014074
S3150800E76800140140003801400008014000440040F8
S3150800E7780000014000480040DFF834D0FFF716FDD6
S3150800E7880C480D490D4A002302E0D458C4500433F6
S3150800E798C4188C42F9D30A4A0A4C002301E01360CC
S3150800E7A80432A242FBD305F09DFDFDF703FD704731
S3150800E7B800000120000000204C020020F470010827
S3150800E7C850020020D4110020FEE7000080B500AFF3
S3150800E7D8084B1B68074A43F010031360032001F02F
S3150800E7E819FD0F2000F008F8FFF796FB00231846D6
S3150800E7F880BD00BF0020024080B582B000AF7860B7
S3150800E808124B1A68124B1B7819464FF47A73B3FBE6
S3150800E818F1F3B2FBF3F3184601F031FD0346002B7A
S3150800E82801D001230EE07B680F2B0AD800227968ED
S3150800E8384FF0FF3001F0F9FC064A7B6813600023A5
S3150800E84800E0012318460837BD4680BD7800002039
S3150800E858800000207C00002080B400AF054B1B78A0
S3150800E8681A46054B1B681344034A136000BFBD4686
S3150800E87880BC7047800000208410002080B400AF58
S3150800E888024B1B681846BD4680BC7047841000209A
S3150800E89880B584B000AF7860FFF7F0FFB8607B6892
S3150800E8A8FB60FB68B3F1FF3F05D00A4B1B781A4695
S3150800E8B8FB681344FB6000BFFFF7E0FF0246BB682E
S3150800E8C8D31AFA689A42F7D800BF00BF1037BD4670
S3150800E8D880BD00BF8000002080B586B000AF786094
S3150800E8E80023FB7500233B610023BB600023FB6004
S3150800E8F87B68002B01D10123BEE07B689B68002B4F
S3150800E9087B689B6A002B09D17B680022DA627B68E0
S3150800E918002283F824207868FAF790FE786800F0D1
S3150800E928F1FB0346FB757B689B6A03F01003002B13
S3150800E93840F09980FB7D002B40F095807B689B6AA8
S3150800E94823F4885323F0020343F002027B689A6291
S3150800E9587B685A687B68DB691A437B681B7B5B00A4
S3150800E9681343BA681343BB607B689B68B3F5807F1B
S3150800E97803D07B689B68012B02D14FF4807300E0B3
S3150800E98800233A6913433B617B681B7D012B19D128
S3150800E9987B681B7B002B09D17B689B69013B5A0363
S3150800E9A83B69134343F400633B610BE07B689B6A4E
S3150800E9B843F020027B689A627B68DB6A43F00102AF
S3150800E9C87B68DA627B681B685B6823F469417B6845
S3150800E9D81B683A690A435A607B681B689A68284B19
S3150800E9E813407A681268B9680B4393607B689B681A
S3150800E9F8B3F5807F03D07B689B68012B04D17B68BD
S3150800EA081B69013B1B05FB607B681B68DB6A23F4F3
S3150800EA1870017B681B68FA680A43DA627B681B68B8
S3150800EA289A68184B1340BA689A420BD17B68002239
S3150800EA38DA627B689B6A23F0030343F001027B686A
S3150800EA489A6218E07B689B6A23F0120343F0100267
S3150800EA587B689A627B68DB6A43F001027B68DA6244
S3150800EA680123FB7507E07B689B6A43F010027B6805
S3150800EA789A620123FB75FB7D18461837BD4680BD8B
S3150800EA88FDF7E1FFFE0E1FFF80B584B000AF786082
S3150800EA980023FB737B6893F82430012B01D10223EA
S3150800EAA898E07B68012283F82420786800F0D0FA79
S3150800EAB80346FB73FB7B002B40F087807B689B6AC9
S3150800EAC823F4407323F0010343F480727B689A6247
S3150800EAD87B681B68414A934205D1414B5B6803F43E
S3150800EAE87023002B15D17B689B6A23F480127B68F8
S3150800EAF89A627B681B685B6803F48063002B26D0E0
S3150800EB087B689B6A23F4405343F480527B689A6275
S3150800EB181DE07B689B6A43F480127B689A627B686F
S3150800EB281B682F4A934204D07B681B682B4A93427A
S3150800EB380DD12B4B5B6803F48063002B07D07B68E9
S3150800EB489B6A23F4405343F480527B689A627B6835
S3150800EB589B6A03F48053002B06D07B68DB6A23F094
S3150800EB6806027B68DA6202E07B680022DA627B6862
S3150800EB78002283F824207B681B686FF002021A605B
S3150800EB887B681B689B6803F46023B3F5602F13D171
S3150800EB987B681B68114A934205D1114B5B6803F4DD
S3150800EBA87023002B08D17B681B689A687B681B68EA
S3150800EBB842F4A0029A600CE07B681B689A687B6836
S3150800EBC81B6842F480129A6003E07B68002283F887
S3150800EBD82420FB7B18461037BD4680BD0028014017
S3150800EBE80024014080B584B000AF78600023FB7329
S3150800EBF87B6893F82430012B01D102231AE07B683D
S3150800EC08012283F82420786800F07CFA0346FB730F
S3150800EC18FB7B002B09D17B689B6A23F4885323F076
S3150800EC28010343F001027B689A627B68002283F835
S3150800EC382420FB7B18461037BD4680BD90B587B0A3
S3150800EC4800AF7860396000237B610023FB600023EE
S3150800EC583B61FFF713FE78617B681B689B6803F4C2
S3150800EC688073002B0BD07B689B6A43F020027B6875
S3150800EC789A627B68002283F824200123D3E07B6804
S3150800EC881B685B6803F48073002B31D17B681B68AB
S3150800EC98DB6A03F47003002B2AD121E03B68B3F141
S3150800ECA8FF3F1DD03B68002B07D0FFF7E7FD02465C
S3150800ECB87B69D31A3A689A4212D27B681B681B6822
S3150800ECC803F00203002B0BD17B689B6A43F004020E
S3150800ECD87B689A627B68002283F824200323A2E0D3
S3150800ECE87B681B681B6803F00203002BD6D070E00C
S3150800ECF84F4B1C68022002F0FBFC0346B4FBF3F2F8
S3150800ED087B681B6819694B4B0B40002B18D17B682D
S3150800ED181B68D968484B0B40002B11D17B681B68C8
S3150800ED281969464B0B40002B08D17B681B68D968C4
S3150800ED38434B0B40002B01D1142320E029231EE066
S3150800ED487B681B6819693D4B0B40002B06D17B680D
S3150800ED581B68D9683A4B0B40002B0DD07B681B689B
S3150800ED681969384B0B40002B08D17B681B68D96892
S3150800ED78344B0B40002B01D1542300E0FC2302FB43
S3150800ED8803F33B6121E03B68B3F1FF3F1AD03B68C8
S3150800ED98002B07D0FFF772FD02467B69D31A3A683B
S3150800EDA89A420FD2FB683A699A420BD97B689B6AE2
S3150800EDB843F004027B689A627B68002283F8242061
S3150800EDC8032330E0FB680133FB60FB683A699A4223
S3150800EDD8D9D87B681B686FF012021A607B689B6A31
S3150800EDE843F400727B689A627B681B689B6803F425
S3150800EDF86023B3F5602F15D17B681B7B002B11D1D7
S3150800EE087B689B6A23F480727B689A627B689B6A34
S3150800EE1803F48053002B05D17B689B6A43F00102F3
S3150800EE287B689A62002318461C37BD4690BD00BF0A
S3150800EE3878000020244992242449920092244912F1
S3150800EE48922449004992240080B483B000AF7860C0
S3150800EE587B681B68DB6C18460C37BD4680BC704758
S3150800EE6880B485B000AF786039600023FB7300234F
S3150800EE78BB607B6893F82430012B01D10223DCE0C0
S3150800EE887B68012283F824203B685B68062B1CD81C
S3150800EE987B681B68596B3B685A6813469B00134482
S3150800EEA8053B1F2202FA03F3DB4319403B6818683F
S3150800EEB83B685A6813469B001344053B00FA03F25D
S3150800EEC87B681B680A435A633CE03B685B680C2B03
S3150800EED81CD87B681B68196B3B685A6813469B00E5
S3150800EEE81344233B1F2202FA03F3DB4319403B680A
S3150800EEF818683B685A6813469B001344233B00FA74
S3150800EF0803F27B681B680A431A631BE07B681B6865
S3150800EF18D96A3B685A6813469B001344413B1F222B
S3150800EF2802FA03F3DB4319403B6818683B685A68DA
S3150800EF3813469B001344413B00FA03F27B681B689F
S3150800EF480A43DA623B681B68092B1CD97B681B686D
S3150800EF58D9683B681A6813465B0013441E3B0722A8
S3150800EF6802FA03F3DB4319403B6898683B681A685A
S3150800EF7813465B0013441E3B00FA03F27B681B68C2
S3150800EF880A43DA6019E07B681B6819693B681A68DE
S3150800EF9813465B001344072202FA03F3DB431940BE
S3150800EFA83B6898683B681A6813465B00134400FA7E
S3150800EFB803F27B681B680A431A613B681B68102BB7
S3150800EFC803D03B681B68112B32D17B681B681D4A26
S3150800EFD8934225D17B681B689B6803F40003002BC2
S3150800EFE826D17B681B689A687B681B6842F400020E
S3150800EFF89A603B681B68102B1AD1134B1B68134A77
S3150800F008A2FB03239A0C13469B0013445B00BB60C0
S3150800F01802E0BB68013BBB60BB68002BF9D107E07F
S3150800F0287B689B6A43F020027B689A620123FB731C
S3150800F0387B68002283F82420FB7B18461437BD46D4
S3150800F04880BC7047002401407800002083DE1B43FB
S3150800F05880B584B000AF78600023FB600023BB60EE
S3150800F0687B681B689B6803F00103012B40D07B680B
S3150800F0781B689A687B681B6842F001029A601F4BF6
S3150800F0881B681F4AA2FB03239B0CBB6002E0BB68F4
S3150800F098013BBB60BB68002BF9D1FFF7EFFBF860B3
S3150800F0A81FE0FFF7EBFB0246FB68D31A022B18D9B9
S3150800F0B87B681B689B6803F00103012B11D07B68EA
S3150800F0C89B6A43F010027B689A627B68DB6A43F0A6
S3150800F0D801027B68DA627B68002283F82420012310
S3150800F0E807E07B681B689B6803F00103012BD8D1EE
S3150800F0F8002318461037BD4680BD00BF780000209B
S3150800F10883DE1B4380B584B000AF78600023FB60BC
S3150800F1187B681B689B6803F00103012B2ED17B686B
S3150800F1281B689A687B681B6822F001029A60FFF7D9
S3150800F138A5FBF8601BE0FFF7A1FB0246FB68D31A9C
S3150800F148022B14D97B681B689B6803F00103012B03
S3150800F1580DD17B689B6A43F010027B689A627B68CC
S3150800F168DB6A43F001027B68DA62012307E07B6801
S3150800F1781B689B6803F00103012BDCD000231846A3
S3150800F1881037BD4680BD000090B587B000AF7860DF
S3150800F1980023FB750023FB607B6893F82430012B5A
S3150800F1A801D1022397E07B68012283F82420786836
S3150800F1B8FFF7A8FF0346FB757868FFF749FF03467C
S3150800F1C8FB75FB7D002B40F081807B689B6A23F4E6
S3150800F1D8885323F0020343F002027B689A62404B85
S3150800F1E81C68022002F084FA0346B4FBF3F35B00BA
S3150800F1F8FB6002E0FB68013BFB60FB68002BF9D16A
S3150800F2087B681B689A687B681B6842F008029A60E4
S3150800F218FFF734FB38611BE0FFF730FB02463B6912
S3150800F228D31A0A2B14D97B681B689B6803F0080352
S3150800F238002B0DD07B689B6A23F0120343F010025B
S3150800F2487B689A627B68002283F82420012342E0BF
S3150800F2587B681B689B6803F00803002BDCD17B6876
S3150800F2681B689A687B681B6842F004029A60FFF775
S3150800F27805FB38611BE0FFF701FB02463B69D31A19
S3150800F2880A2B14D97B681B689B6803F00403002BB8
S3150800F2980DD07B689B6A23F0120343F010027B6843
S3150800F2A89A627B68002283F82420012313E07B688E
S3150800F2B81B689B6803F00403002BDCD17B689B6AF8
S3150800F2C823F0030343F001027B689A627B680022F5
S3150800F2D883F82420FB7D18461C37BD4690BD00BF21
S3150800F2E87800002080B584B000AF78607B68002B72
S3150800F2F801D10123EDE07B6893F82030DBB2002BBF
S3150800F30802D17868FAF714FC7B681B681A687B6868
S3150800F3181B6842F001021A60FFF7B0FAF86012E0BB
S3150800F328FFF7ACFA0246FB68D31A0A2B0BD97B6897
S3150800F3385B6A43F400327B685A627B68052283F865
S3150800F34820200123C5E07B681B685B6803F001037E
S3150800F358002BE5D07B681B681A687B681B6822F057
S3150800F36802021A60FFF78AFAF86012E0FFF786FACF
S3150800F3780246FB68D31A0A2B0BD97B685B6A43F4E7
S3150800F38800327B685A627B68052283F820200123AD
S3150800F3989FE07B681B685B6803F00203002BE5D1D6
S3150800F3A87B681B7E012B08D17B681B681A687B68FB
S3150800F3B81B6842F080021A6007E07B681B681A68B7
S3150800F3C87B681B6822F080021A607B685B7E012BCB
S3150800F3D808D17B681B681A687B681B6842F040027C
S3150800F3E81A6007E07B681B681A687B681B6822F046
S3150800F3F840021A607B689B7E012B08D17B681B68D4
S3150800F4081A687B681B6842F020021A6007E07B6866
S3150800F4181B681A687B681B6822F020021A607B68DA
S3150800F428DB7E012B08D17B681B681A687B681B681A
S3150800F43822F010021A6007E07B681B681A687B6866
S3150800F4481B6842F010021A607B681B7F012B08D1E3
S3150800F4587B681B681A687B681B6842F008021A6092
S3150800F46807E07B681B681A687B681B6822F0080235
S3150800F4781A607B685B7F012B08D17B681B681A6852
S3150800F4887B681B6842F004021A6007E07B681B6801
S3150800F4981A687B681B6822F004021A607B689A68F7
S3150800F4A87B68DB681A437B681B691A437B685B6958
S3150800F4B842EA03017B685B685A1E7B681B680A4335
S3150800F4C8DA617B6800225A627B68012283F8202069
S3150800F4D8002318461037BD4680BD000080B487B0A3
S3150800F4E800AF786039607B681B687B617B6893F836
S3150800F4F82030FB74FB7C012B03D0FB7C022B40F0ED
S3150800F508BE80654B7B617B69D3F8003243F0010204
S3150800F5187B69C3F800227B69D3F8003223F47C524E
S3150800F5287B69C3F800227B69D3F800223B685B6ACB
S3150800F5381B021A437B69C3F800223B685B6903F020
S3150800F5481F03012202FA03F3FB607B69D3F81C2226
S3150800F558FB68DB431A407B69C3F81C223B68DB69F6
S3150800F568002B23D17B69D3F80C22FB68DB431A40AE
S3150800F5787B69C3F80C223B68DB6819043B685B683F
S3150800F5889BB23A68526919437B69483243F8321084
S3150800F5983B689B6819043B681B689AB23B685B69B9
S3150800F5A80A4379694833DB000B445A603B68DB69D0
S3150800F5B8012B22D17B69D3F80C22FB681A437B6995
S3150800F5C8C3F80C223B681B6819043B685B689BB246
S3150800F5D83A68526919437B69483243F832103B68DE
S3150800F5E89B6819043B68DB689AB23B685B690A43FF
S3150800F5F879694833DB000B445A603B689B69002BE2
S3150800F60809D17B69D3F80422FB68DB431A407B6976
S3150800F618C3F8042207E07B69D3F80422FB681A4377
S3150800F6287B69C3F804223B681B69002B09D17B69EF
S3150800F638D3F81422FB68DB431A407B69C3F8142203
S3150800F64807E07B69D3F81422FB681A437B69C3F879
S3150800F65814223B681B6A012B07D17B69D3F81C2245
S3150800F668FB681A437B69C3F81C227B69D3F8003206
S3150800F67823F001027B69C3F80022002306E07B68B1
S3150800F6885B6A43F480227B685A62012318461C3752
S3150800F698BD4680BC704700BF0064004080B584B092
S3150800F6A800AF78607B6893F82030DBB2012B2ED147
S3150800F6B87B68022283F820207B681B681A687B68A7
S3150800F6C81B6822F001021A60FFF7D8F8F86012E002
S3150800F6D8FFF7D4F80246FB68D31A0A2B0BD97B68BE
S3150800F6E85B6A43F400327B685A627B68052283F8B2
S3150800F6F82020012312E07B681B685B6803F001037E
S3150800F708002BE5D17B6800225A62002306E07B6855
S3150800F7185B6A43F400227B685A620123184610374D
S3150800F728BD4680BD80B584B000AF78607B6893F825
S3150800F7382030DBB2022B33D17B681B681A687B68DA
S3150800F7481B6842F001021A60FFF798F8F86012E0A1
S3150800F758FFF794F80246FB68D31A0A2B0BD97B687D
S3150800F7685B6A43F400327B685A627B68052283F831
S3150800F778202001231BE07B681B685B6803F00103F4
S3150800F788002BE5D07B681B681A687B681B6822F023
S3150800F79802021A607B68012283F82020002306E00B
S3150800F7A87B685B6A43F480127B685A6201231846B1
S3150800F7B81037BD4680BD80B489B000AFF860B9601F
S3150800F7C87A603B60FB6893F82030FB77FB681B6818
S3150800F7D89B68BB61FB7F012B03D0FB7F022B40F0A4
S3150800F7E8AD80BB6903F08063002B0AD1BB6903F0BF
S3150800F7F80063002B05D1BB6903F08053002B00F08A
S3150800F8089580BB691B0E03F003037B6101227B69A4
S3150800F8189A403B681A60BB689B68002B0DD1BB6889
S3150800F8281B685A05BB68DB68F96809681A437B6967
S3150800F83818331B010B441A600FE0BB685B68DA00D3
S3150800F848BB689B681A43BB68DB68F96809681A438A
S3150800F8587B6918331B010B441A60FB681968BB6877
S3150800F8681A697B6918331B010B4404331A60BB6891
S3150800F8781B7D012B11D1FB681A687B6918331B019C
S3150800F888134404331B68FA68116843F480727B6969
S3150800F89818331B010B4404331A607B6807331B783B
S3150800F8A81A067B6806331B781B041A437B680533DC
S3150800F8B81B781B0213437A68043212781046FA68D2
S3150800F8C8116843EA00027B691B010B4403F5C673FA
S3150800F8D81A607B6803331B781A067B6802331B7821
S3150800F8E81B041A437B6801331B781B0213437A6887
S3150800F8F812781046FA68116843EA00027B691B0108
S3150800F9080B4403F5C4731A60FB681A687B691833D5
S3150800F9181B0113441B68FA68116843F001027B69E6
S3150800F92818331B010B441A6000230EE0FB685B6A58
S3150800F93843F40012FB685A62012306E0FB685B6A17
S3150800F94843F48022FB685A62012318462437BD46C9
S3150800F95880BC704780B485B000AF78600023FB6030
S3150800F9687B6893F82030FB72FB7A012B02D0FB7A6E
S3150800F978022B1DD17B681B689B6803F08063002BEC
S3150800F98802D0FB680133FB607B681B689B6803F041
S3150800F9980063002B02D0FB680133FB607B681B6899
S3150800F9A89B6803F08053002B02D0FB680133FB6089
S3150800F9B8FB6818461437BD4680BC704780B487B0C4
S3150800F9C800AFF860B9607A603B60FB6893F820304E
S3150800F9D8FB75FB7D012B03D0FB7D022B40F00381D1
S3150800F9E8BB68002B0ED1FB681B68DB6803F00303B2
S3150800F9F8002B16D1FB685B6A43F40012FB685A624F
S3150800FA080123F7E0FB681B681B6903F00303002B57
S3150800FA1807D1FB685B6A43F40012FB685A62012344
S3150800FA28E8E0FB681A68BB681B331B0113441B68AC
S3150800FA3803F004027B689A607B689B68002B0CD1EC
S3150800FA48FB681A68BB681B331B0113441B685B0DEC
S3150800FA58C3F30A027B681A600BE0FB681A68BB687E
S3150800FA681B331B0113441B68DB0823F060427B68C1
S3150800FA785A60FB681A68BB681B331B0113441B686A
S3150800FA8803F002027B68DA60FB681A68BB681B33F6
S3150800FA981B01134404331B6803F00803002B03D027
S3150800FAA87B6808221A610BE0FB681A68BB681B3377
S3150800FAB81B01134404331B6803F00F027B681A61A1
S3150800FAC8FB681A68BB681B331B01134404331B689D
S3150800FAD81B0ADAB27B689A61FB681A68BB681B332B
S3150800FAE81B01134404331B681B0C9AB27B685A61C2
S3150800FAF8FB681A68BB681B01134403F5DC731B68AB
S3150800FB08DAB23B681A70FB681A68BB681B011344AB
S3150800FB1803F5DC731B681A0A3B680133D2B21A70FC
S3150800FB28FB681A68BB681B01134403F5DC731B687A
S3150800FB381A0C3B680233D2B21A70FB681A68BB689B
S3150800FB481B01134403F5DC731B681A0E3B68033361
S3150800FB58D2B21A70FB681A68BB681B01134403F50E
S3150800FB68DE731A683B680433D2B21A70FB681A68DF
S3150800FB78BB681B01134403F5DE731B681A0A3B6846
S3150800FB880533D2B21A70FB681A68BB681B0113449E
S3150800FB9803F5DE731B681A0C3B680633D2B21A7073
S3150800FBA8FB681A68BB681B01134403F5DE731B68F8
S3150800FBB81A0E3B680733D2B21A70BB68002B08D1F5
S3150800FBC8FB681B68DA68FB681B6842F02002DA6083
S3150800FBD807E0FB681B681A69FB681B6842F0200285
S3150800FBE81A61002306E0FB685B6A43F48022FB6817
S3150800FBF85A62012318461C37BD4680BC704780B434
S3150800FC0885B000AF786039607B6893F82030FB735D
S3150800FC18FB7B012B02D0FB7B022B09D17B681B6877
S3150800FC2859697B681B683A680A435A61002306E0E3
S3150800FC387B685B6A43F480227B685A62012318460C
S3150800FC481437BD4680BC704780B58AB000AF786067
S3150800FC5800237B627B681B685B693B627B681B6861
S3150800FC685B68FB617B681B689B68BB617B681B6874
S3150800FC78DB687B617B681B681B693B617B681B6863
S3150800FC889B69FB603B6A03F00103002B7CD0BB69C8
S3150800FC9803F00103002B23D07B681B6801229A60B6
S3150800FCA8BB6903F00203002B03D0786800F083F9D8
S3150800FCB816E0BB6903F00403002B04D07B6A43F4FF
S3150800FCC800637B620CE0BB6903F00803002B04D0D1
S3150800FCD87B6A43F480537B6202E0786800F086F911
S3150800FCE8BB6903F48073002B24D07B681B684FF428
S3150800FCF880729A60BB6903F40073002B03D0786896
S3150800FD0800F062F916E0BB6903F48063002B04D09F
S3150800FD187B6A43F400537B620CE0BB6903F4006317
S3150800FD28002B04D07B6A43F480437B6202E0786840
S3150800FD3800F065F9BB6903F48033002B24D07B688F
S3150800FD481B684FF480329A60BB6903F40033002BB2
S3150800FD5803D0786800F041F916E0BB6903F48023FC
S3150800FD68002B04D07B6A43F400437B620CE0BB6932
S3150800FD7803F40023002B04D07B6A43F480337B62A8
S3150800FD8802E0786800F044F93B6A03F00803002BA0
S3150800FD980CD07B6903F01003002B07D07B6A43F469
S3150800FDA800737B627B681B681022DA603B6A03F083
S3150800FDB80403002B0BD07B6903F00803002B06D03D
S3150800FDC87B681B680822DA60786800F02AF93B6ABB
S3150800FDD803F00203002B09D07B681B68DB6803F075
S3150800FDE80303002B02D07868FBF7AAFD3B6A03F0E9
S3150800FDF84003002B0CD03B6903F01003002B07D0F7
S3150800FE087B6A43F480637B627B681B6810221A61ED
S3150800FE183B6A03F02003002B0BD03B6903F0080369
S3150800FE28002B06D07B681B6808221A61786800F0E0
S3150800FE3801F93B6A03F01003002B09D07B681B689D
S3150800FE481B6903F00303002B02D07868FCF730FB24
S3150800FE583B6A03F40033002B0BD0FB6903F010034D
S3150800FE68002B06D07B681B6810225A60786800F059
S3150800FE78EAF83B6A03F48033002B0BD0FB6903F0DE
S3150800FE880803002B06D07B681B6808225A60786826
S3150800FE9800F0E2F83B6A03F40043002B7BD0FB69C9
S3150800FEA803F00403002B72D03B6A03F48073002B1B
S3150800FEB808D0FB6803F00103002B03D07B6A43F0E4
S3150800FEC801037B623B6A03F40073002B08D0FB68C6
S3150800FED803F00203002B03D07B6A43F002037B621C
S3150800FEE83B6A03F48063002B08D0FB6803F004031D
S3150800FEF8002B03D07B6A43F004037B623B6A03F456
S3150800FF080063002B43D0FB6803F07003002B3ED038
S3150800FF18FB6803F07003602B2BD0602B2ED8502B70
S3150800FF2822D0502B2AD8402B19D0402B26D8302B34
S3150800FF3810D0302B22D8102B02D0202B05D01DE04C
S3150800FF487B6A43F008037B6219E07B6A43F0100377
S3150800FF587B6214E07B6A43F020037B620FE07B6ACE
S3150800FF6843F040037B620AE07B6A43F080037B62C6
S3150800FF7805E07B6A43F480737B6200E000BF7B6818
S3150800FF881B689A697B681B6822F070029A617B680D
S3150800FF981B6804225A607B6A002B08D07B685A6A59
S3150800FFA87B6A1A437B685A62786800F05EF800BF75
S3150800FFB82837BD4680BD80B483B000AF786000BFDF
S3150800FFC80C37BD4680BC704780B483B000AF7860F4
S3150800FFD800BF0C37BD4680BC704780B483B000AFFD
S3150800FFE8786000BF0C37BD4680BC704780B483B0C4
S3150800FFF800AF786000BF0C37BD4680BC704780B438
S3150801000883B000AF786000BF0C37BD4680BC704727
S3150801001880B483B000AF786000BF0C37BD4680BC9A
S31508010028704780B483B000AF786000BF0C37BD460F
S3150801003880BC704780B483B000AF786000BF0C37C6
S31508010048BD4680BC704780B483B000AF786000BFF6
S315080100580C37BD4680BC704780B483B000AF786062
S3150801006800BF0C37BD4680BC704780B483B000AF6B
S31508010078786000BF0C37BD4680BC704780B485B030
S3150801008800AF78607B6803F00703FB600C4BDB68FD
S31508010098BB60BA684FF6FF031340BB60FB681A02D8
S315080100A8BB68134343F0BF6343F40033BB60044A98
S315080100B8BB68D36000BF1437BD4680BC704700BF14
S315080100C800ED00E080B400AF044BDB681B0A03F0BF
S315080100D807031846BD4680BC704700BF00ED00E01F
S315080100E880B483B000AF0346FB7197F90730002B3C
S315080100F80BDBFB7903F01F02064997F907305B0901
S31508010108012000FA02F241F8232000BF0C37BD4648
S3150801011880BC704700E100E080B483B000AF0346B5
S315080101283960FB7197F90730002B0ADB3B68DAB2AD
S315080101380C4997F907301201D2B20B4483F8002308
S315080101480AE03B68DAB20849FB7903F00F03043B76
S315080101581201D2B20B441A7600BF0C37BD4680BCD1
S31508010168704700BF00E100E000ED00E080B489B007
S3150801017800AFF860B9607A60FB6803F00703FB61B2
S31508010188FB69C3F10703042B28BF0423BB61FB6979
S315080101980433062B02D9FB69033B00E000237B6184
S315080101A84FF0FF32BB6902FA03F3DA43BB681A4018
S315080101B87B699A404FF0FF317B6901FA03F3D9430A
S315080101C87B680B40134318462437BD4680BC7047E5
S315080101D880B582B000AF78607B68013BB3F1807F58
S315080101E801D301230FE00A4A7B68013B53600F21BB
S315080101F84FF0FF30FFF790FF054B00229A60044B3A
S3150801020807221A60002318460837BD4680BD00BF75
S3150801021810E000E080B582B000AF78607868FFF733
S315080102282DFF00BF0837BD4680BD80B586B000AF33
S315080102380346B9607A60FB7300237B61FFF742FFC7
S3150801024878617A68B9687869FFF790FF024697F97D
S315080102580F3011461846FFF75FFF00BF1837BD462E
S3150801026880BD80B582B000AF0346FB7197F90730A8
S315080102781846FFF735FF00BF0837BD4680BD80B56C
S3150801028882B000AF78607868FFF7A2FF0346184680
S315080102980837BD4680BD80B582B000AF78607B68F7
S315080102A8002B01D101230EE07B685B79DBB2002BB9
S315080102B805D17B6800221A717868FBF723F87B68F1
S315080102C801225A71002318460837BD4680BD80B4F5
S315080102D885B000AF78600023FB737B6893F82130FB
S315080102E8DBB2022B08D07B6804229A637B6800225A
S315080102F883F82020012320E07B681B681A687B683D
S315080103081B6822F00E021A607B681B681A687B68EC
S315080103181B6822F001021A607B681A6C7B68DB6B22
S31508010328012101FA02F25A607B68012283F8212029
S315080103387B68002283F82020FB7B18461437BD46C4
S3150801034880BC704780B584B000AF78600023FB7322
S315080103587B6893F82130DBB2022B05D07B6804222F
S315080103689A630123FB73D6E07B681B681A687B6866
S315080103781B6822F00E021A607B681B681A687B687C
S315080103881B6822F001021A607B681B681A46644BCF
S315080103989A4258D97B681B68624A93424FD07B6850
S315080103A81B68614A934248D07B681B685F4A934237
S315080103B840D07B681B685E4A934238D07B681B68C5
S315080103C85C4A934230D07B681B685B4A934228D0C3
S315080103D87B681B68524A934220D07B681B68574A38
S315080103E8934219D07B681B68554A934212D07B6899
S315080103F81B68544A93420AD07B681B68524A93423F
S3150801040802D14FF480531BE04FF4803318E04FF4C0
S31508010418807315E0102313E0012311E04FF0807370
S315080104280EE04FF480130BE04FF4803308E04FF4E5
S31508010438805305E04FF4807302E0102300E001239E
S31508010448424A536057E07B681B68364A93424FD045
S315080104587B681B68344A934248D07B681B68334AD1
S31508010468934240D07B681B68314A934238D07B68EF
S315080104781B68304A934230D07B681B682E4A9342E0
S3150801048828D07B681B68264A934220D07B681B685C
S315080104982A4A934219D07B681B68294A934212D083
S315080104A87B681B68274A93420AD07B681B68264AD9
S315080104B8934202D14FF480531BE04FF4803318E07E
S315080104C84FF4807315E0102313E0012311E04FF070
S315080104D880730EE04FF480130BE04FF4803308E085
S315080104E84FF4805305E04FF4807302E0102300E0CF
S315080104F80123174A53607B68012283F821207B6808
S31508010508002283F820207B685B6B002B03D07B686D
S315080105185B6B78689847FB7B18461037BD4680BDE4
S3150801052880000240080002401C00024030000240D8
S3150801053844000240580002406C0002400804024088
S315080105481C040240300402404404024000040240EC
S315080105580000024080B48BB000AF78603960002390
S315080105687B6200233B6269E101227B6A02FA03F393
S31508010578FB613B681B68FA691340BB61BA69FB6989
S315080105889A4240F058813B685B689A4A93425ED022
S31508010598984A934275D8984A934258D0964A9342AC
S315080105A86FD8964A934252D0944A934269D8944A44
S315080105B893424CD0924A934263D8924A934246D080
S315080105C8904A93425DD8122B2AD8122B59D801A2E0
S315080105D852F823F0570601083106010843060108AF
S315080105E8850601088B0601088B0601088B06010892
S315080105F88B0601088B0601088B0601088B0601087C
S315080106088B0601088B0601088B0601088B0601086B
S315080106188B0601088B060108390601084D060108EB
S31508010628794A934213D02CE03B68DB683B6229E0A0
S315080106383B68DB6804333B6224E03B68DB680833C4
S315080106483B621FE03B68DB680C333B621AE03B6898
S315080106589B68002B02D104233B6213E03B689B6825
S31508010668012B05D108233B627B68FA691A6109E0FF
S3150801067808233B627B68FA695A6103E000233B62F7
S3150801068800E000BFBB69FF2B01D87B6801E07B68E6
S3150801069804337B61BB69FF2B02D87B6A9B0002E0A6
S315080106A87B6A083B9B003B617B691A680F213B699A
S315080106B801FA03F3DB431A40396A3B6901FA03F382
S315080106C81A437B691A603B685B6803F08053002B01
S315080106D800F0B1804D4B9B694C4A43F00103936185
S315080106E84A4B9B6903F00103BB60BB68484A7B6AAE
S315080106F89B08023352F82330FB607B6A03F0030335
S315080107089B000F2202FA03F3DB43FA681340FB60E6
S315080107187B68404A934213D07B683F4A93420DD07F
S315080107287B683E4A934207D07B683D4A934201D18A
S31508010738032306E0042304E0022302E0012300E080
S3150801074800237A6A02F0030292009340FA68134377
S31508010758FB602F497B6A9B080233FA6841F8232014
S315080107683B685B6803F48013002B06D02D4B9A6807
S315080107782C49BB6913438B6006E02A4B9A68BB6907
S31508010788DB43284913408B603B685B6803F4001315
S31508010798002B06D0234BDA682249BB691343CB6081
S315080107A806E0204BDA68BB69DB431E491340CB6078
S315080107B83B685B6803F40033002B06D0194B5A686B
S315080107C81849BB6913434B6006E0164B5A68BB695F
S315080107D8DB43144913404B603B685B6803F4803379
S315080107E8002B21D00F4B1A680E49BB6913430B60BE
S315080107F821E000BF0000321000003110000022106D
S31508010808000021100000121000001110001002400B
S315080108180000014000080140000C01400010014099
S3150801082800140140000401400B4B1A68BB69DB43FD
S31508010838094913400B607B6A01337B623B681A6876
S315080108487B6A22FA03F3002B7FF48EAE00BF00BF42
S315080108582C37BD4680BC70470004014080B485B07A
S3150801086800AF78600B467B807B689A687B88134063
S31508010878002B02D00123FB7301E00023FB73FB7BEA
S3150801088818461437BD4680BC704780B483B000AF9C
S3150801089878600B467B8013467B707B78002B03D0E8
S315080108A87A887B681A6103E07B881A047B681A616F
S315080108B800BF0C37BD4680BC7047000080B400AF46
S315080108C8034B01221A6000BFBD4680BC704700BFB2
S315080108D820000E4280B582B000AFFDF7CFFF7860E1
S315080108E8604B1B685F4A43F00103136008E0FDF794
S315080108F8C5FF02467B68D31A022B01D90323ACE04C
S31508010908584B1B6803F00203002BF0D0554B1B68A4
S3150801091823F0F803534A43F080031360FDF7AEFF4B
S315080109287860504B00225A600AE0FDF7A7FF024695
S315080109387B68D31A41F28832934201D903238CE0A2
S31508010948484B5B6803F00C03002BEED1464B474A2C
S315080109581A60474B1B681846FDF74EFF0346002BDE
S3150801096801D0012379E0FDF789FF78603D4B1B68C3
S315080109783C4A23F08073136008E0FDF77FFF0246BF
S315080109887B68D31A022B01D9032366E0354B1B680A
S3150801099803F00073002BF0D1324B00225A60FDF7A1
S315080109A86DFF78602F4B1B682E4A23F410231360BA
S315080109B808E0FDF763FF02467B68D31A642B01D961
S315080109C803234AE0274B1B6803F40033002BF0D1B5
S315080109D8244B1B68234A23F480231360FDF74EFF33
S315080109E87860204B1B681F4A23F08063136008E070
S315080109F8FDF744FF02467B68D31A642B01D9032302
S31508010A082BE0184B1B6803F00063002BF0D1FDF7A8
S31508010A1835FF7860134B1B68124A23F0805313601D
S31508010A2808E0FDF72BFF02467B68D31A642B01D928
S31508010A38032312E00B4B1B6803F00053002BF0D17C
S31508010A48084B0022DA62074B5B6A064A43F0807351
S31508010A585362044B00229A60002318460837BD469C
S31508010A6880BD00BF001002407800002000127A00FD
S31508010A787C00002080B586B000AF78607B68002BC3
S31508010A8801D1012304E37B681B6803F00103002BEA
S31508010A9800F08780924B5B6803F00C03042B0CD09B
S31508010AA88F4B5B6803F00C03082B12D18C4B5B68E0
S31508010AB803F48033B3F5803F0BD1894B1B6803F4E4
S31508010AC80033002B6CD07B689B68002B68D1012307
S31508010AD8DEE27B689B68B3F5803F06D1804B1B68CD
S31508010AE87F4A43F4803313602EE07B689B68002BAA
S31508010AF80CD17B4B1B687A4A23F480331360784BF5
S31508010B081B68774A23F4802313601DE07B689B687A
S31508010B18B3F5A02F0CD1724B1B68714A43F4802395
S31508010B2813606F4B1B686E4A43F4803313600BE0FE
S31508010B386B4B1B686A4A23F480331360684B1B683E
S31508010B48674A23F4802313607B689B68002B13D0BC
S31508010B58FDF794FE386108E0FDF790FE02463B6909
S31508010B68D31A642B01D9032392E25D4B1B6803F45C
S31508010B780033002BF0D014E0FDF780FE386108E059
S31508010B88FDF77CFE02463B69D31A642B01D9032378
S31508010B987EE2534B1B6803F40033002BF0D100E0C7
S31508010BA800BF7B681B6803F00203002B63D04C4B1C
S31508010BB85B6803F00C03002B0BD0494B5B6803F009
S31508010BC80C03082B1CD1464B5B6803F48033002BB6
S31508010BD816D1434B1B6803F00203002B05D07B682B
S31508010BE85B69012B01D0012352E23D4B1B6823F0B7
S31508010BF8F8027B689B69DB00394913430B603AE0C5
S31508010C087B685B69002B20D0364B01221A60FDF7F9
S31508010C1835FE386108E0FDF731FE02463B69D31A0D
S31508010C28022B01D9032333E22D4B1B6803F0020378
S31508010C38002BF0D02A4B1B6823F0F8027B689B69C6
S31508010C48DB00274913430B6015E0264B00221A607F
S31508010C58FDF714FE386108E0FDF710FE02463B6908
S31508010C68D31A022B01D9032312E21D4B1B6803F081
S31508010C780203002BF0D17B681B6803F00803002BDD
S31508010C883AD07B68DB69002B19D0174B01221A6009
S31508010C98FDF7F4FD386108E0FDF7F0FD02463B690A
S31508010CA8D31A022B01D90323F2E10D4B5B6A03F030
S31508010CB80203002BF0D0012000F0CAFB1CE00A4B06
S31508010CC800221A60FDF7DAFD38610FE0FDF7D6FD57
S31508010CD802463B69D31A022B08D90323D8E100BF78
S31508010CE80010024000004242800442429B4B5B6A64
S31508010CF803F00203002BE9D17B681B6803F00403A0
S31508010D08002B00F0A6800023FB75944BDB6903F0E2
S31508010D188053002B0DD1914BDB69904A43F08053E0
S31508010D28D3618E4BDB6903F08053BB60BB68012333
S31508010D38FB758B4B1B6803F48073002B18D1884B02
S31508010D481B68874A43F480731360FDF797FD38617A
S31508010D5808E0FDF793FD02463B69D31A642B01D9CE
S31508010D68032395E17E4B1B6803F48073002BF0D0AF
S31508010D787B681B69012B06D1784B1B6A774A43F0B6
S31508010D88010313622DE07B681B69002B0CD1734B99
S31508010D981B6A724A23F001031362704B1B6A6F4A76
S31508010DA823F0040313621CE07B681B69052B0CD12D
S31508010DB86A4B1B6A694A43F004031362674B1B6A49
S31508010DC8664A43F0010313620BE0644B1B6A634AE4
S31508010DD823F001031362614B1B6A604A23F004037B
S31508010DE813627B681B69002B15D0FDF747FD38612F
S31508010DF80AE0FDF743FD02463B69D31A41F28832F8
S31508010E08934201D9032343E1544B1B6A03F00203B6
S31508010E18002BEED014E0FDF731FD38610AE0FDF745
S31508010E282DFD02463B69D31A41F28832934201D90C
S31508010E3803232DE1494B1B6A03F00203002BEED16C
S31508010E48FB7D012B05D1454BDB69444A23F08053C9
S31508010E58D3617B68DB6A002B00F08C803F4B5B68AB
S31508010E6803F48033B3F5803F0ED13C4B5B6803F03E
S31508010E780C03082B08D1394BDB6A03F48033B3F525
S31508010E88803F01D1012303E17B68DB6A022B4ED13E
S31508010E98324B1B6803F08053002B09D02F4BDB6AB2
S31508010EA803F0F0027B685B6B9A4201D00123EFE0FD
S31508010EB82C4B00221A60FDF7E1FC386108E0FDF7C2
S31508010EC8DDFC02463B69D31A642B01D90323DFE00B
S31508010ED8224B1B6803F00063002BF0D11F4BDB6A1A
S31508010EE823F0F0027B685B6B1C491343CB621B4BEF
S31508010EF8DB6A23F470627B681B6B18491343CB6260
S31508010F08184B01221A60FDF7B9FC386108E0FDF7AC
S31508010F18B5FC02463B69D31A642B01D90323B7E00A
S31508010F280E4B1B6803F00063002BF0D022E00B4B35
S31508010F38DB6A0A4A23F48033D3620A4B00221A6011
S31508010F48FDF79CFC38610FE0FDF798FC02463B6902
S31508010F58D31A642B08D903239AE000BF001002406C
S31508010F6800700040680042424B4B1B6803F000635F
S31508010F78002BE9D17B681B6A002B00F08880464B59
S31508010F885B6803F00C03082B68D07B681B6A022B85
S31508010F984DD1424B00221A60FDF770FC386108E012
S31508010FA8FDF76CFC02463B69D31A022B01D90323C8
S31508010FB86EE0394B1B6803F00073002BF0D17B6890
S31508010FC85B6AB3F5803F0FD1334BDA6A7B685B6896
S31508010FD831491343CB62304BDB6A23F00F027B6836
S31508010FE8DB682D491343CB622B4B5B6823F47412D8
S31508010FF87B68596A7B689B6A0B43274913434B608D
S31508011008264B01221A60FDF739FC386108E0FDF71D
S3150801101835FC02463B69D31A022B01D9032337E06B
S315080110281D4B1B6803F00073002BF0D02FE01B4BF8
S3150801103800221A60FDF722FC386108E0FDF71EFC5C
S3150801104802463B69D31A022B01D9032320E0124B26
S315080110581B6803F00073002BF0D118E07B681B6A44
S31508011068012B01D1012313E00B4B5B68FB60FB687D
S3150801107803F480327B685B6A9A4206D1FB6803F4FB
S3150801108870127B689B6A9A4201D0012300E000230B
S3150801109818461837BD4680BD001002406000424216
S315080110A880B584B000AF786039607B68002B01D1C0
S315080110B80123D0E06A4B1B6803F007033A689A4292
S315080110C810D9674B1B6823F0070265493B68134328
S315080110D80B60634B1B6803F007033A689A4201D011
S315080110E80123B8E07B681B6803F00203002B20D0B4
S315080110F87B681B6803F00403002B05D0594B5B6812
S31508011108584A43F4E06353607B681B6803F0080395
S31508011118002B05D0534B5B68524A43F4605353601E
S31508011128504B5B6823F0F0027B689B684D49134373
S315080111384B607B681B6803F00103002B40D07B6872
S315080111485B68012B07D1474B1B6803F40033002B57
S3150801115815D101237FE07B685B68022B07D1414BD8
S315080111681B6803F00073002B09D1012373E03D4B7B
S315080111781B6803F00203002B01D101236BE0394BED
S315080111885B6823F003027B685B68364913434B6047
S31508011198FDF774FBF8600AE0FDF770FB0246FB6889
S315080111A8D31A41F28832934201D9032353E02D4BCE
S315080111B85B6803F00C027B685B689B009A42EBD17B
S315080111C8274B1B6803F007033A689A4210D2244B47
S315080111D81B6823F0070222493B6813430B60204B1F
S315080111E81B6803F007033A689A4201D0012332E0E3
S315080111F87B681B6803F00403002B08D0194B5B684E
S3150801120823F4E0627B68DB68164913434B607B6805
S315080112181B6803F00803002B09D0124B5B6823F4FB
S3150801122860527B681B69DB000E4913434B6000F06B
S3150801123821F802460B4B5B681B0903F00F030A49A1
S31508011248CB5C22FA03F3094A1360094B1B68184653
S31508011258FDF7D2FA002318461037BD4680BD00BFF0
S315080112680020024000100240C06C010878000020E6
S315080112787C0000202DE9B04F8EB000AF0023FB6239
S315080112880023BB6200237B6300237B6200233B6345
S3150801129800233B620023FB614E4B5B68FB62FB6ADA
S315080112A803F00C03042B02D0082B03D089E04A4B20
S315080112B83B6389E0FB6A9B0C03F00F02474B9B5C77
S315080112C87B62FB6A03F48033002B72D0414BDB6ADD
S315080112D803F00F02424B9B5CBB623E4BDB6A03F48D
S315080112E88033002B53D03B4BDB6A1B0903F00F03F2
S315080112F801333B62374BDB6A1B0A03F00F030233E0
S31508011308FB61FB6900229A4693467B6A00223B6188
S315080113187A613B6903FB0BF27B690AFB03F3134406
S315080113283A69AAFB02010B4419462B4B03FB01F246
S31508011338002300FB03F31344274AA0FB02452B4469
S315080113481D463B6A0022BB60FA60BB6A00223B6005
S315080113587A60D7E902010B46D7E900AB524602FB88
S3150801136803F25B4684460CFB03F3134402465146D3
S31508011378A2FB01894B44994642464B4620462946D3
S31508011388F7F784FF02460B4613467B6307E07B6A39
S31508011398114A03FB02F2BB6AB2FBF3F37B630F4BF9
S315080113A85B7B1A467B6A934208D17B6B5B087B6336
S315080113B804E07B6A0B4A02FB03F37B637B6B3B63A3
S315080113C802E0094B3B6300BF3B6B18463837BD46FD
S315080113D8BDE8B08F0010024040787D01D86C01083D
S315080113E8E86C010800093D0000127A0080B400AFD4
S315080113F8024B1B681846BD4680BC7047780000201A
S3150801140880B500AFFFF7F2FF0246054B5B681B0A7A
S3150801141803F007030349CB5C22FA03F3184680BD98
S3150801142800100240D06C010880B500AFFFF7DEFF57
S315080114380246054B5B68DB0A03F007030349CB5CE5
S3150801144822FA03F3184680BD00100240D06C010841
S3150801145880B485B000AF78600A4B1B680A4AA2FBBC
S3150801146803235B0A7A6802FB03F3FB6000BFFB6888
S315080114785A1EFA60002BF9D100BF00BF1437BD46C2
S3150801148880BC704778000020D34D621080B588B0BB
S3150801149800AF786000237B6100233B610023FB6171
S315080114A87B681B6803F00103002B7DD00023FB76BC
S315080114B88B4BDB6903F08053002B0DD1884BDB6915
S315080114C8874A43F08053D361854BDB6903F0805320
S315080114D8FB60FB680123FB76824B1B6803F4807368
S315080114E8002B18D17F4B1B687E4A43F4807313601F
S315080114F8FDF7C4F9786108E0FDF7C0F902467B698A
S31508011508D31A642B01D90323E5E0764B1B6803F448
S315080115188073002BF0D0724B1B6A03F440733B614E
S315080115283B69002B2ED07B685B6803F440733A69E4
S315080115389A4227D06A4B1B6A23F440733B616A4B6C
S3150801154801221A60684B00221A60654A3B691362D0
S315080115583B6903F00103002B14D0FDF78FF9786175
S315080115680AE0FDF78BF902467B69D31A41F28832FC
S31508011578934201D90323AEE0594B1B6A03F00203D0
S31508011588002BEED0564B1B6A23F440727B685B68C6
S31508011598534913430B62FB7E012B05D1504BDB697B
S315080115A84F4A23F08053D3617B681B6803F0020313
S315080115B8002B08D04A4B5B6823F440427B689B683A
S315080115C8474913434B607B681B6803F00403002BE8
S315080115D808D0434BDB6A23F400327B68DB68404951
S315080115E81343CB627B681B6803F00803002B08D0FA
S315080115F83B4BDB6A23F480227B681B693849134312
S31508011608CB62374BDB6A03F40033002B05D1344B25
S31508011618DB6A03F48023002B01D00123FB61FB69F4
S31508011628012B48D12E4B1B6803F08053002B38D168
S315080116382B4B1B6803F08063002B09D0284BDB6A08
S3150801164803F0F0027B689B699A4201D0012342E0C4
S31508011658234BDB6A23F0F0027B689B692049134315
S31508011668CB621F4BDB6A23F470427B685B691C49B2
S315080116781343CB621D4B01221A60FDF7FFF8786107
S3150801168808E0FDF7FBF802467B69D31A642B01D9F2
S31508011698032320E0124B1B6803F00053002BF0D0FC
S315080116A809E00F4BDB6A03F470427B685B699A426F
S315080116B801D001230FE07B681B6803F01003002B98
S315080116C808D0074B5B6823F480027B68DB69044909
S315080116D813434B60002318462037BD4680BD00BF1B
S315080116E80010024000700040400442427000424225
S315080116F880B58AB000AF78600023FB6100237B625E
S315080117080023BB6100237B6100233B610023FB6047
S315080117180023BB6000233B627B68013B0F2B00F269
S315080117281D8101A252F823F0E51801084919010893
S315080117386519010843180108651901086519010899
S315080117486519010895180108651901086519010837
S315080117586519010865190108651901086519010856
S315080117686519010871170108834B5B68BB60824BD1
S315080117781B6803F08073002B00F0F280BB689B0C92
S3150801178803F00F037D4AD35CBB61BB6803F480335E
S31508011798002B3BD0784BDB6A03F00F03784AD35CFE
S315080117A8FB61754BDB6A03F48033002B1CD0724B43
S315080117B8DB6A1B0903F00F030133FB606E4BDB6A17
S315080117C81B0A03F00F0302337B616E4AFB68B2FBFF
S315080117D8F3F37A6903FB02F2FB69B2FBF3F2BB691D
S315080117E802FB03F37B6207E0664AFB69B2FBF3F285
S315080117F8BB6902FB03F37B62604B5B7B1A46BB69D9
S31508011808934208D17B6A5B087B6204E0BB695E4A3E
S3150801181802FB03F37B62584B5B6803F48003B3F559
S31508011828800F02D17B6A3B629AE07B6A5B00574A62
S31508011838A2FB03235B083B6292E04F4BDB6A03F486
S315080118480033002B03D1FFF715FD38628AE04A4BAE
S315080118581B6803F08053002B00F08480464BDB6A33
S315080118681B0903F00F030133FB60434BDB6A1B0BB0
S3150801187803F00F0302333B61424AFB68B2FBF3F3F9
S315080118883A6902FB03F35B003B626BE03A4BDB6A9E
S3150801189803F48023002B03D1FFF7ECFC386263E0DD
S315080118A8354B1B6803F08053002B5DD0324BDB6A3E
S315080118B81B0903F00F030133FB602F4BDB6A1B0B74
S315080118C803F00F0302333B612E4AFB68B2FBF3F3BD
S315080118D83A6902FB03F35B003B6245E0264B1B6A48
S315080118E8BB60BB6803F44073B3F5807F08D1BB6856
S315080118F803F00203002B03D04FF400433B621EE0BA
S31508011908BB6803F44073B3F5007F09D11A4B5B6AC8
S3150801191803F00203002B03D049F640433B620EE06D
S31508011928BB6803F44073B3F5407F1FD1124B1B689C
S3150801193803F40033002B19D0154B3B6216E015E06A
S31508011948FFF772FD02460C4B5B689B0B03F003031A
S3150801195801335B00B2FBF3F33B6208E000BF06E024
S3150801196800BF04E000BF02E000BF00E000BF3B6A19
S3150801197818462837BD4680BD00100240F86C010894
S31508011988086D010840787D0100093D00ABAAAAAA9D
S31508011998F0FA020080B584B000AF78600023FB60D6
S315080119A87B68002B01D101237AE07B685B7CDBB27B
S315080119B8002B05D17B6800221A747868FBF786FC28
S315080119C87B6802225A74786800F070F80346002B7F
S315080119D804D07B6804225A74012361E0786800F010
S315080119E892F80346002B04D07B6804225A74012313
S315080119F856E07B681B685A687B681B6822F00702F1
S31508011A085A607B689B68002B05D0274B1B6B264AB7
S31508011A1823F001031363244BDB6A23F460727B68A2
S31508011A289B6821491343CB627B685B68B3F1FF3F27
S31508011A3803D07B685B68FB600EE00120FFF758FE60
S31508011A48F860FB68002B04D17B6804225A740123C9
S31508011A5826E0FB68013BFB60FB681A0C7B681B6880
S31508011A6802F00F029A607B681B68FA6892B2DA601C
S31508011A78786800F070F80346002B04D07B680422C6
S31508011A885A7401230CE07B680022DA737B68012209
S31508011A985A737B6801229A737B6801225A74002358
S31508011AA818461037BD4680BD006C004080B584B025
S31508011AB800AF78600023FB607B68002B01D1012306
S31508011AC81DE07B681B685A687B681B6822F0080258
S31508011AD85A60FCF7D3FEF86009E0FCF7CFFE024628
S31508011AE8FB68D31AB3F57A7F01D9032307E07B6824
S31508011AF81B685B6803F00803002BEED00023184621
S31508011B081037BD4680BD80B584B000AF7860002324
S31508011B18FB60FCF7B3FEF86009E0FCF7AFFE024686
S31508011B28FB68D31AB3F57A7F01D903230FE07B68DB
S31508011B381B685B6803F02003002BEED07B681B68E3
S31508011B485A687B681B6842F010025A6000231846D7
S31508011B581037BD4680BD80B584B000AF78600023D4
S31508011B68FB607B681B685A687B681B6822F0100251
S31508011B785A60FCF783FEF86009E0FCF77FFE024627
S31508011B88FB68D31AB3F57A7F01D9032307E07B6883
S31508011B981B685B6803F02003002BEED00023184668
S31508011BA81037BD4680BD80B582B000AF78607B68C6
S31508011BB8002B01D1012341E07B6893F83D30DBB264
S31508011BC8002B06D17B68002283F83C207868FCF74D
S31508011BD87FFB7B68022283F83D207B681A687B684D
S31508011BE804331946104600F0B9FA7B68012283F8CE
S31508011BF846207B68012283F83E207B68012283F808
S31508011C083F207B68012283F840207B68012283F8FC
S31508011C1841207B68012283F842207B68012283F8E8
S31508011C2843207B68012283F844207B68012283F8D4
S31508011C3845207B68012283F83D200023184608378A
S31508011C48BD4680BD80B582B000AF78607B68002B41
S31508011C5801D1012341E07B6893F83D30DBB2002BC3
S31508011C6806D17B68002283F83C20786800F039F8A9
S31508011C787B68022283F83D207B681A687B680433EF
S31508011C881946104600F06AFA7B68012283F846204D
S31508011C987B68012283F83E207B68012283F83F206E
S31508011CA87B68012283F840207B68012283F841205A
S31508011CB87B68012283F842207B68012283F8432046
S31508011CC87B68012283F844207B68012283F8452032
S31508011CD87B68012283F83D20002318460837BD464C
S31508011CE880BD80B483B000AF786000BF0C37BD46AD
S31508011CF880BC704780B584B000AF786039603B68AE
S31508011D08002B09D17B6893F83E30DBB2012B14BF4F
S31508011D1801230023DBB222E03B68042B09D17B6847
S31508011D2893F83F30DBB2012B14BF01230023DBB242
S31508011D3815E03B68082B09D17B6893F84030DBB27C
S31508011D48012B14BF01230023DBB208E07B6893F853
S31508011D584130DBB2012B14BF01230023DBB2002B70
S31508011D6801D0012363E03B68002B04D17B6802227A
S31508011D7883F83E2013E03B68042B04D17B680222D2
S31508011D8883F83F200BE03B68082B04D17B680222C5
S31508011D9883F8402003E07B68022283F841207B68A8
S31508011DA81B6801223968184600F06EFC7B681B68B7
S31508011DB8214A934207D17B681B685A6C7B681B6862
S31508011DC842F400425A647B681B681B4A934213D043
S31508011DD87B681B68B3F1804F0ED07B681B68174A6E
S31508011DE8934209D07B681B68154A934204D07B68DD
S31508011DF81B68144A934211D17B681B689B6803F0D8
S31508011E080703FB60FB68062B10D07B681B681A68FA
S31508011E187B681B6842F001021A6007E07B681B6849
S31508011E281A687B681B6842F001021A600023184683
S31508011E381037BD4680BD00BF002C01400004004094
S31508011E4800080040000C004080B586B000AFF86075
S31508011E58B9607A600023FB75FB6893F83C30012B5F
S31508011E6801D10223AEE0FB68012283F83C207B6896
S31508011E780C2B00F29F8001A252F823F0B91E010823
S31508011E88BD1F0108BD1F0108BD1F0108F91E01086C
S31508011E98BD1F0108BD1F0108BD1F01083B1F010819
S31508011EA8BD1F0108BD1F0108BD1F01087B1F0108C9
S31508011EB8FB681B68B968184600F0C8F9FB681B680F
S31508011EC89A69FB681B6842F008029A61FB681B68F5
S31508011ED89A69FB681B6822F004029A61FB681B6809
S31508011EE89969BB681A69FB681B680A439A6164E0C1
S31508011EF8FB681B68B968184600F00EFAFB681B6888
S31508011F089A69FB681B6842F400629A61FB681B6858
S31508011F189A69FB681B6822F480629A61FB681B68E8
S31508011F289969BB681B691A02FB681B680A439A61A7
S31508011F3843E0FB681B68B968184600F057FAFB685E
S31508011F481B68DA69FB681B6842F00802DA61FB68F4
S31508011F581B68DA69FB681B6822F00402DA61FB6808
S31508011F681B68D969BB681A69FB681B680A43DA6181
S31508011F7823E0FB681B68B968184600F0A1FAFB68F4
S31508011F881B68DA69FB681B6842F40062DA61FB6858
S31508011F981B68DA69FB681B6822F48062DA61FB68E8
S31508011FA81B68D969BB681B691A02FB681B680A435F
S31508011FB8DA6102E00123FB7500BFFB68002283F89A
S31508011FC83C20FB7D18461837BD4680BD80B584B0D0
S31508011FD800AF786039600023FB737B6893F83C305F
S31508011FE8012B01D10223B4E07B68012283F83C2046
S31508011FF87B68022283F83D207B681B689B68BB6067
S31508012008BB6823F07703BB60BB6823F47F43BB60D7
S315080120187B681B68BA689A603B681B68B3F5005FFA
S315080120283ED0B3F5005F00F28780B3F5805F00F014
S315080120388680B3F5805F7FD8702B1AD0702B7BD832
S31508012048602B50D0602B77D8502B3CD0502B73D8A7
S31508012058402B58D0402B6FD8302B64D0302B6BD8F7
S31508012068202B60D0202B67D8002B5CD0102B5AD098
S3150801207862E07B6818683B6899683B685A683B68F8
S31508012088DB6800F0E2FA7B681B689B68BB60BB6883
S3150801209843F07703BB607B681B68BA689A604FE0B0
S315080120A87B6818683B6899683B685A683B68DB68C7
S315080120B800F0CBFA7B681B689A687B681B6842F450
S315080120C880429A603CE07B6818683B6859683B68B7
S315080120D8DB681A4600F042FA7B681B6850211846E5
S315080120E800F099FA2CE07B6818683B6859683B68E0
S315080120F8DB681A4600F060FA7B681B686021184697
S3150801210800F089FA1CE07B6818683B6859683B68DF
S31508012118DB681A4600F022FA7B681B6840211846D4
S3150801212800F079FA0CE07B681A683B681B6819465F
S31508012138104600F070FA03E00123FB7300E000BFC4
S315080121487B68012283F83D207B68002283F83C20BE
S31508012158FB7B18461037BD4680BD000080B485B0A4
S3150801216800AF786039607B681B68FB607B68334A17
S3150801217893420FD07B68B3F1804F0BD07B68304A06
S31508012188934207D07B682F4A934203D07B682E4A2D
S31508012198934208D1FB6823F07003FB603B685B68D0
S315080121A8FA681343FB607B68244A93420FD07B681D
S315080121B8B3F1804F0BD07B68214A934207D07B68DD
S315080121C8204A934203D07B681F4A934208D1FB6889
S315080121D823F44073FB603B68DB68FA681343FB60CA
S315080121E8FB6823F080023B685B691343FB607B68E5
S315080121F8FA681A603B689A687B68DA623B681A6803
S315080122087B689A627B680D4A934203D13B681A69CF
S315080122187B681A637B6801225A617B681B6903F02C
S315080122280103002B05D07B681B6923F001027B6833
S315080122381A6100BF1437BD4680BC7047002C01409F
S315080122480004004000080040000C004080B487B034
S3150801225800AF786039607B681B6A7B617B681B6A9B
S3150801226823F001027B681A627B685B683B617B68BD
S315080122789B69FB60FB6823F07003FB60FB6823F02E
S315080122880303FB603B681B68FA681343FB607B69B9
S3150801229823F002037B613B689B687A6913437B6178
S315080122A87B681C4A93420CD17B6923F008037B613E
S315080122B83B68DB687A6913437B617B6923F004030E
S315080122C87B617B68134A934211D13B6923F4807376
S315080122D83B613B6923F400733B613B685B693A6977
S315080122E813433B613B689B693A6913433B617B68C6
S315080122F83A695A607B68FA689A613B685A687B68E2
S315080123085A637B687A691A6200BF1C37BD4680BC66
S31508012318704700BF002C014080B487B000AF7860D1
S3150801232839607B681B6A7B617B681B6A23F010022C
S315080123387B681A627B685B683B617B689B69FB60A3
S31508012348FB6823F4E043FB60FB6823F44073FB60F6
S315080123583B681B681B02FA681343FB607B6923F019
S3150801236820037B613B689B681B017A6913437B6180
S315080123787B681D4A93420DD17B6923F080037B61F3
S315080123883B68DB681B017A6913437B617B6923F028
S3150801239840037B617B68144A934213D13B6923F452
S315080123A880633B613B6923F400633B613B685B6976
S315080123B89B003A6913433B613B689B699B003A69F1
S315080123C813433B617B683A695A607B68FA689A6184
S315080123D83B685A687B689A637B687A691A6200BFA0
S315080123E81C37BD4680BC7047002C014080B487B0B5
S315080123F800AF786039607B681B6A7B617B681B6AFA
S3150801240823F480727B681A627B685B683B617B6828
S31508012418DB69FB60FB6823F07003FB60FB6823F04C
S315080124280303FB603B681B68FA681343FB607B6917
S3150801243823F400737B613B689B681B027A69134323
S315080124487B617B681D4A93420DD17B6923F400633E
S315080124587B613B68DB681B027A6913437B617B698D
S3150801246823F480637B617B68144A934213D13B69E1
S3150801247823F480533B613B6923F400533B613B6872
S315080124885B691B013A6913433B613B689B691B01FD
S315080124983A6913433B617B683A695A607B68FA680B
S315080124A8DA613B685A687B68DA637B687A691A6213
S315080124B800BF1C37BD4680BC704700BF002C0140D1
S315080124C880B487B000AF786039607B681B6A3B6166
S315080124D87B681B6A23F480527B681A627B685B688F
S315080124E87B617B68DB69FB60FB6823F4E043FB607F
S315080124F8FB6823F44073FB603B681B681B02FA6898
S315080125081343FB603B6923F400533B613B689B68B3
S315080125181B033A6913433B617B680F4A934209D106
S315080125287B6923F480437B613B685B699B017A6914
S3150801253813437B617B687A695A607B68FA68DA6152
S315080125483B685A687B681A647B683A691A6200BFED
S315080125581C37BD4680BC7047002C014080B487B043
S3150801256800AFF860B9607A60FB681B6A7B61FB6833
S315080125781B6A23F00102FB681A62FB689B693B61C7
S315080125883B6923F0F0033B617B681B013A691343F6
S315080125983B617B6923F00A037B617A69BB6813434C
S315080125A87B61FB683A699A61FB687A691A6200BFB6
S315080125B81C37BD4680BC704780B487B000AFF86049
S315080125C8B9607A60FB681B6A7B61FB681B6A23F042
S315080125D81002FB681A62FB689B693B613B6923F435
S315080125E870433B617B681B033A6913433B617B690B
S315080125F823F0A0037B61BB681B017A6913437B61DE
S31508012608FB683A699A61FB687A691A6200BF1C37DE
S31508012618BD4680BC704780B485B000AF7860396024
S315080126287B689B68FB60FB6823F07003FB603A686C
S31508012638FB68134343F00703FB607B68FA689A60F3
S3150801264800BF1437BD4680BC704780B487B000AF59
S31508012658F860B9607A603B60FB689B687B617B6957
S3150801266823F47F437B613B681A027B681A43BB687C
S3150801267813437A6913437B61FB687A699A6000BFD9
S315080126881C37BD4680BC704780B487B000AFF86078
S31508012698B9607A60BB6803F01F03012202FA03F3E3
S315080126A87B61FB681A6A7B69DB431A40FB681A6215
S315080126B8FB681A6ABB6803F01F03796801FA03F312
S315080126C81A43FB681A6200BF1C37BD4680BC7047AF
S315080126D880B485B000AF786039607B6893F83C3080
S315080126E8012B01D102234BE07B68012283F83C20A8
S315080126F87B68022283F83D207B681B685B68FB6060
S315080127087B681B689B68BB60FB6823F07003FB60EA
S315080127183B681B68FA681343FB607B681B68FA68A1
S315080127285A607B681B68194A934213D07B681B68F1
S31508012738B3F1804F0ED07B681B68154A934209D0BE
S315080127487B681B68134A934204D07B681B68124A44
S3150801275893420CD1BB6823F08003BB603B685B6876
S31508012768BA681343BB607B681B68BA689A607B685A
S31508012778012283F83D207B68002283F83C20002348
S3150801278818461437BD4680BC704700BF002C014067
S315080127980004004000080040000C004080B582B0E3
S315080127A800AF78607B68002B01D1012342E07B6882
S315080127B893F84130DBB2002B06D17B68002283F8F7
S315080127C840207868FBF78EFE7B68242283F841202F
S315080127D87B681B68DA687B681B6822F40052DA6032
S315080127E8786800F0B3FE7B681B681A697B681B6802
S315080127F822F490421A617B681B685A697B681B68D0
S3150801280822F02A025A617B681B68DA687B681B68AA
S3150801281842F40052DA607B6800225A647B682022F7
S3150801282883F841207B68202283F842207B680022AE
S315080128385A63002318460837BD4680BD80B485B05B
S3150801284800AFF860B9601346FB80FB6893F841301E
S31508012858DBB2202B21D1BB68002B02D0FB88002BC9
S3150801286801D101231AE0FB68BA681A62FB68FA887B
S315080128789A84FB68FA88DA84FB6800225A64FB683A
S31508012888212283F84120FB681B68DA68FB681B6804
S3150801289842F08002DA60002300E002231846143762
S315080128A8BD4680BC704780B58CB000AFF860B9608A
S315080128B81346FB80FB6893F84230DBB2202B4AD1DA
S315080128C8BB68002B02D0FB88002B01D1012343E00A
S315080128D8FB6801221A63FB6800225A63FB881A46B9
S315080128E8B968F86800F0FDFB034687F82F3097F8B2
S315080128F82F30002B2CD1FB681B6B012B25D100230C
S315080129083B61FB681B681B683B61FB681B685B6866
S315080129183B613B69FB681B680C33BB61BB6953E8C0
S31508012928003F7B617B6943F01003BB62FB681B6848
S315080129380C33BA6A7A623B62396A7A6A41E80023D1
S31508012948FB61FB69002BE5D102E0012387F82F30EB
S3150801295897F82F3000E0022318463037BD4680BD68
S3150801296880B5A2B000AF78600123C7F884307B68C8
S315080129781B680C333B663B6E53E8003FFB65FB6DF2
S3150801298823F4F073C7F880307B681B680C33D7F8D3
S315080129988020FA66BB66B96EFA6E41E800237B6643
S315080129A87B6E002BE3D17B681B681433FB64FB6CD5
S315080129B853E8003FBB64BB6C23F00103FB677B68E4
S315080129C81B681433FA6FBA657B65796DBA6D41E888
S315080129D800233B653B6D002BE5D17B681B6B012BFF
S315080129E819D17B681B680C33BB63BB6B53E8003F83
S315080129F87B637B6B23F01003BB677B681B680C330F
S31508012A08BA6F7A643B64396C7A6C41E80023FB63D4
S31508012A18FB6B002BE5D17B689B6B002B0FD07B6882
S31508012A281B685B6903F08003002B04D07B689B6BEA
S31508012A38534A5A6303E07B689B6B00225A637B6897
S31508012A48DB6B002B0FD07B681B685B6903F04003BF
S31508012A58002B04D07B68DB6B4A4A5A6303E07B6820
S31508012A68DB6B00225A637B681B685B6903F080038A
S31508012A78002B2DD07B681B6814337B627B6A53E86D
S31508012A88003F3B623B6A23F080037B677B681B68D0
S31508012A9814337A6F3A63FB62F96A3A6B41E80023A1
S31508012AA8BB62BB6A002BE5D17B689B6B002B0FD0F9
S31508012AB87B689B6B1846FDF745FC0346002B04D03B
S31508012AC87B689B6B00225A6302E00023C7F88430AF
S31508012AD87B681B685B6903F04003002B30D07B6871
S31508012AE81B6814333B613B6953E8003FFB60FB688D
S31508012AF823F040033B677B681B6814333A6FFA6116
S31508012B08BB61B969FA6941E800237B617B69002BD6
S31508012B18E5D17B68DB6B002B12D07B68DB6B18462B
S31508012B28FDF710FC0346002B07D07B68DB6B0022F8
S31508012B385A630123C7F8843002E00023C7F88430B2
S31508012B48D7F88430012B16D17B680022DA847B6892
S31508012B580022DA857B6800225A647B68202283F87A
S31508012B6841207B68202283F842207B6800221A6369
S31508012B78786800F0ADFA002318468837BD4680BD47
S31508012B8849320108A932010880B5BAB000AF7860A0
S31508012B987B681B681B68C7F8E4307B681B68DB68B9
S31508012BA8C7F8E0307B681B685B69C7F8DC30002327
S31508012BB8C7F8D8300023C7F8D430D7F8E43003F07B
S31508012BC80F03C7F8D830D7F8D830002B0FD1D7F864
S31508012BD8E43003F02003002B09D0D7F8E03003F0DE
S31508012BE82003002B03D0786800F0F1FB5BE2D7F8E5
S31508012BF8D830002B00F0DE80D7F8DC3003F001036B
S31508012C08002B06D1D7F8E03003F49073002B00F0B7
S31508012C18D180D7F8E43003F00103002B0BD0D7F89D
S31508012C28E03003F48073002B05D07B685B6C43F0B6
S31508012C3801027B685A64D7F8E43003F00403002BD1
S31508012C480BD0D7F8DC3003F00103002B05D07B68DD
S31508012C585B6C43F002027B685A64D7F8E43003F0E8
S31508012C680203002B0BD0D7F8DC3003F00103002B45
S31508012C7805D07B685B6C43F004027B685A64D7F815
S31508012C88E43003F00803002B11D0D7F8E03003F03D
S31508012C982003002B05D1D7F8DC3003F00103002BFC
S31508012CA805D07B685B6C43F008027B685A647B68CD
S31508012CB85B6C002B00F0F281D7F8E43003F02003AF
S31508012CC8002B08D0D7F8E03003F02003002B02D0F8
S31508012CD8786800F07CFB7B681B685B6903F0400336
S31508012CE8002B14BF01230023DBB2C7F8D4307B6855
S31508012CF85B6C03F00803002B03D1D7F8D430002BFB
S31508012D084FD0786800F026FA7B681B685B6903F080
S31508012D184003002B41D07B681B681433C7F89C30E5
S31508012D28D7F89C3053E8003FC7F89830D7F8983059
S31508012D3823F04003C7F8D0307B681B681433D7F8EB
S31508012D48D020C7F8A820C7F8A430D7F8A410D7F810
S31508012D58A82041E80023C7F8A030D7F8A030002BEF
S31508012D68D9D17B68DB6B002B13D07B68DB6B7E4A7A
S31508012D785A637B68DB6B1846FDF7E4FA0346002BB2
S31508012D8816D07B68DB6B5B6B7A68D26B1046984703
S31508012D980EE0786800F093F90AE0786800F08FF990
S31508012DA806E0786800F08BF97B6800225A6475E1B9
S31508012DB800BF73E17B681B6B012B40F04F81D7F885
S31508012DC8E43003F01003002B00F04881D7F8E0300F
S31508012DD803F01003002B00F041810023BB607B68D8
S31508012DE81B681B68BB607B681B685B68BB60BB6844
S31508012DF87B681B685B6903F04003002B00F0B6800B
S31508012E087B68DB6B1B685B68A7F8BE30B7F8BE3012
S31508012E18002B00F045817B689B8DB7F8BE209A4246
S31508012E2880F03E817B68B7F8BE20DA857B68DB6B64
S31508012E389B69202B00F088807B681B680C33C7F8D0
S31508012E488830D7F8883053E8003FC7F88430D7F870
S31508012E58843023F48073C7F8B8307B681B680C3351
S31508012E68D7F8B820C7F89420C7F89030D7F8901043
S31508012E78D7F8942041E80023C7F88C30D7F88C3066
S31508012E88002BD9D17B681B6814337B677B6F53E8A2
S31508012E98003F3B673B6F23F00103C7F8B4307B68F3
S31508012EA81B681433D7F8B420C7F88020FB67F96F75
S31508012EB8D7F8802041E80023BB67BB6F002BE1D117
S31508012EC87B681B6814333B663B6E53E8003FFB651A
S31508012ED8FB6D23F04003C7F8B0307B681B681433D1
S31508012EE8D7F8B020FA66BB66B96EFA6E41E80023D0
S31508012EF87B667B6E002BE3D17B68202283F8422010
S31508012F087B6800221A637B681B680C33FB64FB6CBD
S31508012F1853E8003FBB64BB6C23F01003C7F8AC3019
S31508012F287B681B680C33D7F8AC20BA657B65796D65
S31508012F38BA6D41E800233B653B6D002BE3D17B68FD
S31508012F48DB6B1846FDF7C3F97B6802225A637B686F
S31508012F589A8D7B68DB8D9BB2D31A9BB21946786822
S31508012F68FAF776FA9CE000BF213201087B689A8D48
S31508012F787B68DB8D9BB2D31AA7F8CE307B68DB8DCD
S31508012F889BB2002B00F08E80B7F8CE30002B00F0EC
S31508012F9889807B681B680C33BB63BB6B53E8003FAE
S31508012FA87B637B6B23F49073C7F8C8307B681B680F
S31508012FB80C33D7F8C8207A643B64396C7A6C41E8D3
S31508012FC80023FB63FB6B002BE3D17B681B68143377
S31508012FD87B627B6A53E8003F3B623B6A23F0010345
S31508012FE8C7F8C4307B681B681433D7F8C4203A631A
S31508012FF8FB62F96A3A6B41E80023BB62BB6A002B9C
S31508013008E3D17B68202283F842207B6800221A6371
S315080130187B681B680C333B613B6953E8003FFB60DF
S31508013028FB6823F01003C7F8C0307B681B680C33AC
S31508013038D7F8C020FA61BB61B969FA6941E8002382
S315080130487B617B69002BE3D17B6802225A63B7F857
S31508013058CE3019467868FAF7FBF923E0D7F8E43051
S3150801306803F08003002B09D0D7F8E03003F080037A
S31508013078002B03D0786800F043F914E0D7F8E43058
S3150801308803F04003002B0ED0D7F8E03003F04003D5
S31508013098002B08D0786800F082F904E000BF02E046
S315080130A800BF00E000BFE837BD4680BD80B483B0E5
S315080130B800AF786000BF0C37BD4680BC704780B446
S315080130C883B000AF786000BF0C37BD4680BC704737
S315080130D880B483B000AF786000BF0C37BD4680BCAA
S315080130E8704780B485B000AFF860B9601346FB80B5
S315080130F8FB68BA689A62FB68FA889A85FB68FA884F
S31508013108DA85FB6800225A64FB68222283F8422082
S31508013118FB681B69002B07D0FB681B68DA68FB6824
S315080131281B6842F48072DA60FB681B685A69FB6897
S315080131381B6842F001025A61FB681B68DA68FB687A
S315080131481B6842F02002DA60002318461437BD4688
S3150801315880BC704780B495B000AF78607B681B68FF
S315080131680C337B637B6B53E8003F3B633B6B23F470
S315080131789073FB647B681B680C33FA6C3A64FB63CF
S31508013188F96B3A6C41E80023BB63BB6B002BE5D1AD
S315080131987B681B6814333B623B6A53E8003FFB6153
S315080131A8FB6923F00103BB647B681B681433BA6C9B
S315080131B8FA62BB62B96AFA6A41E800237B627B6AEA
S315080131C8002BE5D17B681B6B012B19D17B681B6822
S315080131D80C33FB60FB6853E8003FBB60BB6823F010
S315080131E810037B647B681B680C337A6CBA617B6154
S315080131F87969BA6941E800233B613B69002BE5D146
S315080132087B68202283F842207B6800221A6300BF64
S315080132185437BD4680BC704780B584B000AF786026
S315080132287B685B6AFB60FB680022DA85FB6800221B
S31508013238DA84F868FFF743FF00BF1037BD4680BD3B
S3150801324880B584B000AF78607B685B6AFB60FB6811
S315080132589B6B00225A63FB68DB6B002B04D0FB6867
S31508013268DB6B5B6B002B17D1FB680022DA84FB68E2
S315080132780022DA85FB6800225A64FB68202283F853
S315080132884120FB68202283F84220FB6800221A6342
S31508013298F868FFF71DFF00E000BF1037BD4680BD7F
S315080132A880B584B000AF78607B685B6AFB60FB68B1
S315080132B8DB6B00225A63FB689B6B002B04D0FB6807
S315080132C89B6B5B6B002B17D1FB680022DA84FB68C2
S315080132D80022DA85FB6800225A64FB68202283F8F3
S315080132E84120FB68202283F84220FB6800221A63E2
S315080132F8F868FFF7EDFE00E000BF1037BD4680BD50
S3150801330880B485B000AF78607B6893F84130DBB24A
S31508013318212B3ED17B689B68B3F5805F14D17B6806
S315080133281B69002B10D17B681B6AFB60FB681B882D
S315080133381A467B681B68C2F308025A607B681B6ACF
S315080133489A1C7B681A6208E07B681B6A591C7A68AA
S3150801335811621A787B681B685A607B68DB8C9BB29A
S31508013368013B9BB27A681946D184002B0FD17B6839
S315080133781B68DA687B681B6822F08002DA607B685A
S315080133881B68DA687B681B6842F04002DA6000232A
S3150801339800E0022318461437BD4680BC704780B53D
S315080133A882B000AF78607B681B68DA687B681B683F
S315080133B822F04002DA607B68202283F84120786887
S315080133C8FAF798F8002318460837BD4680BD80B530
S315080133D88CB000AF78607B6893F84230DBB2222B59
S315080133E840F0AE807B689B68B3F5805F17D17B6830
S315080133F81B69002B13D10023FB627B689B6ABB629E
S315080134087B681B685B689BB2C3F308039AB2BB6AFD
S315080134181A807B689B6A9A1C7B689A6226E07B6895
S315080134289B6AFB620023BB627B689B68B3F5805F76
S3150801343807D07B689B68002B0AD17B681B69002B20
S3150801344806D17B681B685B68DAB2FB6A1A7008E002
S315080134587B681B685B68DBB203F07F03DAB2FB6A39
S315080134681A707B689B6A5A1C7B689A627B68DB8D33
S315080134789BB2013B9BB27A681946D185002B5DD16F
S315080134887B681B68DA687B681B6822F02002DA60A9
S315080134987B681B68DA687B681B6822F48072DA60C5
S315080134A87B681B685A697B681B6822F001025A61A6
S315080134B87B68202283F842207B6800225A637B684E
S315080134C81B6B012B35D17B6800221A637B681B6845
S315080134D80C337B617B6953E8003F3B613B6923F009
S315080134E810037B627B681B680C337A6A3A62FB6154
S315080134F8F9693A6A41E80023BB61BB69002BE5D142
S315080135087B681B681B6803F01003102B0AD100237C
S31508013518FB607B681B681B68FB607B681B685B68CC
S31508013528FB60FB687B689B8D19467868F9F790FFFD
S3150801353802E07868FFF7BAFD002302E0002300E0FD
S31508013548022318463037BD4680BD000080B584B0D1
S3150801355800AF78607B681B681B6923F440517B6858
S31508013568DA687B681B680A431A617B689A687B680C
S315080135781B691A437B685B691343BB607B681B68D5
S31508013588DB6823F4B05323F00C037A681268B96828
S315080135980B43D3607B681B685B6923F440717B68BE
S315080135A89A697B681B680A435A617B681B682C4AB7
S315080135B8934203D1FDF738FFF86002E0FDF720FFD3
S315080135C8F860FA6813469B0013449A001A447B6804
S315080135D85B689B00B2FBF3F3224AA2FB03235B0950
S315080135E81901FA6813469B0013449A001A447B6822
S315080135F85B689B00B2FBF3F21A4BA3FB02035B0958
S31508013608642000FB03F3D31A1B013233154AA2FBC4
S3150801361803235B0903F0F0031944FA6813469B0070
S3150801362813449A001A447B685B689B00B2FBF3F261
S315080136380C4BA3FB02035B09642000FB03F3D31AB3
S315080136481B013233074AA2FB03235B0903F00F0266
S315080136587B681B680A449A6000BF1037BD4680BD5F
S31508013668003801401F85EB51002B2DE9F0471D460F
S31508013678BBBF03F100431D4600232D2388B014461A
S31508013688B8BF1446129A109E1370149BDDF84CA005
S3150801369823F02008B8F1460F05D0B8F1450F00D137
S315080136A80136022300E0032307AA049206AACDE9F4
S315080136B802A2CDE9003622462B4600F001FFB8F1F1
S315080136C8470F074619D1119BDB070ED500EB0609EB
S315080136D80022002320462946F5F7CEF908B1CDF888
S315080136E81C903022079B4B451ED33846079B159AD3
S315080136F8DB1B136008B0BDE8F087B8F1460F00EB8D
S315080137080609E5D10378302B0AD100220023204681
S315080137182946F5F7B1F918B9C6F10106CAF80060DC
S31508013728DAF800309944D3E7591C07911A70D9E792
S31508013738F7B50029B6BF2D232B234942092902705B
S31508013748437029DD0DF107031D460A27B1FBF7F674
S315080137581A4607FB1614303402F8014C0C46632C3A
S31508013768314603F1FF33F1DC3031941E03F8011CAD
S315080137782346411CAB420AD30DF109039B1AAC42F5
S3150801378888BF002302330344181A03B0F0BD13F89F
S31508013798016B01F8016FEDE7302330318370C17091
S315080137A8031DF1E72DE9F04F91B00C46DDF8688065
S315080137B816461F46054600F0BDFD036818460893D8
S315080137C8F4F72EFD00230E93D8F800300990073335
S315080137D823F0070303F1080294F818A0D4F800B0F7
S315080137E8C8F80020D3E9008929F000430B93CDF8DE
S315080137F828804FF0FF32DDE90A01C4E912899C4B9A
S31508013808F5F76CF970BBDDE90A014FF0FF32984B01
S31508013818F5F746F930BB0022002340464946F5F735
S3150801382835F910B12D2384F84330924A924BBAF1EF
S31508013838470F8CBF9046984603234FF0000923612A
S315080138482BF00403236033462146284600970FAA1E
S3150801385800F0D4F9013040F090804FF0FF3011B0F4
S31508013868BDE8F08F42464B4640464946F5F736F9D4
S3150801387848B14B46002BB8BF2D23804AB8BF84F8F8
S3150801388843307F4BD3E763680AF0DF015A1C3FD1FF
S315080138980623636000224BF48063236006920EAA0E
S315080138A8CDE904A20DAA03920DF13302CDE901323D
S315080138B863684246009328464B460A91FFF7D4FEA9
S315080138C80A99804647290D9928D1C81C02DB6368DD
S315080138D8994240DDAAF1020A5FFA8AFA5246013983
S315080138E804F150000D91FFF723FF0E9A814613182C
S315080138F8012A236102DC2268D20701D50133236133
S315080139089DF83330002B9ED02D2384F843309AE74F
S315080139184729BFD1002BBDD10123BAE7BAF1650FF3
S31508013928DCD9BAF1660F18D1002963680BDD216164
S3150801393813B92268D00702D501330B4423614FF026
S315080139480009A165DCE713B92268D20701D5023354
S31508013958F4E70123F2E74FF0670A0E9B994205DB64
S3150801396823682161D807EAD54B1CE7E70029CCBFAC
S315080139780122C1F102021344E0E723685A0507D474
S315080139882369424631462846B84701302BD164E7B0
S31508013998BAF1650F40F2DC80D4E91201002200234E
S315080139A8F5F76AF8002833D0012331462846354AFF
S315080139B8B84701303FF451AFDDE90D38434502DB1D
S315080139C82368D8070FD5DDE9082331462846B847BD
S315080139D801303FF442AF4FF0000908F1FF3804F10E
S315080139E81A0AC84509DC23689B0700F10281E068C1
S315080139F80F9B9842B8BF184631E70123524631460C
S31508013A082846B84701303FF428AF09F10109E8E724
S31508013A180D9B002B38DC012331462846194AB8473D
S31508013A2801303FF41AAFDDE90D3959EA030302D12A
S31508013A382368D907D7D5DDE9082331462846B84783
S31508013A4801303FF40AAF4FF0000A04F11A0B0D9B37
S31508013A585B42534501DC4B4693E701235A463146F7
S31508013A682846B84701303FF4F8AE0AF1010AEEE7ED
S31508013A78FFFFEF7F1C6D0108186D0108246D010809
S31508013A88206D0108286D0108A36DDDF838A0534596
S31508013A98A8BF5346002B994636DC4FF0000B29EA96
S31508013AA8E97904F11A02A36D0A93A3EB09035B45A5
S31508013AB831DC0D9B9A453ADC2368DA0737D40D9B26
S31508013AC8AAEB03090A9BAAEB03039945A8BF9946DA
S31508013AD8B9F1000F33DC4FF0000829EAE97904F156
S31508013AE81A0B0D9BAAEB0303A3EB090343457FF7BF
S31508013AF87AAF01235A4631462846B84701303FF47A
S31508013B08ACAE08F10108ECE7424631462846B84703
S31508013B180130C2D1A1E60123314628460A92B8479F
S31508013B2801303FF49AAE0A9A0BF1010BBBE731460D
S31508013B38DDE908232846B8470130C0D18DE60A9A37
S31508013B484B46314628464244B8470130C3D184E634
S31508013B58DDF838A0BAF1010F01DCDB0736D50123F8
S31508013B68424631462846B84701303FF476AEDDE984
S31508013B78082331462846B84701303FF46EAED4E9E2
S31508013B881201002200230AF1FF3AF4F775FFC0B9BA
S31508013B98534608F1010231462846B84701300CD187
S31508013BA85BE601235A4631462846B84701303FF4B1
S31508013BB854AE08F10108D045F3DB4B4604F150022F
S31508013BC8E0E64FF0000804F11A0BF4E70123424630
S31508013BD8E1E701234A4631462846B84701303FF40A
S31508013BE83CAE08F10108E3680F995B1A4345F0DC16
S31508013BF8FDE64FF0000804F11909F4E72DE9F04745
S31508013C08164698468A680B6907469342B8BF13460B
S31508013C18336091F843200C46DDF820900AB1013348
S31508013C2833602368990642BF3368023333602568CF
S31508013C3815F0060506D104F1190AE36832689B1AD4
S31508013C48AB422BDC94F843302268003B18BF0123AA
S31508013C58920630D44146384604F14302C847013032
S31508013C6823D02368226903F00603042B14BF002511
S31508013C7833684FF0000608BFE56804F11A0408BF5F
S31508013C88ED1A54F8123C08BF25EAE5759342C4BFF4
S31508013C989B1AED18B5421AD1002008E001235246AD
S31508013CA841463846C847013003D14FF0FF30BDE8D1
S31508013CB8F0870135C1E73020E11881F843005A1C1D
S31508013CC894F845102244023382F84310C2E70123C7
S31508013CD8224641463846C8470130E6D00136D9E773
S31508013CE82DE9FF470F7E9146782F80460C469A465E
S31508013CF80C9E01F1430207D8622F0AD8002F00F05B
S31508013D08D180582F00F0B88004F1420684F8427031
S31508013D183AE0A7F16303152BF6D801A151F823F068
S31508013D28813D0108953D0108113D0108113D01082C
S31508013D38113D0108113D0108953D0108113D01088C
S31508013D48113D0108113D0108113D0108933E01087D
S31508013D58BF3D01084D3E0108113D0108113D010805
S31508013D68B53E0108113D0108BF3D0108113D01088D
S31508013D78113D0108553E010833681A1D1B68326052
S31508013D8804F1420684F8423001239CE0336820682E
S31508013D98191D3160060601D51D6803E04506FBD5E0
S31508013DA8B3F90050002D03DA2D236D4284F8433008
S31508013DB80A23584811E021683368080653F8045B52
S31508013DC802D4490648BFADB26F2F336014BF0A2320
S31508013DD808235048002184F843106668002EA66017
S31508013DE805DB21682E4321F0040121604BD01646D4
S31508013DF8B5FBF3F103FB1157C75D06F8017D2F469D
S31508013E08BB420D46F4D9082B0BD12368DF0708D521
S31508013E18236961689942DEBF302306F8013C06F139
S31508013E28FF36921B22614B4621464046CDF800A033
S31508013E3803AAFFF7E3FE01304AD14FF0FF3004B079
S31508013E48BDE8F087236843F02003236078273248C2
S31508013E5884F84570236831681F0651F8045B02D453
S31508013E685F0648BFADB23160D90744BF43F02003A6
S31508013E7823601DB11023ADE72648E9E7236823F037
S31508013E8820032360F6E71646BDE733682568181D3B
S31508013E98616930602E061B6801D5196002E068065B
S31508013EA8FBD51980002316462361BCE73368002130
S31508013EB81A1D32601E686268304600F03FFA08B17A
S31508013EC8801B606063682361002384F84330AAE78E
S31508013ED83246494640462369D0470130ADD0236862
S31508013EE89B0713D4E068039B9842B8BF1846A6E710
S31508013EF80123324649464046D04701309DD001350F
S31508013F08E36803995B1AAB42F2DCEBE7002504F197
S31508013F181906F5E72A6D01083B6D0108002310B556
S31508013F280446C0E90033C0E90433836081814366E6
S31508013F38C2818361194608225C3000F0FFF80D4BEF
S31508013F48246263620C4BA3620C4BE3620C4B23633A
S31508013F580C4B9C4206D003F16802944202D0D03336
S31508013F689C4205D104F15800BDE8104000F0DEB9BD
S31508013F7810BD00BF515F0108735F0108AB5F0108F7
S31508013F88CF5F010888100020024A0349034800F058
S31508013F98A5B800BF84000020F55701089400002041
S31508013FA841680C4B10B59942044601D001F01EFC34
S31508013FB8A168094B994202D0204601F017FCE1682D
S31508013FC8064B994204D02046BDE8104001F00EBCC4
S31508013FD810BD00BF88100020F010002058110020DD
S31508013FE810B50B4B0B4C0C4A20461A6004210022CB
S31508013FF8FFF794FF04F1680001220921FFF78EFFF4
S3150801400804F1D0000222BDE810401221FFF786BF4D
S31508014018C011002088100020913F0108014800F0CE
S3150801402886B900BFC5110020014800F081B900BF53
S31508014038C511002010B50446FFF7F0FF236A1BB126
S31508014048BDE81040FFF7F0BF044B2362044B1B6819
S31508014058002BF5D1FFF7C4FFF2E700BFA93F010816
S31508014068C011002030B51446002C05461A469BB0E7
S3150801407805DA8B2303604FF0FF301BB030BD4FF4D0
S315080140880273ADF80C304FF0000319930CBF2346A1
S3150801409804F1FF33029305934FF6FF7300910491D8
S315080140A8ADF80E3069461E9B01F03AF8431CBCBFB1
S315080140B88B232B60002CE0D00022009B1A70DCE7CA
S315080140C807B5009313460A46014603480068FFF7F1
S315080140D8C9FF03B05DF804FB900000202DE9F843F9
S315080140E80746884614460026D4E90195B9F1010917
S315080140F805D52468002CF7D13046BDE8F883AB8985
S31508014108012B07D9B5F90E30013303D029463846AC
S31508014118C04706436835E9E70FB407B5064904AB4E
S31508014128086853F8042B8168019301F01DF903B057
S315080141385DF804EB04B0704790000020034602447A
S31508014148934200D1704703F8011BF9E738B50B4BC1
S3150801415804461D686B6B53B9242001F01DFA024603
S31508014168686320B93D21064B064800F003F9204645
S31508014178696BBDE8384000F007B800BF9000002019
S315080141884C6D0108636D01082DE9F04100230C46C1
S31508014198D0E900014C4AF5F729F84FF46161002A7C
S315080141A8BCBF02F5A83202F5C072B2FBF1F301FBF6
S315080141B813224FF03C01A360B2FBF1F301FB132272
S315080141C822604FF0070200F52F20ACBF00F66C20DD
S315080141D800F66B206360C31C93FBF2F2C2EBC202C2
S315080141E89B1A3A4955D50733A361A0F50E33A3F5AA
S315080141F82C7393FBF1F1364B40F2B45C03FB0100D7
S3150801420848F6AC63B0FBF3F3B0FBFCF203449B1A24
S31508014218304A40F26D17B0FBF2F29B1AB3FBF7F27C
S315080142286426B3FBFCF3B2FBF6F5EB1A03449920B3
S3150801423807FB123303EB83070237B7FBF0FC4FF092
S31508014248050800FB0CF00230B0FBF8F003F1010E8B
S31508014258AEEB000040F2F95E77458CBF6FF00907AF
S31508014268022767444FF4C87C0CFB0121012F98BF2C
S315080142780131B3F5997F12D3A3F59973E361002345
S31508014288A1F26C71E060C4E9047120462362BDE8B5
S31508014298F0810028A361A8DB90FBF1F1ABE712F0E6
S315080142A8030F02D106FB15255DB94FF4C875B2FB94
S315080142B8F5F605FB1622B2FA82F252093B33134484
S315080142C8DCE70122FAE700BF80510100B13A020092
S315080142D84FC5FDFFB03A0200014B1868704700BF89
S315080142E89000002070B500260C4D0D4C641BA410D7
S315080142F8A64209D102F004F900260A4D0A4C641BA4
S31508014308A410A64205D170BD55F8043B9847013655
S31508014318EEE755F8043B98470136F2E7EC700108D1
S31508014328EC700108EC700108F070010870477047D5
S315080143387047000000487047D0010020034610B5B1
S31508014348C9B202449342184601D1002003E0047811
S3150801435801338C42F6D110BD0A44914200F1FF336C
S3150801436800D1704710B511F8014B914203F8014F76
S31508014378F9D110BD1FB514461A46094B05461B68DF
S31508014388D8684CB1074BCDE9013400912B4606494B
S3150801439801F01EFE01F0E4FF044B1C46F3E700BFDB
S315080143A890000020BB6D0108C86D0108F66D01086B
S315080143B82DE9F74F03690C690746A3427EDB013CE1
S315080143C8A30000F1140501F11408009305EB840311
S315080143D8019358F8243055F8242001339A42B2FB40
S315080143E8F3F608EB84092ED34FF0000AC446AE4605
S315080143F8D3465CF8043B98B206FB00A01B0C020CDA
S3150801440806FB0323DEF8002080B292B2121A5A4438
S31508014418DEF800004FEA134A9BB2C3EB224303EBCB
S31508014428104392B242EA0342E1454FEA234B4EF85A
S31508014438042BDED2009BEB582BB9019B043B9D420A
S315080144481A462FD33C61384601F076FC002825DB4D
S315080144582946002058F8042BD1F800C01FFA82FE15
S315080144681FFA8CF3A3EB0E030344120CC2EB234287
S3150801447802EB1C429BB243EA0243C1454FEA22407A
S3150801448841F8043BE6D255F8242005EB840322B902
S31508014498043B9D421A460BD33C610136304603B0AC
S315080144A8BDE8F08F1268043B002ACBD1013CC6E768
S315080144B81268043B002AEFD1013CEAE70020EEE73F
S315080144C82DE9F04F14461D46C76997B08146CDE9CF
S315080144D80645239E7FB9102001F05EF80246C9F801
S315080144E81C0020B9EF21AC4BAC48FFF743FFC0E9E4
S315080144F801770760C760D9F81C30196859B15A6835
S31508014508012393404A608B60484601F0E3F900228B
S31508014518D9F81C301A602B1EAFBF0023012223F0DD
S3150801452800430793A8BF3360DDF81C809C4BB8BFCE
S31508014538326033EA080312D142F20F73229A1360E2
S31508014548C8F31303234300F05E85249BDFF854A2BE
S31508014558002B00F060850AF1030300F05ABDDDE976
S315080145680623CDE90C23DDE90C0100220023F4F723
S3150801457883FA074658B10123229A1360249B13B17B
S31508014588894B249A1360DFF824A200F044BD14ABC2
S31508014598019315AB00934846DDE90C2301F07CFC31
S315080145A8C8F30A560390002E78D0DDE90C010D9B55
S315080145B8A6F2FF36C3F3130343F07F5343F44013BC
S315080145C81297194600227A4BF3F736FE6CA3D3E9FC
S315080145D80023F3F7E9FF6CA3D3E90023F3F72EFECB
S315080145E8044630460D46F3F775FF69A3D3E9002358
S315080145F8F3F7DAFF02460B4620462946F3F71EFE6D
S3150801460804460D46F4F780FA002207460023204699
S315080146182946F4F73BFA40B13846F3F75BFF2246D9
S315080146282B46F4F729FA00B9013F162F54D8DDE9C4
S315080146380C01604B03EBC703D3E90023F4F726FA09
S3150801464800284BD00023013F0F93149B9B1B5A1E2E
S3150801465849BFC3F10103002304930023099254BFF8
S3150801466804930993002F3BDB099B0E973B44099357
S3150801467800230A93209B092B65D8052BC4BF043B45
S315080146882093209BC8BF0024A3F10203D8BF0124A5
S31508014698032B64D8DFE803F05355382CDDE9146396
S315080146A81E4406F23243202BC1BFC3F1400308FA60
S315080146B803F806F2124324FA03F3D6BFC3F120031B
S315080146C848EA030004FA03F0F3F7F4FE0122A1F11C
S315080146D8F873013E129274E70123B5E70F90B4E720
S315080146E8049BDB1B04937B420A9300230E93C1E7C1
S315080146F801230B93219B07EB030B0BF10103012BF9
S315080147080893B8BF012306E001230B93219B002BCD
S3150801471828DD9B46089300210422D9F81C0002F1DA
S3150801472814059D4226D94160484601F093F8824608
S31508014738002843D1024640F2AF111F4BD4E60023A5
S31508014748E3E70023D5E7012400230B9420934FF0D0
S31508014758FF3B00221223CDF820B02192DBE7012383
S315080147680B93F4E74FF0010B5B46CDF820B0CDF873
S3150801477884B0D0E701315200D1E700BFAFF300801A
S3150801478861436F63A787D23FB3C8608B288AC63F40
S31508014798FB799F501344D33F4C6D0108046E0108F9
S315080147A80000F07F006E0108296D0108286D0108CF
S315080147B80000F83F186F01085C6E0108D9F81C302B
S315080147C81860089B0E2B00F2A180002C00F09E8031
S315080147D8002F33DD9C4B07F00F0203EBC203F805E4
S315080147E8D3E90034CDE910344FEA271416D5DDE9A3
S315080147F80C01964B0326D3E90823F3F7FFFFCDE906
S31508014808060104F00F04914D54B9DDE91023DDE9D9
S315080148180601F3F7F3FFCDE9060128E00226F2E7D8
S31508014828E10708D5DDE91001D5E90023F3F7BCFE50
S31508014838CDE91001013664100835E5E700F0AF80C7
S31508014848DDE90C017C42804B04F00F0203EBC2033D
S31508014858D3E90023F3F7A8FE02260023CDE90601CA
S315080148687A4D2411002C40F08F80002BD3D1DDE935
S3150801487806450F9B002B00F0948000222046294606
S31508014888734BF4F703F9002800F08B80089B002B7B
S3150801489800F08780BBF1000F34DD20460022294647
S315080148A86C4BF3F781FE5C46CDE9060107F1FF3843
S315080148B801363046F3F70EFEDDE90623F3F774FEF3
S315080148C80022654BF3F7BAFC0546A1F15076002C90
S315080148D86AD1DDE906010022604BF3F7ADFC024611
S315080148E80B46CDE906232A463346F4F7EDF80028A0
S315080148F840F09882DDE906012A4606F10043F4F7F5
S31508014908C5F838BBDDE90C34CDE90634159B002B0F
S31508014918C0F257810E2F00F354814B4B03EBC703A3
S31508014928D3E90034CDE90434219B002B80F2E580D4
S31508014938089B002B00F3E1800CD1DDE90401002274
S31508014948464BF3F731FEDDE90623F4F7B3F80028F9
S3150801495800F0668200242546219B56466FEA03081D
S3150801496800272146484600F0B5FF002D00F0BD8016
S315080149782FB1AF4203D03946484600F0ABFF294666
S31508014988484600F0A7FFB0E0E20705D5D5E90023B8
S31508014998F3F70AFE012301366410083562E7022691
S315080149A865E7B846089C84E7274B0B9903EBC403CC
S315080149B853E902235444002954D000202849F3F71F
S315080149C81DFF33462A46F3F737FC5646CDE910014B
S315080149D8DDE90601F4F798F80546F3F77BFD024683
S315080149E80B46DDE90601F3F727FC02460B46303587
S315080149F8CDE90623DDE9102306F8015BF4F746F845
S31508014A08002872D1DDE9062300201149F3F714FCC1
S31508014A18DDE91023F4F73AF8002840F0B480A642F5
S31508014A283FF470AFDDE9100100220A4BF3F7BCFD2C
S31508014A380022CDE91001DDE90601064BF3F7B4FDBD
S31508014A48CDE90601C4E700BF186F0108F06E010831
S31508014A580000F03F0000244000001C4000001440FC
S31508014A680000E03F31462846F3F79EFD5646CDE954
S31508014A7810011394DDE90601F4F746F80546F3F73C
S31508014A8829FD02460B46DDE90601F3F7D5FB024681
S31508014A980B46303506F8015BA642CDE906234FF0E9
S31508014AA8000224D1DDE91001AE4BF3F7C7FB024634
S31508014AB80B46DDE90601F4F707F8002863D1DDE9B5
S31508014AC810230020A749F3F7B7FB02460B46DDE991
S31508014AD80601F3F7DBFF00283FF414AF139E731E94
S31508014AE8139316F8013C302BF8D047463BE09E4B0A
S31508014AF8F3F75AFDCDE90601BCE75646DDE9064551
S31508014B08DDE9042320462946F3F778FEF3F7FCFF87
S31508014B188046F3F7DFFCDDE90423F3F745FD024692
S31508014B280B4620462946F3F787FB08F13004089D0A
S31508014B3806F8014BA6EB0A04A54202460B4633D1F1
S31508014B48F3F77CFBDDE9042304460D46F3F7BCFFBE
S31508014B58C0B9DDE9042320462946F3F78DFF10B1CC
S31508014B6818F0010F0ED14846039900F0B3FE002349
S31508014B783370229B01371F60249B002B00F04B8260
S31508014B881E6048E2B84633461E4613F8012D392AEF
S31508014B9806D19A45F8D1302208F101088AF8002089
S31508014BA81A7801321A70A0E700226F4BF3F7FCFC5A
S31508014BB80022002304460D46F3F75EFF00289FD01E
S31508014BC8D1E70B9A002A00F0EA80209A012A00F315
S31508014BD8CD80129A002A00F0C18003F233430A9C59
S31508014BE8049E049A01211A440492099A48461A44C9
S31508014BF8099200F023FF054666B1099B002B09DDDA
S31508014C08B342A8BF3346049AF61AD21A0492099AE5
S31508014C18D31A09930A9B0BB30B9B002B00F0C6808A
S31508014C28002C00F0C08029462246484600F0BEFFFF
S31508014C38039A01460546484600F016FF0399804639
S31508014C48484600F047FE0A9B1B1B0A9300F0B180F1
S31508014C5841460A9A484600F0A9FF039001214846A9
S31508014C6800F0ECFE0E9B0446002B00F0D8811A468C
S31508014C780146484600F09AFF209B0446012B00F39B
S31508014C889F80069B002B40F09780079BC3F313036D
S31508014C98002B40F09380079B23F000431B0D1B054F
S31508014CA833B1049B01330493099B01330993012307
S31508014CB80A930E9B002B00F0B881236904EB830342
S31508014CC8186900F06FFEC0F12000099B184410F01E
S31508014CD81F0000F08280C0F12003042B73DD049BBA
S31508014CE8C0F11C0003440493099B06440344099331
S31508014CF8049B002B05DD1A464846039900F0B0FFC8
S31508014D080390099B002B05DD21461A46484600F003
S31508014D18A7FF04460F9B002B61D02146039801F093
S31508014D280BF800285BDA00230A224846039900F0A3
S31508014D38F3FD0B9B07F1FF380390002B00F07781F1
S31508014D48294600230A22484600F0E6FDBBF1000F72
S31508014D5805466FDC209B022B49DC6BE0149BC3F1EB
S31508014D6836033CE70000E03F00002440089B5C1E30
S31508014D780A9BA34209DB1C1B089B002BBFF630AF15
S31508014D88049B089A9E1A00232BE70A9B0E9AE31A94
S31508014D981A440A94049E0024089B0E9221E70A9C49
S31508014DA8049E0B9D28E7DDF80C8051E70A9A0399BA
S31508014DB850E7CDF80C8051E7002379E7069B77E79A
S31508014DC800230A9379E793D0049A1C331A44049268
S31508014DD8099A1E441A4409928AE70346F4E7089B86
S31508014DE8B846002B20DC9B46209B022B1EDDBBF117
S31508014DF8000F7FF4B1AD21465B460522484600F00F
S31508014E088BFD01460446039800F096FF00287FF7B4
S31508014E18A3AD5646312308F1010806F8013B9FE57B
S31508014E28B846089C2546F4E7DDF820B00B9B002B0D
S31508014E3800F00181002E05DD29463246484600F074
S31508014E480FFF05460A9B002B5CD04846696800F0A7
S31508014E5801FD064628B9024640F2EF21804BFFF7C5
S31508014E6843BB2A6905F10C01023292000C30FFF79F
S31508014E7873FA01223146484600F0F2FE2F460546E6
S31508014E880AF1010304930AEB0B030A93069B03F041
S31508014E9801030993049B2146039803F1FF3BFFF796
S31508014EA887FA034639463033069003980B9300F080
S31508014EB843FF2A4608902146484600F059FFC2682A
S31508014EC806460B9B02BB0146039800F035FF0246CE
S31508014ED80B9B31464846CDE90B3200F0FBFC209B7B
S31508014EE80C9A049E42EA0301099B19430B9B0DD1AF
S31508014EF8392B27D0089A002A01DD069B31338BF80E
S31508014F0800302EE52846B9E70122E2E70899002983
S31508014F1804DB209801430998014320D1002AEEDDD4
S31508014F28012203994846049300F09AFE2146039004
S31508014F3800F002FF0028049B02DCE0D1DA07DED57F
S31508014F48392BDAD139238BF8003033461E4616F841
S31508014F58012C013B392A4ED001321A7001E5002A83
S31508014F6803DD392BEED00133C9E7049A0A9902F809
S31508014F78013C8A4228D000230A220399484600F0B0
S31508014F88CBFCAF4203904FF000034FF00A023946B3
S31508014F98484607D100F0C0FC07460546049B01337D
S31508014FA8049377E700F0B8FC2946074600230A2246
S31508014FB8484600F0B1FC0546F0E7BBF1000FCCBF47
S31508014FC85E4601260027564401220399484604935A
S31508014FD800F046FE2146039000F0AEFE0028B4DC38
S31508014FE802D1049BDB07B0D433461E4613F8012DBC
S31508014FF8302AFAD0B5E49A45A8D1312308F101082F
S315080150088AF80030ADE4249BDFF858A01BB10AF1F1
S315080150180803249A1360504617B0BDE8F08F209B01
S31508015028012B7FF72EAE0E9B0A9301204DE6BBF1A5
S31508015038000F7FF7D9AE564621460398FFF7B8F908
S3150801504800F1300306F8013BA6EB0A029345B4DDE5
S3150801505800230A224846039900F05EFC0390EBE711
S315080150685C6E0108F76D01082DE9F0471F468E6841
S315080150788246BE420C4690460B682DD8B1F90C20DB
S3150801508812F4906F26D06569096905EB4505A3EB06
S31508015098010905EBD5757B1C4B446D109D4238BF3C
S315080150A81D46530527D5294600F0A0FA064660B3DA
S315080150B84A462169FFF750F9A38923F4906343F017
S315080150C88003A38126614E4426603E466561A5EBA9
S315080150D80905A560BE4200D93E46324641462068C2
S315080150E801F0ABF80020A3689B1BA360236833442F
S315080150F82360BDE8F0872A4600F07CFF06460028AB
S31508015108E0D15046216901F047F90C23CAF8003065
S31508015118A3894FF0FF3043F04003A381E9E7000074
S315080151282DE9F04F98468B8907461B060D46144606
S315080151389DB010D50B6973B9402100F057FA28605C
S31508015148286130B90C233B604FF0FF301DB0BDE82C
S31508015158F08F40236B610023099320238DF82930AA
S3150801516830234FF00109CDF80C80DFF898818DF8C6
S315080151782A3023469A4613F8012B0AB1252AF9D16A
S31508015188BAEB040B0BD05B46224629463846FFF78D
S315080151986BFF013000F0A780099A5A4409929AF8D8
S315080151A80030002B00F09F8000234FF0FF32CDE935
S315080151B805230AF1010A049307938DF853301A93C4
S315080151C85446052214F8011B4E48FFF7B7F8049A06
S315080151D8D8B9D00644BF20238DF85330110744BFE8
S315080151E82B238DF853309AF800302A2B15D05446BC
S315080151F800204FF00A0C079A214611F8013B303B6B
S31508015208092B4BD9B0B1079214E0A0EB080309FAA8
S3150801521803F31343A2460493D2E7039B191D1B689C
S315080152280391002BBBBF5B4242F002020793079327
S31508015238B8BF049223782E2B0AD163782A2B32D148
S31508015248039B02341A1D1B68039243EAE373059309
S31508015258DFF8B4A0032250462178FFF76FF838B172
S315080152684022049BA0EB0A008240134301340493AD
S3150801527814F8011B062225488DF82810FFF75EF851
S31508015288002836D0224B1BBB039B073323F00703A1
S3150801529808330393099B334409936AE70C460120AB
S315080152A80CFB0232A8E700234FF00A0C1946013411
S315080152B80593204610F8012B303A092A03D9002B01
S315080152C8C6D00591C4E7044601230CFB0121F0E782
S315080152D803AB00932A4638460E4B04A9FEF762FA31
S315080152E8421C0646D6D1AB895B063FF52DAF099810
S315080152F82CE703AB00932A463846064B04A9FEF762
S31508015308EFFCEDE76D6E0108736E0108776E01080B
S31508015318AD37010871500108936810B4013B002B99
S31508015328936007DA9469A34201DB0A2902D110BC02
S3150801533800F08EBE1368581C10601970084610BC18
S315080153487047F8B506460F461446D518AC4201D13A
S31508015358002007E03A46304614F8011BFFF7DCFF40
S31508015368431CF3D1F8BD00002DE9F04F0D4614464C
S31508015378984606469DB018B1036A0BB9FEF75AFE58
S315080153886B6ED90705D4AB899A0502D4A86DFEF7C1
S31508015398CEFFAB891B0701D52B699BB92946304630
S315080153A800F094FE70B16B6EDC0704D54FF0FF3040
S315080153B81DB0BDE8F08FAB899805F7D4A86DFEF73F
S315080153C8B7FFF3E70023099320238DF82930302303
S315080153D84FF00109CDF80C80DFF8A8818DF82A303D
S315080153E823469A4613F8012B0AB1252AF9D1BAEBAD
S315080153F8040B0BD05B46224629463046FFF7A1FF28
S31508015408013000F0A780099A5A4409929AF800309F
S31508015418002B00F09F8000234FF0FF32CDE90523CA
S315080154280AF1010A049307938DF853301A935446DF
S31508015438052214F8011B5348FEF780FF049AD8B9C8
S31508015448D10644BF20238DF85330130744BF2B23B5
S315080154588DF853309AF800302A2B15D05446002077
S315080154684FF00A0C079A214611F8013B303B092BE4
S315080154784BD9B0B1079214E0A0EB080309FA03F374
S315080154881343A2460493D2E7039B191D1B6803918C
S31508015498002BBBBF5B4242F0020207930793B8BFD2
S315080154A8049223782E2B0AD163782A2B32D1039BAF
S315080154B802341A1D1B68039243EAE3730593DFF85E
S315080154C8C8A0032250462178FEF738FF38B1402292
S315080154D8049BA0EB0A00824013430134049314F891
S315080154E8011B062229488DF82810FEF727FF0028F0
S315080154F83FD0274B1BBB039B073323F0070308330E
S315080155080393099B3B4409936AE70C4601200CFB64
S315080155180232A8E700234FF00A0C1946013405930D
S31508015528204610F8012B303A092A03D9002BC6D090
S315080155380591C4E7044601230CFB0121F0E703ABF7
S3150801554800932A463046134B04A9FEF72BF907465A
S31508015558781CD6D16B6ED90705D4AB899A0502D4BE
S31508015568A86DFEF7E5FEAB895B063FF51FAF0998FF
S315080155781EE703AB00932A463046064B04A9FEF7F5
S31508015588AFFBE4E76D6E0108736E0108776E0108D3
S31508015598AD3701084B530108024B0146186800F05C
S315080155A825B800BF9000002070B50F4E0C4631682B
S315080155B8054611B900F090FE30602146284600F0EC
S315080155C88BFE431C03D14FF0FF34204670BDC41C23
S315080155D824F00304A042F8D0211A284600F07CFEDC
S315080155E80130F2D1EFE700BFC81100202DE9F843D1
S315080155F8CD1C25F0030508350C2D38BF0C25002DC3
S31508015608064601DBA94204D90C2333600020BDE80C
S31508015618F883DFF8D48000F011F9D8F800301C4671
S3150801562844BB29463046FFF7BFFF431C044658D1F9
S31508015638D8F800402746002F43D1002C4BD02368C1
S315080156483946304604EB030900F046FE814542D146
S31508015658216830466D1A2946FFF7A6FF01303AD068
S3150801566823682B442360D8F800305A6862BBC8F807
S3150801567800700FE02268521B20D40B2A17D961192A
S31508015688A342256018BF5960636808BFC8F80010A7
S3150801569862514B60304600F0D7F804F10B00231D20
S315080156A820F00700C21A1CBF1B1AA350AFE762688D
S315080156B8A3420CBFC8F800205A60EBE72346646882
S315080156C8AEE73C467F68B6E71A465B68A342FBD154
S315080156D800235360DEE70C233046336000F0B4F844
S315080156E894E70560D6E700BFCC110020B1F90C2074
S315080156F8F8B5160705460C4654D44B68002B02DC48
S315080157080B6C002B48DDE66A002E45D0002312F4FF
S3150801571880522F68216A2B6030D0626DA389590798
S3150801572805D56368D21A636B0BB1236CD21A0023A9
S315080157382846E66A216AB047431CA38906D129681F
S315080157481D292BD8284ACA40D60727D500226260C0
S315080157582269D904226004D5421C01D12B6803B9F0
S315080157686065616B2F60B9B104F14403994202D0AF
S31508015778284600F011FE002363630DE0012328463D
S31508015788B0470246501CC9D12B68002BC6D01D2B21
S3150801579801D0162B1DD12F60002021E043F04003CC
S315080157A81BB21AE00F69002FF6D0930718BF00231A
S315080157B80E6808BF4B69F61B0F608B60002EEBDD80
S315080157C833463A462846216AD4F828C0E0470028CD
S315080157D807DCB4F90C3043F040034FF0FF30A381DE
S315080157E8F8BD0744361AE9E70100402038B50B69C0
S315080157F805460C4613B90025284638BD18B1036A6B
S315080158080BB9FEF717FCB4F90C30002BF3D0626E0E
S31508015818D00704D4990502D4A06DFEF788FD284659
S315080158282146FFF763FF636E0546DA07E4D4A389C1
S315080158389B05E1D4A06DFEF77BFDDDE70148FEF780
S3150801584876BD00BFC41100200148FEF771BD00BF2F
S31508015858C411002070B5C66904460D4676B91020EC
S31508015868FFF79AFE0246E06120B96B21174B1848E3
S31508015878FEF780FDC0E901660660C660E669F36859
S3150801588883B1E369DB6853F82500B8B9012101FA40
S3150801589805F6721D2046920000F069FD60B1C0E95F
S315080158A801560EE021220421204600F060FDE36935
S315080158B8F060DB68002BE4D1002070BD026843F86C
S315080158C825200023C0E90333F7E700BF4C6D01081B
S315080158D87E6E010870B5C66905460C4676B910206C
S315080158E8FFF75AFE0246E86120B98F21084B094895
S315080158F8FEF740FDC0E901660660C6603CB1EB6982
S315080159086268DB6853F82210216043F8224070BDAB
S315080159184C6D01087E6E01082DE9F04107460C46D3
S315080159281E4600200D6901F1140CDCF8003001301F
S3150801593899B202FB01611E0C0B0C02FB063389B2F4
S3150801594801EB034185424FEA13464CF8041BECDC8C
S315080159580EB3A368AB4219DC616838460131FFF713
S3150801596879FF804628B90246BA210C4B0C48FEF73E
S3150801597801FD226904F10C01023292000C30FEF78E
S31508015988EBFC21463846FFF7A5FF444604EB850399
S3150801599801355E6125612046BDE8F0815C6E010826
S315080159A87E6E01080346B0F5803F3ABF030410200E
S315080159B80020B3F1807F3CBF1B020830B3F1805F3A
S315080159C83CBF1B010430B3F1804F3CBF9B0002303A
S315080159D8002B05DB13F0804F00F1010008BF2020DA
S315080159E870470368024613F007000BD0D90721D47C
S315080159F8980749BF5B089B08012013605CBF022012
S31508015A081360704799B209B910201B0CD9B209B9A4
S31508015A1808301B0A190704BF1B090430990704BF74
S31508015A289B080230D90703D45B0800F1010003D0AB
S31508015A3813607047002070472020704710B50C4640
S31508015A480121FFF707FF024628B940F24511044B21
S31508015A580448FEF78FFC01234461036110BD00BFAA
S31508015A685C6E01087E6E01082DE9F04F17460A6932
S31508015A783B6989469A42A2BF3B460F4699463D6904
S31508015A88D9F810A0BB68796805EB0A06B34285B050
S31508015A98B8BF0131FFF7DEFE30B902464FF4B171DE
S31508015AA8404B4148FEF766FC00F1140423460022E0
S31508015AB804EB860E734520D307F1140809F114017E
S31508015AC808EB850501EB8A030293EB1B153B23F0CB
S31508015AD8030304331537BD4238BF04230193029BD8
S31508015AE803918B420CD8002E03DD5EF8043D002B8A
S31508015AF855D0066105B0BDE8F08F43F8042BD9E700
S31508015B08B1F800A0BAF1000F1FD0C446A146002774
S31508015B185CF8042BD9F800301FFA82FB9BB20AFB02
S31508015B280B333B44D9F80070120C3F0C0AFB02727E
S31508015B3802EB13429BB243EA024365454FEA124711
S31508015B4849F8043BE4D8019BE750039B0431B3F8B1
S31508015B580290B9F1000F20D04746A4464FF0000A33
S31508015B682368B7F800B0BCF802209BB209FB0B22E0
S31508015B78524443EA02434CF8043B57F8043B4FEABC
S31508015B88134ABCF80030BD4209FB0A3303EB12433A
S31508015B984FEA134AE5D8019AA35004349FE7013E10
S31508015BA8A1E700BF5C6E01087E6E01082DE9F8437E
S31508015BB8154612F0030207460E4607D0254C013A48
S31508015BC8002354F82220FFF7A7FE0646AD103DD05C
S31508015BD8FC697CB91020FFF7DFFC0246F86128B991
S31508015BE840F2B3111C4B1D48FEF7C4FBC0E901443A
S31508015BF80460C460D7F81C80D8F808404CB940F24C
S31508015C0871213846FFF71AFF00230446C8F8080029
S31508015C1803604FF00009EB070AD531462246384694
S31508015C28FFF722FF804631463846FFF753FE4646B8
S31508015C386D100BD0206838B9224621463846FFF739
S31508015C4813FF2060C0F800900446E4E73046BDE833
S31508015C58F88300BFE46E01084C6D01087E6E0108E1
S31508015C682DE9F0470C46074691462369496803EB2F
S31508015C786218A3684FEA621A08F10106B3420BDBF8
S31508015C883846FFF7E7FD054648B902464FF4EF716E
S31508015C98274B2848FEF76EFB01315B00EEE7002328
S31508015CA800F1140100F110021846534533DB206947
S31508015CB82AEAEA7A04F1140319F01F0901EB8A01A1
S31508015CC803EB800C2BD08A460022C9F1200E1868EE
S31508015CD800FA09F010434AF8040B53F8042B9C45BB
S31508015CE822FA0EF2F3D8ACEB0403153B23F00303AF
S31508015CF8043304F11500604588BF0423CA500AB164
S31508015D0808F10206013E384621462E61FFF7E2FDF3
S31508015D182846BDE8F08742F8040F0133C5E7043978
S31508015D2853F8042B9C4541F8042FF9D8EAE700BF34
S31508015D385C6E01087E6E010803460A69006930B57A
S31508015D48801A0ED11433143103EB820401EB820154
S31508015D5854F8045D51F8042D954203D005D24FF045
S31508015D68FF3030BDA342F3D3FBE70120F9E7000072
S31508015D782DE9F74F89460646114648461446FFF760
S31508015D88DBFF051E12D129463046FFF763FD024699
S31508015D9828B940F237213E4B3E48FEF7EBFA012374
S31508015DA8C0E90435104603B0BDE8F08FBCBF4B46C1
S31508015DB8A1463046D9F80410BABF1C460125002564
S31508015DC8FFF748FD024618B940F24521304BE3E78B
S31508015DD800F1140BD9F8107009F11003C5604FF0DA
S31508015DE8000C09F11405D946266904F1140E05EBC8
S31508015DF887080EEB86060193019B5EF8040B53F898
S31508015E0804AF81B201931FFA8AF35B1A000C634443
S31508015E18C0EB1A4000EB23409BB243EA00437645A0
S31508015E284FEA204C49F8043BE6D8331B153B23F0C7
S31508015E38030315340433A64238BF04231D445B44BF
S31508015E481E462C4644450ED308F10301491B21F089
S31508015E580301033DA84538BF00210B4453F8041D27
S31508015E6899B117619EE7E64654F8041B1FFA81FCA7
S31508015E78F444080C714400EB2C4089B241EA00410C
S31508015E884FEA204C46F8041BDCE7013FE6E700BF6A
S31508015E985C6E01087E6E01082DE97343012190465F
S31508015EA89946089EFFF7D6FC044630B9024640F2E1
S31508015EB80F31234B2348FEF75DFAC9F30A55C9F38F
S31508015EC813030DB143F480130193B8F1000324D0E9
S31508015ED868460093FFF785FDDDE90012D8B1C0F1E0
S31508015EE8200302FA03F30B43C24063610192019B43
S31508015EF8002B0CBF01220222A3612261ADB1A5F2D2
S31508015F08334505443560C0F13500099B18602046BC
S31508015F1802B0BDE870836161E9E701A8FFF761FD91
S31508015F28019B012263612030E7E7A0F2324004EBC6
S31508015F38820330601869FFF735FDC0EB4210E4E7C4
S31508015F485C6E01087E6E010810B50C46B1F90E1093
S31508015F5800F0B0F90028ABBF636DA3891B1823F4B9
S31508015F688053ACBF6365A38110BD2DE9F0411F4677
S31508015F788B890546DB050C46164605D502230022FC
S31508015F88B1F90E1000F084F9A389324623F4805337
S31508015F98A38128463B46B4F90E10BDE8F04100F046
S31508015FA8ABB910B50C46B1F90E1000F071F9431CDE
S31508015FB8A38915BF606523F4805343F48053A381ED
S31508015FC818BFA38110BDB1F90E1000F0A7B90000DA
S31508015FD80EB403B5014603AB054853F8042B00680C
S31508015FE80193FFF7C1F902B05DF804EB03B07047F6
S31508015FF8900000202DE9F041074614460D4621B9BF
S315080160081146BDE8F041FFF7F1BA2AB900F0C4F91B
S3150801601825462846BDE8F08100F018FA8442064666
S3150801602802D8B4EB500FF4D821463846FFF7DEFA02
S31508016038804608B94546ECE7B4422246294628BFB0
S315080160483246FEF789F92946384600F0A5F9F1E7F7
S31508016058F8B50E461446054618B1036A0BB9FDF795
S31508016068E9FFA369A360A3891A0701D5236943B977
S315080160782146284600F02AF818B14FF0FF37384666
S31508016088F8BD23682269F6B2981A636937468342C6
S3150801609805DC21462846FFF7A9FB0028EDD1A368A8
S315080160A8013BA36023685A1C22601E706269431C5F
S315080160B89A4204D0A389DB07E1D50A2EDFD1214606
S315080160C82846FFF793FB0028D9D0D6E738B5294BD8
S315080160D8054618680C4618B1036A0BB9FDF7AAFFF5
S315080160E8B4F90C30190722D4DA0607D409222A602A
S315080160F843F040034FF0FF30A38133E0580712D528
S31508016108616B41B104F14403994202D0284600F073
S3150801611843F900236363A38923F02403A381002396
S31508016128636023692360A38943F00803A38123696C
S315080161384BB9A38903F42073B3F5007F03D021462D
S31508016148284600F03EF8B4F90C3013F001020AD0DB
S315080161580022A26062695242A261226942B913F019
S315080161688000C5D138BD990758BF6269A260F4E7AE
S315080161780020F7E79000002070B50C46B1F90E101B
S31508016188154600291E4696B00CDAA389002113F094
S31508016198800F14BF40234FF48063002031602B60C1
S315080161A816B070BD6A4600F0C9F80028EDDB0199FA
S315080161B801F47041A1F50053594259414FF48063DE
S315080161C8EBE78B89F7B59D0706460C4607D504F113
S315080161D84703236023610123636103B0F0BD6A465F
S315080161E801ABFFF7C9FF009F054639463046FFF759
S315080161F8FDF948B9B4F90C309A05EED423F003032E
S3150801620843F00203A381E2E7A389C4E9040743F03B
S315080162188003A381019B20605BB13046B4F90E1057
S3150801622800F026F828B1A38923F0030343F00103F4
S31508016238A381A3891D43A581CFE7884210B501EB40
S31508016248020402D98442234607D8431EA14208D02C
S3150801625811F8012B03F8012FF8E7014602448A428F
S3150801626800D110BD13F8014D02F8014DF7E70000FA
S3150801627838B50023054D044608462B60F7F749FF4C
S31508016288431C02D12B6803B1236038BDD011002005
S3150801629838B50446084611460022054D2A601A46AD
S315080162A8F7F741FF431C02D12B6803B1236038BDB8
S315080162B8D011002038B50446084611460022054D76
S315080162C82A601A46F7F7EEFE431C02D12B6803B17A
S315080162D8236038BDD011002038B50023054D044682
S315080162E808462B60F7F72CFF431C02D12B6803B12C
S315080162F8236038BDD011002038B504460846114632
S315080163080022054D2A601A46F5F71AF8431C02D1E8
S315080163182B6803B1236038BDD011002038B5002396
S31508016328054D044608462B60F7F7D9FE431C02D1EA
S315080163382B6803B1236038BDD011002038B5002376
S31508016348064D0446084611462B60F7F7D3FE431C4B
S3150801635802D12B6803B1236038BD00BFD0110020D4
S31508016368062008B500F0B0F80120F7F790FE70B5D9
S31508016378A1FB025434B92946FFF738F9064628B964
S31508016388304670BD0C2200260260F9E72A462146E6
S31508016398FDF7D4FEF4E7000038B50546002940D0D4
S315080163A851F8043C0C1F002BB8BFE418FFF746FA4E
S315080163B81C4A136833B9636014602846BDE8384037
S315080163C8FFF742BAA34208D9206821188B4201BFB0
S315080163D819685B6809182160EDE71A465B680BB10D
S315080163E8A342FAD911685018A0420BD12068014472
S315080163F8501883421160E0D118685B680844106038
S315080164085360DAE702D90C232B60D6E720682118EE
S315080164188B4201BF19685B6809182160636054607B
S31508016428CBE738BDCC11002082B001B901A942B128
S315080164384BB113780B601278101E18BF012002B0F1
S3150801644870471046FBE76FF00100F8E751F8043C7E
S31508016458181F002BBCBF0B58C018704703460846BF
S3150801646841B1FF2A04D98A224FF0FF301A607047D2
S3150801647801200A7070471F2938B505460C4604D904
S31508016488162303604FF0FF3038BDC26B12B152F8BC
S3150801649821304BB9284600F031F8224601462846EC
S315080164A8BDE8384000F018B8012B0AD0591C03D1A9
S315080164B8162303600120E7E70021204642F8241045
S315080164C898470020E0E70000024B01461868FFF7E5
S315080164D8D2BF00BF9000002038B50023064D0446F8
S315080164E8084611462B60F7F7C2FD431C02D12B68F3
S315080164F803B1236038BD00BFD0110020F7F7B0BD3E
S31508016508F8B500BFF8BC08BC9E467047F8B500BF89
S30D08016518F8BC08BC9E46704759
S31508016520434F4E4E2564204572726F723A20256498
S315080165300A000000434F4E4E256420436861726786
S31508016540696E672046696E69736865643A0A000070
S315080165504368617267696E6720456E657267793A45
S315080165602025640A0000000042484D2054696D65E3
S315080165706F75740A000000005053552072656164F6
S31508016580792074696D656F75742C2073746F7070DA
S31508016590696E672E2E2E0A00505355206F6E207491
S315080165A0696D656F75742C2073746F7070696E6789
S315080165B02E2E2E0A0000000049736F6C6174696FF4
S315080165C06E207761726E696E670A00004375727292
S315080165D0656E74206C65616B6167652C20696E73E5
S315080165E0756C6174696F6E206572726F722C207397
S315080165F0746F7070696E672E2E2E0A0050535520DF
S315080166006F66662074696D656F75742C2073746F77
S315080166107070696E672E2E2E0A0000004556206995
S315080166206E666F3A0A0000004742545F766572202B
S315080166305625642E256425640A0000004261747497
S3150801664065727920747970653A2025640A0000001C
S3150801665042617474657279206361706163697479E2
S315080166603A2025640A000000426174746572792033
S31508016670766F6C746167653A2025640A000000002C
S31508016680426174746572792076656E646F723A2018
S31508016690252E34730A0000004261747465727920EC
S315080166A0534E3A20256C750A000000004261747445
S315080166B0657279206D616E756661637475726520A0
S315080166C0646174653A20253032642E253032642E91
S315080166D0253034640A0000004261747465727920B9
S315080166E06379636C65733A2025640A004F776E20D7
S315080166F06175746F3A2025640A0000004556494EB3
S315080167003A20252E3137730A0000000045565F539B
S31508016710575F5645523A20252E38730A0000000065
S3150801672042524D2054696D656F75740A0000000068
S315080167304261747465727920696E666F3A0A00005F
S315080167406D61784356202564560A00006D617843C9
S3150801675043202564410A0000746F74452025646B43
S3150801676057680A006D617854202564430A000000C1
S31508016770534F43202564700A00000000566F6C745D
S315080167802E202564560A00004243502054696D653F
S315080167906F75740A0000000042524F2054696D65F6
S315080167A06F75740A000000004556206E6F742072DA
S315080167B06561647920666F722061203630730A003C
S315080167C0505355206E6F742072656164792C20735D
S315080167D0746F7070696E672E2E2E0A0042434C2F15
S315080167E04243532F42534D2074696D656F75742C5E
S315080167F02073746F7070696E672E2E2E0A00000062
S315080168004C6F636B206572726F722C2073746F7094
S3150801681070696E672E2E2E0A00000000486F74708C
S315080168206C75672064657465637465642C2073747C
S315080168306F7070696E672E2E2E0A0000436F6E6E9A
S315080168406563746F72206F76657268656174202559
S31508016850642025642C2073746F7070696E672E2E00
S315080168602E0A00004253442054696D656F75740AF7
S315080168700000000044697361626C65640A000000E7
S315080168804368617267696E672073746172746564BF
S315080168900A00000057616974696E6720666F722085
S315080168A042484D0A0000000057616974696E672005
S315080168B0666F72205053552072656164790A00002B
S315080168C049736F6C6174696F6E20746573740A001D
S315080168D057616974696E6720666F722062617474A4
S315080168E065727920696E666F0A00000057616974DE
S315080168F0696E6720666F72206261747465727920A9
S315080169007374617475730A0057616974696E6720D7
S31508016910666F7220424D530A00000000496E697481
S3150801692069616C697A696E67206368617267657205
S315080169300A00000057616974696E6720666F7220E4
S3150801694042434C0A000000004368617267696E673A
S3150801695020696E2070726F67726573730A00000092
S315080169604368617267696E672053746F70706564F6
S315080169700A0000004368617267696E672053746F85
S31508016980707065642077697468204353440A00006F
S315080169904368617267696E67204572726F720A0091
S315080169A04368617267696E672046696E69736865CF
S315080169B0640A0000474254204572726F7220636F61
S315080169C064653A20307825580A000000436F6E6ED8
S315080169D06563746F723A20556E6B6E6F776E0A0037
S315080169E0436F6E6E6563746F723A20556E706C757F
S315080169F0676765640A000000436F6E6E6563746FAE
S31508016A00723A2044697361626C65640A0000000089
S31508016A10436F6E6E6563746F723A2050726570616A
S31508016A2072696E670A000000436F6E6E6563746F64
S31508016A30723A204175746852657175697265640A9E
S31508016A4000000000436F6E6E6563746F723A2057DB
S31508016A50616974696E67466F72456E657267790A10
S31508016A6000000000436F6E6E6563746F723A2043CF
S31508016A7068617267696E6750617573656445560A20
S31508016A8000000000436F6E6E6563746F723A2043AF
S31508016A9068617267696E67506175736564455653B7
S31508016AA0450A0000436F6E6E6563746F723A204340
S31508016AB068617267696E670A00000000436F6E6E4F
S31508016AC06563746F723A204175746854696D656FB0
S31508016AD075740A00436F6E6E6563746F723A204669
S31508016AE0696E69736865640A00000000436F6E6E1B
S31508016AF06563746F723A2046696E697368656445A1
S31508016B005653450A00000000436F6E6E6563746F45
S31508016B10723A2046696E697368656445560A0000CB
S31508016B20436F6E6E6563746F723A205265706C7549
S31508016B306767696E670A000042454D2052656365BD
S31508016B40697665642C20666F7263652073746F704D
S31508016B5070696E672E2E2E0A0000000042454D3AD6
S31508016B6020253032582025303258202530325820F9
S31508016B7025303258000000002025303258202530B3
S31508016B803258202530325820253032580A00000064
S31508016B904253542052656365697665642C20737483
S31508016BA06F7070696E672E2E2E0A00004253543A92
S31508016BB020253032582025303258202530325820A9
S31508016BC025303258000000004C6F636B20657272E5
S31508016BD06F720A004C6F636B206572726F72207256
S31508016BE0657365740A000000474254204368617260
S31508016BF0676572207625642E25640A0053657269D5
S31508016C00616C206E756D6265723A2025640A000012
S31508016C10426F617264207265766973696F6E3A2094
S31508016C2025640A0046572076657273696F6E3A20A5
S31508016C3025642E25642E25640A000000505355202C
S31508016C406F6E2074696D656F75740A00436F6E7493
S31508016C506163746F72206572726F722C2073746F20
S31508016C607070696E672E2E2E0A000000505355204B
S31508016C706F66662074696D656F75740A0000000099
S31508016C8053657420436F6E6669673A20257320251C
S31508016C90640A0000506F776572206C696D69743AF1
S31508016CA02025640A00000000436861726765207048
S31508016CB065726D69743A2025640A0005E09304003B
S31508016CC0000000000000000001020304060708098D
S31508016CD00000000001020304000004050607080974
S31508016CE000000000000D0000010203040506070864
S31508016CF0090A0B0C0D0E0F100000040506070809FA
S31508016D0000000000000D0000010203040506070843
S31508016D10090A0B0C0D0E0F10494E4600696E6600E6
S31508016D204E414E006E616E003000303132333435DB
S31508016D3036373839414243444546003031323334D7
S31508016D403536373839616263646566005245454EA2
S31508016D5054206D616C6C6F6320737563636565643C
S31508016D606564002F6275696C642F676E752D746F83
S31508016D706F6C732D666F722D73746D33325F313399
S31508016D802E332E72656C312E32303234303932362A
S31508016D902D313731352F7372632F6E65776C6962C2
S31508016DA02F6E65776C69622F6C6962632F74696DE2
S31508016DB0652F676D74696D652E63002C2066756E87
S31508016DC06374696F6E3A2000617373657274696FD3
S31508016DD06E2022257322206661696C65643A2066F5
S31508016DE0696C6520222573222C206C696E65202525
S31508016DF064257325730A00496E66696E697479009C
S31508016E004E614E002F6275696C642F676E752D741D
S31508016E106F6F6C732D666F722D73746D33325F31BC
S31508016E20332E332E72656C312E323032343039328C
S31508016E30362D313731352F7372632F6E65776C694D
S31508016E40622F6E65776C69622F6C6962632F737442
S31508016E50646C69622F64746F612E630042616C6CA5
S31508016E606F632073756363656564656400232D30FC
S31508016E702B2000686C4C00656667454647002F6203
S31508016E8075696C642F676E752D746F6F6C732D66DB
S31508016E906F722D73746D33325F31332E332E7265F3
S31508016EA06C312E32303234303932362D3137313574
S31508016EB02F7372632F6E65776C69622F6E65776CB7
S31508016EC069622F6C6962632F7374646C69622F6DD2
S31508016ED0707265632E63004300504F534958002E64
S31508016EE00000000005000000190000007D000000F8
S31508016EF00080E03779C34143176E05B5B5B89346A7
S31508016F00F5F93FE9034F384D321D30F94877825A72
S31508016F103CBF737FDD4F1575000000000000F03F90
S31508016F200000000000002440000000000000594055
S31508016F300000000000408F40000000000088C340A8
S31508016F4000000000006AF8400000000080842E411D
S31508016F5000000000D01263410000000084D7974169
S31508016F600000000065CDCD41000000205FA002426F
S31508016F70000000E876483742000000A2941A6D42E4
S31508016F80000040E59C30A2420000901EC4BCD642D7
S31508016F9000003426F56B0C430080E03779C3414382
S31508016FA000A0D8855734764300C84E676DC1AB43F8
S31508016FB0003D9160E458E143408CB5781DAF154416
S31508016FC050EFE2D6E41A4B4492D54D06CFF08044F1
S31508016FD0F64AE1C7022DB544B49DD9794378EA4406
S31508016FE0002020202020202020202828282828208A
S31508016FF02020202020202020202020202020202082
S3150801700020881010101010101010101010101010E9
S3150801701010040404040404040404041010101010D9
S3150801702010104141414141410101010101010101A3
S3150801703001010101010101010101010110101010F5
S315080170401010424242424242020202020202020275
S3150801705002020202020202020202020210101010C9
S3150801706020000000000000000000000000000000F1
S315080170700000000000000000000000000000000001
S3150801708000000000000000000000000000000000F1
S3150801709000000000000000000000000000000000E1
S315080170A000000000000000000000000000000000D1
S315080170B000000000000000000000000000000000C1
S315080170C000000000000000000000000000000000B1
S315080170D000000000000000000000000000000000A1
S309080170E0000000009D
S30D080170E44411FF7F01000000C1
S309080170EC0D820008FA
S309080170F0E98100081B
S315080170F4E4010000010164000000FF000000000033
S315080171040000000000000000400000320A3200407E
S3150801711400000000008000320A32000080000000EE
S315080171240000FA320A32000000FA000000FF0032B9
S315080171340A32000020000000FFFFFF320A3200FF76
S31508017144FFFF0000FF0000320A32002000000000A1
S3150801715400FFFF0000000000000000005255530123
S31508017164000000FE529E66000024F4001000000090
S315080171740100000000000000030000008810002040
S31508017184940000200000000088100020F010002060
S315080171945811002000000000000000000000000053
S315080171A400000000000000000000000000000000CC
S315080171B400000000000000000000000000000000BC
S315080171C400000000000000000000000000000000AC
S315080171D44300000000000000000000000000000059
S315080171E4000000000000000000000000000000008C
S315080171F44300000000000000000000000000000039
S31508017204000000000000000000000000000000006B
S315080172144300000000000000000000000000000018
S31508017224000000000000000000000000000000004B
S3150801723443000000000000000000000000000000F8
S31508017244000000000000000000000000000000002B
S3150801725443000000000000000000000000000000D8
S31508017264000000000000000000000000000000000B
S3150801727443000000000000000000000000000000B8
S3150801728400000000000000000000000000000000EB
S315080172944300000000000000000000000000000098
S315080172A400000000000000000000000000000000CB
S315080172B4656401083164010800000000E06F0108F3
S315080172C4DF6E0108F66D0108F66D0108F66D010811
S315080172D4F66D0108F66D0108F66D0108F66D0108EB
S315080172E4F66D0108F66D0108FFFFFFFFFFFFFFFFBB
S315080172F4FFFFFFFFFFFF0000010041534349490017
S31508017304000000000000000000000000000000006A
S3150801731400000000000000000000415343494900F1
S31508017324000000000000000000000000000000004A
S311080173340000000000000000000000003E
S7050800E7818A
